
internal_8MHz_W_SPI_CPP.elf:     file format elf32-littlearm

Sections:
Idx Name          Size      VMA       LMA       File off  Algn
  0 .text         000018ac  00000000  00000000  00010000  2**2
                  CONTENTS, ALLOC, LOAD, READONLY, CODE
  1 .ARM.exidx    00000008  000018ac  000018ac  000118ac  2**2
                  CONTENTS, ALLOC, LOAD, READONLY, DATA
  2 .relocate     00000854  20000000  000018b4  00020000  2**3
                  CONTENTS, ALLOC, LOAD, DATA
  3 .bss          000000c8  20000854  00002108  00020854  2**2
                  ALLOC
  4 .stack        00000404  2000091c  000021d0  00020854  2**0
                  ALLOC
  5 .ARM.attributes 00000028  00000000  00000000  00020854  2**0
                  CONTENTS, READONLY
  6 .comment      00000059  00000000  00000000  0002087c  2**0
                  CONTENTS, READONLY
  7 .debug_info   00025d49  00000000  00000000  000208d5  2**0
                  CONTENTS, READONLY, DEBUGGING
  8 .debug_abbrev 00002b9b  00000000  00000000  0004661e  2**0
                  CONTENTS, READONLY, DEBUGGING
  9 .debug_loc    0000b629  00000000  00000000  000491b9  2**0
                  CONTENTS, READONLY, DEBUGGING
 10 .debug_aranges 00000968  00000000  00000000  000547e2  2**0
                  CONTENTS, READONLY, DEBUGGING
 11 .debug_ranges 00000a78  00000000  00000000  0005514a  2**0
                  CONTENTS, READONLY, DEBUGGING
 12 .debug_macro  000192bd  00000000  00000000  00055bc2  2**0
                  CONTENTS, READONLY, DEBUGGING
 13 .debug_line   0000da35  00000000  00000000  0006ee7f  2**0
                  CONTENTS, READONLY, DEBUGGING
 14 .debug_str    00087ff7  00000000  00000000  0007c8b4  2**0
                  CONTENTS, READONLY, DEBUGGING
 15 .debug_frame  00001b98  00000000  00000000  001048ac  2**2
                  CONTENTS, READONLY, DEBUGGING

Disassembly of section .text:

00000000 <exception_table>:
       0:	20 0d 00 20 65 01 00 00 63 01 00 00 63 01 00 00      .. e...c...c...
	...
      2c:	63 01 00 00 00 00 00 00 00 00 00 00 63 01 00 00     c...........c...
      3c:	63 01 00 00 63 01 00 00 63 01 00 00 63 01 00 00     c...c...c...c...
      4c:	c9 08 00 00 63 01 00 00 63 01 00 00 63 01 00 00     ....c...c...c...
      5c:	63 01 00 00 63 01 00 00 63 01 00 00 63 01 00 00     c...c...c...c...
      6c:	63 01 00 00 63 01 00 00 00 00 00 00 00 00 00 00     c...c...........
      7c:	63 01 00 00 63 01 00 00 63 01 00 00 63 01 00 00     c...c...c...c...
      8c:	63 01 00 00 63 01 00 00 00 00 00 00 00 00 00 00     c...c...........
      9c:	63 01 00 00 63 01 00 00 63 01 00 00 63 01 00 00     c...c...c...c...
      ac:	63 01 00 00 00 00 00 00                             c.......

000000b4 <__do_global_dtors_aux>:
      b4:	b510      	push	{r4, lr}
      b6:	4c06      	ldr	r4, [pc, #24]	; (d0 <__do_global_dtors_aux+0x1c>)
      b8:	7823      	ldrb	r3, [r4, #0]
      ba:	2b00      	cmp	r3, #0
      bc:	d107      	bne.n	ce <__do_global_dtors_aux+0x1a>
      be:	4b05      	ldr	r3, [pc, #20]	; (d4 <__do_global_dtors_aux+0x20>)
      c0:	2b00      	cmp	r3, #0
      c2:	d002      	beq.n	ca <__do_global_dtors_aux+0x16>
      c4:	4804      	ldr	r0, [pc, #16]	; (d8 <__do_global_dtors_aux+0x24>)
      c6:	e000      	b.n	ca <__do_global_dtors_aux+0x16>
      c8:	bf00      	nop
      ca:	2301      	movs	r3, #1
      cc:	7023      	strb	r3, [r4, #0]
      ce:	bd10      	pop	{r4, pc}
      d0:	20000854 	.word	0x20000854
      d4:	00000000 	.word	0x00000000
      d8:	000018b4 	.word	0x000018b4

000000dc <frame_dummy>:
      dc:	4b08      	ldr	r3, [pc, #32]	; (100 <frame_dummy+0x24>)
      de:	b510      	push	{r4, lr}
      e0:	2b00      	cmp	r3, #0
      e2:	d003      	beq.n	ec <frame_dummy+0x10>
      e4:	4907      	ldr	r1, [pc, #28]	; (104 <frame_dummy+0x28>)
      e6:	4808      	ldr	r0, [pc, #32]	; (108 <frame_dummy+0x2c>)
      e8:	e000      	b.n	ec <frame_dummy+0x10>
      ea:	bf00      	nop
      ec:	4807      	ldr	r0, [pc, #28]	; (10c <frame_dummy+0x30>)
      ee:	6803      	ldr	r3, [r0, #0]
      f0:	2b00      	cmp	r3, #0
      f2:	d100      	bne.n	f6 <frame_dummy+0x1a>
      f4:	bd10      	pop	{r4, pc}
      f6:	4b06      	ldr	r3, [pc, #24]	; (110 <frame_dummy+0x34>)
      f8:	2b00      	cmp	r3, #0
      fa:	d0fb      	beq.n	f4 <frame_dummy+0x18>
      fc:	4798      	blx	r3
      fe:	e7f9      	b.n	f4 <frame_dummy+0x18>
     100:	00000000 	.word	0x00000000
     104:	20000858 	.word	0x20000858
     108:	000018b4 	.word	0x000018b4
     10c:	000018b4 	.word	0x000018b4
     110:	00000000 	.word	0x00000000

00000114 <atmel_start_init>:

/**
 * Initializes MCU, drivers and middleware in the project
 **/
void atmel_start_init(void)
{
     114:	b510      	push	{r4, lr}
	system_init();
     116:	4b01      	ldr	r3, [pc, #4]	; (11c <atmel_start_init+0x8>)
     118:	4798      	blx	r3
}
     11a:	bd10      	pop	{r4, pc}
     11c:	0000036d 	.word	0x0000036d

00000120 <_ZN5Color9set_colorEh>:
 */ 
#include "color.h"
#include "hal/include/hal_gpio.h"

void Color::set_color(const uint8_t color)
{
     120:	b5f0      	push	{r4, r5, r6, r7, lr}
	bool bit_on = false;
	for(uint8_t bit = 0; bit < 7; bit++){
     122:	2300      	movs	r3, #0
     124:	e007      	b.n	136 <_ZN5Color9set_colorEh+0x16>
	((Port *)hw)->Group[submodule_index].OUTCLR.reg = ~data;
}

static inline void hri_port_clear_OUT_reg(const void *const hw, uint8_t submodule_index, hri_port_out_reg_t mask)
{
	((Port *)hw)->Group[submodule_index].OUTCLR.reg = mask;
     126:	01d2      	lsls	r2, r2, #7
     128:	25c0      	movs	r5, #192	; 0xc0
     12a:	05ed      	lsls	r5, r5, #23
     12c:	46ac      	mov	ip, r5
     12e:	4462      	add	r2, ip
     130:	6154      	str	r4, [r2, #20]
     132:	3301      	adds	r3, #1
     134:	b2db      	uxtb	r3, r3
     136:	2b06      	cmp	r3, #6
     138:	dc12      	bgt.n	160 <_ZN5Color9set_colorEh+0x40>
		bit_on = (color & 0b1<<bit) > 0;
     13a:	2401      	movs	r4, #1
     13c:	0027      	movs	r7, r4
     13e:	409f      	lsls	r7, r3
		gpio_set_pin_level(RGB_pins[7-bit], bit_on);
     140:	2207      	movs	r2, #7
     142:	1ad2      	subs	r2, r2, r3
     144:	5c86      	ldrb	r6, [r0, r2]
 * \param[in] level true  = Pin level set to "high" state
 *                  false = Pin level set to "low" state
 */
static inline void gpio_set_pin_level(const uint8_t pin, const bool level)
{
	_gpio_set_level((enum gpio_port)GPIO_PORT(pin), 1U << GPIO_PIN(pin), level);
     146:	1172      	asrs	r2, r6, #5
     148:	251f      	movs	r5, #31
     14a:	4035      	ands	r5, r6
     14c:	40ac      	lsls	r4, r5
/**
 * \brief Set output level on port with mask
 */
static inline void _gpio_set_level(const enum gpio_port port, const uint32_t mask, const bool level)
{
	if (level) {
     14e:	420f      	tst	r7, r1
     150:	d0e9      	beq.n	126 <_ZN5Color9set_colorEh+0x6>
	((Port *)hw)->Group[submodule_index].OUTSET.reg = mask;
     152:	01d2      	lsls	r2, r2, #7
     154:	25c0      	movs	r5, #192	; 0xc0
     156:	05ed      	lsls	r5, r5, #23
     158:	46ac      	mov	ip, r5
     15a:	4462      	add	r2, ip
     15c:	6194      	str	r4, [r2, #24]
     15e:	e7e8      	b.n	132 <_ZN5Color9set_colorEh+0x12>
	}
}
     160:	bdf0      	pop	{r4, r5, r6, r7, pc}

00000162 <Dummy_Handler>:

/**
 * \brief Default interrupt handler for unused IRQs.
 */
void Dummy_Handler(void)
{
     162:	e7fe      	b.n	162 <Dummy_Handler>

00000164 <Reset_Handler>:
{
     164:	b5f8      	push	{r3, r4, r5, r6, r7, lr}
        if (pSrc != pDest) {
     166:	4a23      	ldr	r2, [pc, #140]	; (1f4 <Reset_Handler+0x90>)
     168:	4b23      	ldr	r3, [pc, #140]	; (1f8 <Reset_Handler+0x94>)
     16a:	429a      	cmp	r2, r3
     16c:	d009      	beq.n	182 <Reset_Handler+0x1e>
     16e:	4b22      	ldr	r3, [pc, #136]	; (1f8 <Reset_Handler+0x94>)
     170:	4a20      	ldr	r2, [pc, #128]	; (1f4 <Reset_Handler+0x90>)
     172:	e003      	b.n	17c <Reset_Handler+0x18>
                        *pDest++ = *pSrc++;
     174:	6811      	ldr	r1, [r2, #0]
     176:	6019      	str	r1, [r3, #0]
     178:	3304      	adds	r3, #4
     17a:	3204      	adds	r2, #4
                for (; pDest < &_erelocate;) {
     17c:	491f      	ldr	r1, [pc, #124]	; (1fc <Reset_Handler+0x98>)
     17e:	428b      	cmp	r3, r1
     180:	d3f8      	bcc.n	174 <Reset_Handler+0x10>
                        *pDest++ = *pSrc++;
     182:	4b1f      	ldr	r3, [pc, #124]	; (200 <Reset_Handler+0x9c>)
     184:	e002      	b.n	18c <Reset_Handler+0x28>
                *pDest++ = 0;
     186:	2200      	movs	r2, #0
     188:	601a      	str	r2, [r3, #0]
     18a:	3304      	adds	r3, #4
        for (pDest = &_szero; pDest < &_ezero;) {
     18c:	4a1d      	ldr	r2, [pc, #116]	; (204 <Reset_Handler+0xa0>)
     18e:	4293      	cmp	r3, r2
     190:	d3f9      	bcc.n	186 <Reset_Handler+0x22>
        SCB->VTOR = ((uint32_t) pSrc & SCB_VTOR_TBLOFF_Msk);
     192:	4a1d      	ldr	r2, [pc, #116]	; (208 <Reset_Handler+0xa4>)
     194:	21ff      	movs	r1, #255	; 0xff
     196:	4b1d      	ldr	r3, [pc, #116]	; (20c <Reset_Handler+0xa8>)
     198:	438b      	bics	r3, r1
     19a:	6093      	str	r3, [r2, #8]
        SBMATRIX->SFR[SBMATRIX_SLAVE_HMCRAMC0].reg = 2;
     19c:	39fd      	subs	r1, #253	; 0xfd
     19e:	2390      	movs	r3, #144	; 0x90
     1a0:	005b      	lsls	r3, r3, #1
     1a2:	4a1b      	ldr	r2, [pc, #108]	; (210 <Reset_Handler+0xac>)
     1a4:	50d1      	str	r1, [r2, r3]
        USB->DEVICE.QOSCTRL.bit.CQOS = 2;
     1a6:	4a1b      	ldr	r2, [pc, #108]	; (214 <Reset_Handler+0xb0>)
     1a8:	78d3      	ldrb	r3, [r2, #3]
     1aa:	2503      	movs	r5, #3
     1ac:	43ab      	bics	r3, r5
     1ae:	2402      	movs	r4, #2
     1b0:	4323      	orrs	r3, r4
     1b2:	70d3      	strb	r3, [r2, #3]
        USB->DEVICE.QOSCTRL.bit.DQOS = 2;
     1b4:	78d3      	ldrb	r3, [r2, #3]
     1b6:	270c      	movs	r7, #12
     1b8:	43bb      	bics	r3, r7
     1ba:	2608      	movs	r6, #8
     1bc:	4333      	orrs	r3, r6
     1be:	70d3      	strb	r3, [r2, #3]
        DMAC->QOSCTRL.bit.DQOS = 2;
     1c0:	4b15      	ldr	r3, [pc, #84]	; (218 <Reset_Handler+0xb4>)
     1c2:	7b98      	ldrb	r0, [r3, #14]
     1c4:	2230      	movs	r2, #48	; 0x30
     1c6:	4390      	bics	r0, r2
     1c8:	2220      	movs	r2, #32
     1ca:	4310      	orrs	r0, r2
     1cc:	7398      	strb	r0, [r3, #14]
        DMAC->QOSCTRL.bit.FQOS = 2;
     1ce:	7b99      	ldrb	r1, [r3, #14]
     1d0:	43b9      	bics	r1, r7
     1d2:	4331      	orrs	r1, r6
     1d4:	7399      	strb	r1, [r3, #14]
        DMAC->QOSCTRL.bit.WRBQOS = 2;
     1d6:	7b9a      	ldrb	r2, [r3, #14]
     1d8:	43aa      	bics	r2, r5
     1da:	4322      	orrs	r2, r4
     1dc:	739a      	strb	r2, [r3, #14]
        NVMCTRL->CTRLB.bit.MANW = 1;
     1de:	4a0f      	ldr	r2, [pc, #60]	; (21c <Reset_Handler+0xb8>)
     1e0:	6851      	ldr	r1, [r2, #4]
     1e2:	2380      	movs	r3, #128	; 0x80
     1e4:	430b      	orrs	r3, r1
     1e6:	6053      	str	r3, [r2, #4]
        __libc_init_array();
     1e8:	4b0d      	ldr	r3, [pc, #52]	; (220 <Reset_Handler+0xbc>)
     1ea:	4798      	blx	r3
        main();
     1ec:	4b0d      	ldr	r3, [pc, #52]	; (224 <Reset_Handler+0xc0>)
     1ee:	4798      	blx	r3
     1f0:	e7fe      	b.n	1f0 <Reset_Handler+0x8c>
     1f2:	46c0      	nop			; (mov r8, r8)
     1f4:	000018b4 	.word	0x000018b4
     1f8:	20000000 	.word	0x20000000
     1fc:	20000854 	.word	0x20000854
     200:	20000854 	.word	0x20000854
     204:	2000091c 	.word	0x2000091c
     208:	e000ed00 	.word	0xe000ed00
     20c:	00000000 	.word	0x00000000
     210:	41007000 	.word	0x41007000
     214:	41005000 	.word	0x41005000
     218:	41004800 	.word	0x41004800
     21c:	41004000 	.word	0x41004000
     220:	00000ded 	.word	0x00000ded
     224:	00000c91 	.word	0x00000c91

00000228 <TIMER_0_init>:
 * \brief Timer initialization function
 *
 * Enables Timer peripheral, clocks and initializes Timer driver
 */
static void TIMER_0_init(void)
{
     228:	b510      	push	{r4, lr}
			peripheral = (uint32_t)_pm_get_ahb_index(module);
			PM->AHBMASK.reg |= 1 << peripheral;
		}
		break;
	case PM_BUS_APBA:
		PM->APBAMASK.reg |= 1 << peripheral;
     22a:	4a08      	ldr	r2, [pc, #32]	; (24c <TIMER_0_init+0x24>)
     22c:	6993      	ldr	r3, [r2, #24]
     22e:	2120      	movs	r1, #32
     230:	430b      	orrs	r3, r1
     232:	6193      	str	r3, [r2, #24]
}

static inline void hri_gclk_write_CLKCTRL_reg(const void *const hw, hri_gclk_clkctrl_reg_t data)
{
	GCLK_CRITICAL_SECTION_ENTER();
	((Gclk *)hw)->CLKCTRL.reg = data;
     234:	4a06      	ldr	r2, [pc, #24]	; (250 <TIMER_0_init+0x28>)
     236:	4b07      	ldr	r3, [pc, #28]	; (254 <TIMER_0_init+0x2c>)
     238:	805a      	strh	r2, [r3, #2]
	_pm_enable_bus_clock(PM_BUS_APBA, RTC);
	_gclk_enable_channel(RTC_GCLK_ID, CONF_GCLK_RTC_SRC);
	timer_init(&TIMER_0, RTC, _rtc_get_timer());
     23a:	4b07      	ldr	r3, [pc, #28]	; (258 <TIMER_0_init+0x30>)
     23c:	4798      	blx	r3
     23e:	0002      	movs	r2, r0
     240:	4906      	ldr	r1, [pc, #24]	; (25c <TIMER_0_init+0x34>)
     242:	4807      	ldr	r0, [pc, #28]	; (260 <TIMER_0_init+0x38>)
     244:	4b07      	ldr	r3, [pc, #28]	; (264 <TIMER_0_init+0x3c>)
     246:	4798      	blx	r3
}
     248:	bd10      	pop	{r4, pc}
     24a:	46c0      	nop			; (mov r8, r8)
     24c:	40000400 	.word	0x40000400
     250:	00004004 	.word	0x00004004
     254:	40000c00 	.word	0x40000c00
     258:	000008c5 	.word	0x000008c5
     25c:	40001400 	.word	0x40001400
     260:	200008d8 	.word	0x200008d8
     264:	000006e5 	.word	0x000006e5

00000268 <SPI_0_PORT_init>:
{
     268:	b5f0      	push	{r4, r5, r6, r7, lr}
     26a:	46c6      	mov	lr, r8
     26c:	b500      	push	{lr}
	((Port *)hw)->Group[submodule_index].OUTCLR.reg = mask;
     26e:	22c0      	movs	r2, #192	; 0xc0
     270:	05d2      	lsls	r2, r2, #23
     272:	2310      	movs	r3, #16
     274:	6153      	str	r3, [r2, #20]
	((Port *)hw)->Group[submodule_index].DIRSET.reg = mask;
     276:	6093      	str	r3, [r2, #8]

static inline void hri_port_write_WRCONFIG_reg(const void *const hw, uint8_t submodule_index,
                                               hri_port_wrconfig_reg_t data)
{
	PORT_CRITICAL_SECTION_ENTER();
	((Port *)hw)->Group[submodule_index].WRCONFIG.reg = data;
     278:	4b25      	ldr	r3, [pc, #148]	; (310 <SPI_0_PORT_init+0xa8>)
     27a:	4926      	ldr	r1, [pc, #152]	; (314 <SPI_0_PORT_init+0xac>)
     27c:	6299      	str	r1, [r3, #40]	; 0x28
     27e:	21c0      	movs	r1, #192	; 0xc0
     280:	0609      	lsls	r1, r1, #24
     282:	468c      	mov	ip, r1
     284:	6299      	str	r1, [r3, #40]	; 0x28
	tmp = ((Port *)hw)->Group[submodule_index].PINCFG[index].reg;
     286:	2044      	movs	r0, #68	; 0x44
     288:	5c19      	ldrb	r1, [r3, r0]
	tmp &= ~PORT_PINCFG_PMUXEN;
     28a:	2701      	movs	r7, #1
     28c:	43b9      	bics	r1, r7
	tmp |= value << PORT_PINCFG_PMUXEN_Pos;
     28e:	2601      	movs	r6, #1
     290:	4331      	orrs	r1, r6
     292:	b2c9      	uxtb	r1, r1
	((Port *)hw)->Group[submodule_index].PINCFG[index].reg = tmp;
     294:	5419      	strb	r1, [r3, r0]
	tmp = ((Port *)hw)->Group[submodule_index].PMUX[index].reg;
     296:	2132      	movs	r1, #50	; 0x32
     298:	5c58      	ldrb	r0, [r3, r1]
	tmp &= ~PORT_PMUX_PMUXE_Msk;
     29a:	250f      	movs	r5, #15
     29c:	43a8      	bics	r0, r5
	tmp |= PORT_PMUX_PMUXE(data);
     29e:	2403      	movs	r4, #3
     2a0:	46a0      	mov	r8, r4
     2a2:	4644      	mov	r4, r8
     2a4:	4320      	orrs	r0, r4
     2a6:	b2c0      	uxtb	r0, r0
	((Port *)hw)->Group[submodule_index].PMUX[index].reg = tmp;
     2a8:	5458      	strb	r0, [r3, r1]
	((Port *)hw)->Group[submodule_index].OUTCLR.reg = mask;
     2aa:	2020      	movs	r0, #32
     2ac:	6150      	str	r0, [r2, #20]
	((Port *)hw)->Group[submodule_index].DIRSET.reg = mask;
     2ae:	6090      	str	r0, [r2, #8]
	((Port *)hw)->Group[submodule_index].WRCONFIG.reg = data;
     2b0:	4819      	ldr	r0, [pc, #100]	; (318 <SPI_0_PORT_init+0xb0>)
     2b2:	6298      	str	r0, [r3, #40]	; 0x28
     2b4:	4660      	mov	r0, ip
     2b6:	6298      	str	r0, [r3, #40]	; 0x28
	tmp = ((Port *)hw)->Group[submodule_index].PINCFG[index].reg;
     2b8:	2045      	movs	r0, #69	; 0x45
     2ba:	4684      	mov	ip, r0
     2bc:	5c18      	ldrb	r0, [r3, r0]
	tmp &= ~PORT_PINCFG_PMUXEN;
     2be:	43b8      	bics	r0, r7
	tmp |= value << PORT_PINCFG_PMUXEN_Pos;
     2c0:	4330      	orrs	r0, r6
     2c2:	b2c0      	uxtb	r0, r0
	((Port *)hw)->Group[submodule_index].PINCFG[index].reg = tmp;
     2c4:	4664      	mov	r4, ip
     2c6:	5518      	strb	r0, [r3, r4]
	tmp = ((Port *)hw)->Group[submodule_index].PMUX[index].reg;
     2c8:	5c58      	ldrb	r0, [r3, r1]
	tmp &= ~PORT_PMUX_PMUXO_Msk;
     2ca:	3c36      	subs	r4, #54	; 0x36
     2cc:	4020      	ands	r0, r4
	tmp |= PORT_PMUX_PMUXO(data);
     2ce:	2430      	movs	r4, #48	; 0x30
     2d0:	46a4      	mov	ip, r4
     2d2:	4664      	mov	r4, ip
     2d4:	4320      	orrs	r0, r4
     2d6:	b2c0      	uxtb	r0, r0
	((Port *)hw)->Group[submodule_index].PMUX[index].reg = tmp;
     2d8:	5458      	strb	r0, [r3, r1]
	((Port *)hw)->Group[submodule_index].DIRCLR.reg = mask;
     2da:	310e      	adds	r1, #14
     2dc:	6051      	str	r1, [r2, #4]
	((Port *)hw)->Group[submodule_index].WRCONFIG.reg = data;
     2de:	4a0f      	ldr	r2, [pc, #60]	; (31c <SPI_0_PORT_init+0xb4>)
     2e0:	629a      	str	r2, [r3, #40]	; 0x28
     2e2:	4a0f      	ldr	r2, [pc, #60]	; (320 <SPI_0_PORT_init+0xb8>)
     2e4:	629a      	str	r2, [r3, #40]	; 0x28
	((Port *)hw)->Group[submodule_index].PINCFG[index].reg &= ~PORT_PINCFG_PULLEN;
     2e6:	2246      	movs	r2, #70	; 0x46
     2e8:	5c99      	ldrb	r1, [r3, r2]
     2ea:	2004      	movs	r0, #4
     2ec:	4381      	bics	r1, r0
     2ee:	5499      	strb	r1, [r3, r2]
	tmp = ((Port *)hw)->Group[submodule_index].PINCFG[index].reg;
     2f0:	5c99      	ldrb	r1, [r3, r2]
	tmp &= ~PORT_PINCFG_PMUXEN;
     2f2:	43b9      	bics	r1, r7
	tmp |= value << PORT_PINCFG_PMUXEN_Pos;
     2f4:	4331      	orrs	r1, r6
     2f6:	b2c9      	uxtb	r1, r1
	((Port *)hw)->Group[submodule_index].PINCFG[index].reg = tmp;
     2f8:	5499      	strb	r1, [r3, r2]
	tmp = ((Port *)hw)->Group[submodule_index].PMUX[index].reg;
     2fa:	2133      	movs	r1, #51	; 0x33
     2fc:	5c5a      	ldrb	r2, [r3, r1]
	tmp &= ~PORT_PMUX_PMUXE_Msk;
     2fe:	43aa      	bics	r2, r5
	tmp |= PORT_PMUX_PMUXE(data);
     300:	4640      	mov	r0, r8
     302:	4302      	orrs	r2, r0
     304:	b2d2      	uxtb	r2, r2
	((Port *)hw)->Group[submodule_index].PMUX[index].reg = tmp;
     306:	545a      	strb	r2, [r3, r1]
}
     308:	bc04      	pop	{r2}
     30a:	4690      	mov	r8, r2
     30c:	bdf0      	pop	{r4, r5, r6, r7, pc}
     30e:	46c0      	nop			; (mov r8, r8)
     310:	41004400 	.word	0x41004400
     314:	40000010 	.word	0x40000010
     318:	40000020 	.word	0x40000020
     31c:	40020040 	.word	0x40020040
     320:	c0020000 	.word	0xc0020000

00000324 <SPI_0_CLOCK_init>:
			peripheral = (uint32_t)_pm_get_apbb_index(module);
			PM->APBBMASK.reg |= 1 << peripheral;
		}
		break;
	case PM_BUS_APBC:
		PM->APBCMASK.reg |= 1 << peripheral;
     324:	4a04      	ldr	r2, [pc, #16]	; (338 <SPI_0_CLOCK_init+0x14>)
     326:	6a13      	ldr	r3, [r2, #32]
     328:	2104      	movs	r1, #4
     32a:	430b      	orrs	r3, r1
     32c:	6213      	str	r3, [r2, #32]
     32e:	4a03      	ldr	r2, [pc, #12]	; (33c <SPI_0_CLOCK_init+0x18>)
     330:	4b03      	ldr	r3, [pc, #12]	; (340 <SPI_0_CLOCK_init+0x1c>)
     332:	805a      	strh	r2, [r3, #2]
}
     334:	4770      	bx	lr
     336:	46c0      	nop			; (mov r8, r8)
     338:	40000400 	.word	0x40000400
     33c:	00004014 	.word	0x00004014
     340:	40000c00 	.word	0x40000c00

00000344 <SPI_0_init>:
{
     344:	b510      	push	{r4, lr}
	SPI_0_CLOCK_init();
     346:	4b04      	ldr	r3, [pc, #16]	; (358 <SPI_0_init+0x14>)
     348:	4798      	blx	r3
	spi_m_sync_init(&SPI_0, SERCOM0);
     34a:	4904      	ldr	r1, [pc, #16]	; (35c <SPI_0_init+0x18>)
     34c:	4804      	ldr	r0, [pc, #16]	; (360 <SPI_0_init+0x1c>)
     34e:	4b05      	ldr	r3, [pc, #20]	; (364 <SPI_0_init+0x20>)
     350:	4798      	blx	r3
	SPI_0_PORT_init();
     352:	4b05      	ldr	r3, [pc, #20]	; (368 <SPI_0_init+0x24>)
     354:	4798      	blx	r3
}
     356:	bd10      	pop	{r4, pc}
     358:	00000325 	.word	0x00000325
     35c:	42000800 	.word	0x42000800
     360:	200008c0 	.word	0x200008c0
     364:	00000511 	.word	0x00000511
     368:	00000269 	.word	0x00000269

0000036c <system_init>:

void system_init(void)
{
     36c:	b570      	push	{r4, r5, r6, lr}
 * Currently the following initialization functions are supported:
 *  - System clock initialization
 */
static inline void init_mcu(void)
{
	_init_chip();
     36e:	4b50      	ldr	r3, [pc, #320]	; (4b0 <STACK_SIZE+0xb0>)
     370:	4798      	blx	r3
	tmp = ((Port *)hw)->Group[submodule_index].PINCFG[index].reg;
     372:	4b50      	ldr	r3, [pc, #320]	; (4b4 <STACK_SIZE+0xb4>)
     374:	2040      	movs	r0, #64	; 0x40
     376:	5c1a      	ldrb	r2, [r3, r0]
	tmp &= ~PORT_PINCFG_PMUXEN;
     378:	2101      	movs	r1, #1
     37a:	438a      	bics	r2, r1
	((Port *)hw)->Group[submodule_index].PINCFG[index].reg = tmp;
     37c:	541a      	strb	r2, [r3, r0]
	tmp = ((Port *)hw)->Group[submodule_index].PINCFG[index].reg;
     37e:	3001      	adds	r0, #1
     380:	5c1a      	ldrb	r2, [r3, r0]
	tmp &= ~PORT_PINCFG_PMUXEN;
     382:	438a      	bics	r2, r1
	((Port *)hw)->Group[submodule_index].PINCFG[index].reg = tmp;
     384:	541a      	strb	r2, [r3, r0]
	((Port *)hw)->Group[submodule_index].OUTCLR.reg = mask;
     386:	22c0      	movs	r2, #192	; 0xc0
     388:	05d2      	lsls	r2, r2, #23
     38a:	383d      	subs	r0, #61	; 0x3d
     38c:	6150      	str	r0, [r2, #20]
	((Port *)hw)->Group[submodule_index].DIRSET.reg = mask;
     38e:	6090      	str	r0, [r2, #8]
	((Port *)hw)->Group[submodule_index].WRCONFIG.reg = data;
     390:	4849      	ldr	r0, [pc, #292]	; (4b8 <STACK_SIZE+0xb8>)
     392:	6298      	str	r0, [r3, #40]	; 0x28
     394:	20c0      	movs	r0, #192	; 0xc0
     396:	0600      	lsls	r0, r0, #24
     398:	6298      	str	r0, [r3, #40]	; 0x28
	tmp = ((Port *)hw)->Group[submodule_index].PINCFG[index].reg;
     39a:	2542      	movs	r5, #66	; 0x42
     39c:	5d5c      	ldrb	r4, [r3, r5]
	tmp &= ~PORT_PINCFG_PMUXEN;
     39e:	438c      	bics	r4, r1
	((Port *)hw)->Group[submodule_index].PINCFG[index].reg = tmp;
     3a0:	555c      	strb	r4, [r3, r5]
	((Port *)hw)->Group[submodule_index].OUTCLR.reg = mask;
     3a2:	2408      	movs	r4, #8
     3a4:	6154      	str	r4, [r2, #20]
	((Port *)hw)->Group[submodule_index].DIRSET.reg = mask;
     3a6:	6094      	str	r4, [r2, #8]
	((Port *)hw)->Group[submodule_index].WRCONFIG.reg = data;
     3a8:	4c44      	ldr	r4, [pc, #272]	; (4bc <STACK_SIZE+0xbc>)
     3aa:	629c      	str	r4, [r3, #40]	; 0x28
     3ac:	6298      	str	r0, [r3, #40]	; 0x28
	tmp = ((Port *)hw)->Group[submodule_index].PINCFG[index].reg;
     3ae:	3501      	adds	r5, #1
     3b0:	5d5c      	ldrb	r4, [r3, r5]
	tmp &= ~PORT_PINCFG_PMUXEN;
     3b2:	438c      	bics	r4, r1
	((Port *)hw)->Group[submodule_index].PINCFG[index].reg = tmp;
     3b4:	555c      	strb	r4, [r3, r5]
	((Port *)hw)->Group[submodule_index].OUTCLR.reg = mask;
     3b6:	2480      	movs	r4, #128	; 0x80
     3b8:	6154      	str	r4, [r2, #20]
	((Port *)hw)->Group[submodule_index].DIRSET.reg = mask;
     3ba:	6094      	str	r4, [r2, #8]
	((Port *)hw)->Group[submodule_index].WRCONFIG.reg = data;
     3bc:	4c40      	ldr	r4, [pc, #256]	; (4c0 <STACK_SIZE+0xc0>)
     3be:	629c      	str	r4, [r3, #40]	; 0x28
     3c0:	6298      	str	r0, [r3, #40]	; 0x28
	tmp = ((Port *)hw)->Group[submodule_index].PINCFG[index].reg;
     3c2:	3504      	adds	r5, #4
     3c4:	5d5c      	ldrb	r4, [r3, r5]
	tmp &= ~PORT_PINCFG_PMUXEN;
     3c6:	438c      	bics	r4, r1
	((Port *)hw)->Group[submodule_index].PINCFG[index].reg = tmp;
     3c8:	555c      	strb	r4, [r3, r5]
	((Port *)hw)->Group[submodule_index].OUTCLR.reg = mask;
     3ca:	2480      	movs	r4, #128	; 0x80
     3cc:	0064      	lsls	r4, r4, #1
     3ce:	6154      	str	r4, [r2, #20]
	((Port *)hw)->Group[submodule_index].DIRSET.reg = mask;
     3d0:	6094      	str	r4, [r2, #8]
	((Port *)hw)->Group[submodule_index].WRCONFIG.reg = data;
     3d2:	4c3c      	ldr	r4, [pc, #240]	; (4c4 <STACK_SIZE+0xc4>)
     3d4:	629c      	str	r4, [r3, #40]	; 0x28
     3d6:	6298      	str	r0, [r3, #40]	; 0x28
	tmp = ((Port *)hw)->Group[submodule_index].PINCFG[index].reg;
     3d8:	3501      	adds	r5, #1
     3da:	5d5c      	ldrb	r4, [r3, r5]
	tmp &= ~PORT_PINCFG_PMUXEN;
     3dc:	438c      	bics	r4, r1
	((Port *)hw)->Group[submodule_index].PINCFG[index].reg = tmp;
     3de:	555c      	strb	r4, [r3, r5]
	((Port *)hw)->Group[submodule_index].OUTCLR.reg = mask;
     3e0:	2480      	movs	r4, #128	; 0x80
     3e2:	00a4      	lsls	r4, r4, #2
     3e4:	6154      	str	r4, [r2, #20]
	((Port *)hw)->Group[submodule_index].DIRSET.reg = mask;
     3e6:	6094      	str	r4, [r2, #8]
	((Port *)hw)->Group[submodule_index].WRCONFIG.reg = data;
     3e8:	4c37      	ldr	r4, [pc, #220]	; (4c8 <STACK_SIZE+0xc8>)
     3ea:	629c      	str	r4, [r3, #40]	; 0x28
     3ec:	6298      	str	r0, [r3, #40]	; 0x28
	tmp = ((Port *)hw)->Group[submodule_index].PINCFG[index].reg;
     3ee:	3501      	adds	r5, #1
     3f0:	5d5c      	ldrb	r4, [r3, r5]
	tmp &= ~PORT_PINCFG_PMUXEN;
     3f2:	438c      	bics	r4, r1
	((Port *)hw)->Group[submodule_index].PINCFG[index].reg = tmp;
     3f4:	555c      	strb	r4, [r3, r5]
	((Port *)hw)->Group[submodule_index].OUTCLR.reg = mask;
     3f6:	2480      	movs	r4, #128	; 0x80
     3f8:	00e4      	lsls	r4, r4, #3
     3fa:	6154      	str	r4, [r2, #20]
	((Port *)hw)->Group[submodule_index].DIRSET.reg = mask;
     3fc:	6094      	str	r4, [r2, #8]
	((Port *)hw)->Group[submodule_index].WRCONFIG.reg = data;
     3fe:	4c33      	ldr	r4, [pc, #204]	; (4cc <STACK_SIZE+0xcc>)
     400:	629c      	str	r4, [r3, #40]	; 0x28
     402:	6298      	str	r0, [r3, #40]	; 0x28
	tmp = ((Port *)hw)->Group[submodule_index].PINCFG[index].reg;
     404:	3501      	adds	r5, #1
     406:	5d5c      	ldrb	r4, [r3, r5]
	tmp &= ~PORT_PINCFG_PMUXEN;
     408:	438c      	bics	r4, r1
	((Port *)hw)->Group[submodule_index].PINCFG[index].reg = tmp;
     40a:	555c      	strb	r4, [r3, r5]
	((Port *)hw)->Group[submodule_index].OUTCLR.reg = mask;
     40c:	2480      	movs	r4, #128	; 0x80
     40e:	0124      	lsls	r4, r4, #4
     410:	6154      	str	r4, [r2, #20]
	((Port *)hw)->Group[submodule_index].DIRSET.reg = mask;
     412:	6094      	str	r4, [r2, #8]
	((Port *)hw)->Group[submodule_index].WRCONFIG.reg = data;
     414:	4c2e      	ldr	r4, [pc, #184]	; (4d0 <STACK_SIZE+0xd0>)
     416:	629c      	str	r4, [r3, #40]	; 0x28
     418:	6298      	str	r0, [r3, #40]	; 0x28
	tmp = ((Port *)hw)->Group[submodule_index].PINCFG[index].reg;
     41a:	244b      	movs	r4, #75	; 0x4b
     41c:	5d18      	ldrb	r0, [r3, r4]
	tmp &= ~PORT_PINCFG_PMUXEN;
     41e:	4388      	bics	r0, r1
	((Port *)hw)->Group[submodule_index].PINCFG[index].reg = tmp;
     420:	5518      	strb	r0, [r3, r4]
	tmp = ((Port *)hw)->Group[submodule_index].PINCFG[index].reg;
     422:	3403      	adds	r4, #3
     424:	5d18      	ldrb	r0, [r3, r4]
	tmp &= ~PORT_PINCFG_PMUXEN;
     426:	4388      	bics	r0, r1
	((Port *)hw)->Group[submodule_index].PINCFG[index].reg = tmp;
     428:	5518      	strb	r0, [r3, r4]
	tmp = ((Port *)hw)->Group[submodule_index].PINCFG[index].reg;
     42a:	3401      	adds	r4, #1
     42c:	5d18      	ldrb	r0, [r3, r4]
	tmp &= ~PORT_PINCFG_PMUXEN;
     42e:	4388      	bics	r0, r1
	((Port *)hw)->Group[submodule_index].PINCFG[index].reg = tmp;
     430:	5518      	strb	r0, [r3, r4]
	((Port *)hw)->Group[submodule_index].OUTCLR.reg = mask;
     432:	2080      	movs	r0, #128	; 0x80
     434:	0240      	lsls	r0, r0, #9
     436:	6150      	str	r0, [r2, #20]
	((Port *)hw)->Group[submodule_index].DIRSET.reg = mask;
     438:	6090      	str	r0, [r2, #8]
	((Port *)hw)->Group[submodule_index].WRCONFIG.reg = data;
     43a:	2080      	movs	r0, #128	; 0x80
     43c:	05c0      	lsls	r0, r0, #23
     43e:	6298      	str	r0, [r3, #40]	; 0x28
     440:	4c24      	ldr	r4, [pc, #144]	; (4d4 <STACK_SIZE+0xd4>)
     442:	629c      	str	r4, [r3, #40]	; 0x28
	tmp = ((Port *)hw)->Group[submodule_index].PINCFG[index].reg;
     444:	3506      	adds	r5, #6
     446:	5d5c      	ldrb	r4, [r3, r5]
	tmp &= ~PORT_PINCFG_PMUXEN;
     448:	438c      	bics	r4, r1
	((Port *)hw)->Group[submodule_index].PINCFG[index].reg = tmp;
     44a:	555c      	strb	r4, [r3, r5]
	((Port *)hw)->Group[submodule_index].OUTCLR.reg = mask;
     44c:	2480      	movs	r4, #128	; 0x80
     44e:	02a4      	lsls	r4, r4, #10
     450:	6154      	str	r4, [r2, #20]
	((Port *)hw)->Group[submodule_index].DIRSET.reg = mask;
     452:	6094      	str	r4, [r2, #8]
	((Port *)hw)->Group[submodule_index].WRCONFIG.reg = data;
     454:	6298      	str	r0, [r3, #40]	; 0x28
     456:	4c20      	ldr	r4, [pc, #128]	; (4d8 <STACK_SIZE+0xd8>)
     458:	629c      	str	r4, [r3, #40]	; 0x28
	tmp = ((Port *)hw)->Group[submodule_index].PINCFG[index].reg;
     45a:	3501      	adds	r5, #1
     45c:	5d5c      	ldrb	r4, [r3, r5]
	tmp &= ~PORT_PINCFG_PMUXEN;
     45e:	438c      	bics	r4, r1
	((Port *)hw)->Group[submodule_index].PINCFG[index].reg = tmp;
     460:	555c      	strb	r4, [r3, r5]
	((Port *)hw)->Group[submodule_index].OUTCLR.reg = mask;
     462:	2480      	movs	r4, #128	; 0x80
     464:	02e4      	lsls	r4, r4, #11
     466:	6154      	str	r4, [r2, #20]
	((Port *)hw)->Group[submodule_index].DIRSET.reg = mask;
     468:	6094      	str	r4, [r2, #8]
	((Port *)hw)->Group[submodule_index].WRCONFIG.reg = data;
     46a:	6298      	str	r0, [r3, #40]	; 0x28
     46c:	4c1b      	ldr	r4, [pc, #108]	; (4dc <STACK_SIZE+0xdc>)
     46e:	629c      	str	r4, [r3, #40]	; 0x28
	tmp = ((Port *)hw)->Group[submodule_index].PINCFG[index].reg;
     470:	3501      	adds	r5, #1
     472:	5d5c      	ldrb	r4, [r3, r5]
	tmp &= ~PORT_PINCFG_PMUXEN;
     474:	438c      	bics	r4, r1
	((Port *)hw)->Group[submodule_index].PINCFG[index].reg = tmp;
     476:	555c      	strb	r4, [r3, r5]
	((Port *)hw)->Group[submodule_index].OUTCLR.reg = mask;
     478:	2480      	movs	r4, #128	; 0x80
     47a:	0324      	lsls	r4, r4, #12
     47c:	6154      	str	r4, [r2, #20]
	((Port *)hw)->Group[submodule_index].DIRSET.reg = mask;
     47e:	6094      	str	r4, [r2, #8]
	((Port *)hw)->Group[submodule_index].WRCONFIG.reg = data;
     480:	6298      	str	r0, [r3, #40]	; 0x28
     482:	4c17      	ldr	r4, [pc, #92]	; (4e0 <STACK_SIZE+0xe0>)
     484:	629c      	str	r4, [r3, #40]	; 0x28
	tmp = ((Port *)hw)->Group[submodule_index].PINCFG[index].reg;
     486:	3501      	adds	r5, #1
     488:	5d5c      	ldrb	r4, [r3, r5]
	tmp &= ~PORT_PINCFG_PMUXEN;
     48a:	438c      	bics	r4, r1
	((Port *)hw)->Group[submodule_index].PINCFG[index].reg = tmp;
     48c:	555c      	strb	r4, [r3, r5]
	((Port *)hw)->Group[submodule_index].OUTCLR.reg = mask;
     48e:	2480      	movs	r4, #128	; 0x80
     490:	03e4      	lsls	r4, r4, #15
     492:	6154      	str	r4, [r2, #20]
	((Port *)hw)->Group[submodule_index].DIRSET.reg = mask;
     494:	6094      	str	r4, [r2, #8]
	((Port *)hw)->Group[submodule_index].WRCONFIG.reg = data;
     496:	6298      	str	r0, [r3, #40]	; 0x28
     498:	4a12      	ldr	r2, [pc, #72]	; (4e4 <STACK_SIZE+0xe4>)
     49a:	629a      	str	r2, [r3, #40]	; 0x28
	tmp = ((Port *)hw)->Group[submodule_index].PINCFG[index].reg;
     49c:	2056      	movs	r0, #86	; 0x56
     49e:	5c1a      	ldrb	r2, [r3, r0]
	tmp &= ~PORT_PINCFG_PMUXEN;
     4a0:	438a      	bics	r2, r1
	((Port *)hw)->Group[submodule_index].PINCFG[index].reg = tmp;
     4a2:	541a      	strb	r2, [r3, r0]
	// Set pin direction to output
	gpio_set_pin_direction(VSYNC, GPIO_DIRECTION_OUT);

	gpio_set_pin_function(VSYNC, GPIO_PIN_FUNCTION_OFF);

	SPI_0_init();
     4a4:	4b10      	ldr	r3, [pc, #64]	; (4e8 <STACK_SIZE+0xe8>)
     4a6:	4798      	blx	r3

	TIMER_0_init();
     4a8:	4b10      	ldr	r3, [pc, #64]	; (4ec <STACK_SIZE+0xec>)
     4aa:	4798      	blx	r3
}
     4ac:	bd70      	pop	{r4, r5, r6, pc}
     4ae:	46c0      	nop			; (mov r8, r8)
     4b0:	000007dd 	.word	0x000007dd
     4b4:	41004400 	.word	0x41004400
     4b8:	40000004 	.word	0x40000004
     4bc:	40000008 	.word	0x40000008
     4c0:	40000080 	.word	0x40000080
     4c4:	40000100 	.word	0x40000100
     4c8:	40000200 	.word	0x40000200
     4cc:	40000400 	.word	0x40000400
     4d0:	40000800 	.word	0x40000800
     4d4:	c0000001 	.word	0xc0000001
     4d8:	c0000002 	.word	0xc0000002
     4dc:	c0000004 	.word	0xc0000004
     4e0:	c0000008 	.word	0xc0000008
     4e4:	c0000040 	.word	0xc0000040
     4e8:	00000345 	.word	0x00000345
     4ec:	00000229 	.word	0x00000229

000004f0 <delay_ms>:

/**
 * \brief Perform delay in ms
 */
void delay_ms(const uint16_t ms)
{
     4f0:	b510      	push	{r4, lr}
	_delay_cycles(hardware, _get_cycles_for_ms(ms));
     4f2:	4b04      	ldr	r3, [pc, #16]	; (504 <delay_ms+0x14>)
     4f4:	681c      	ldr	r4, [r3, #0]
     4f6:	4b04      	ldr	r3, [pc, #16]	; (508 <delay_ms+0x18>)
     4f8:	4798      	blx	r3
     4fa:	0001      	movs	r1, r0
     4fc:	0020      	movs	r0, r4
     4fe:	4b03      	ldr	r3, [pc, #12]	; (50c <delay_ms+0x1c>)
     500:	4798      	blx	r3
}
     502:	bd10      	pop	{r4, pc}
     504:	20000870 	.word	0x20000870
     508:	000007b5 	.word	0x000007b5
     50c:	000007d5 	.word	0x000007d5

00000510 <spi_m_sync_init>:
	ASSERT(spi);
	spi->func = (struct _spi_m_sync_hpl_interface *)func;
}

int32_t spi_m_sync_init(struct spi_m_sync_descriptor *spi, void *const hw)
{
     510:	b570      	push	{r4, r5, r6, lr}
     512:	0004      	movs	r4, r0
     514:	000d      	movs	r5, r1
	int32_t rc = 0;
	ASSERT(spi && hw);
     516:	2800      	cmp	r0, #0
     518:	d017      	beq.n	54a <spi_m_sync_init+0x3a>
     51a:	2900      	cmp	r1, #0
     51c:	d013      	beq.n	546 <spi_m_sync_init+0x36>
     51e:	2001      	movs	r0, #1
     520:	2240      	movs	r2, #64	; 0x40
     522:	490b      	ldr	r1, [pc, #44]	; (550 <spi_m_sync_init+0x40>)
     524:	4b0b      	ldr	r3, [pc, #44]	; (554 <spi_m_sync_init+0x44>)
     526:	4798      	blx	r3
	spi->dev.prvt = (void *)hw;
     528:	6065      	str	r5, [r4, #4]
	rc            = _spi_m_sync_init(&spi->dev, hw);
     52a:	1d20      	adds	r0, r4, #4
     52c:	0029      	movs	r1, r5
     52e:	4b0a      	ldr	r3, [pc, #40]	; (558 <spi_m_sync_init+0x48>)
     530:	4798      	blx	r3

	if (rc < 0) {
     532:	2800      	cmp	r0, #0
     534:	db06      	blt.n	544 <spi_m_sync_init+0x34>
		return rc;
	}

	spi->flags    = SPI_DEACTIVATE_NEXT;
     536:	4b09      	ldr	r3, [pc, #36]	; (55c <spi_m_sync_init+0x4c>)
     538:	82a3      	strh	r3, [r4, #20]
	spi->io.read  = _spi_m_sync_io_read;
     53a:	4b09      	ldr	r3, [pc, #36]	; (560 <spi_m_sync_init+0x50>)
     53c:	6123      	str	r3, [r4, #16]
	spi->io.write = _spi_m_sync_io_write;
     53e:	4b09      	ldr	r3, [pc, #36]	; (564 <spi_m_sync_init+0x54>)
     540:	60e3      	str	r3, [r4, #12]

	return ERR_NONE;
     542:	2000      	movs	r0, #0
}
     544:	bd70      	pop	{r4, r5, r6, pc}
	ASSERT(spi && hw);
     546:	2000      	movs	r0, #0
     548:	e7ea      	b.n	520 <spi_m_sync_init+0x10>
     54a:	2000      	movs	r0, #0
     54c:	e7e8      	b.n	520 <spi_m_sync_init+0x10>
     54e:	46c0      	nop			; (mov r8, r8)
     550:	000017a8 	.word	0x000017a8
     554:	00000729 	.word	0x00000729
     558:	000008ed 	.word	0x000008ed
     55c:	ffff8000 	.word	0xffff8000
     560:	000005ed 	.word	0x000005ed
     564:	000005b1 	.word	0x000005b1

00000568 <spi_m_sync_transfer>:

	return spi_m_sync_transfer(spi, &xfer);
}

int32_t spi_m_sync_transfer(struct spi_m_sync_descriptor *spi, const struct spi_xfer *p_xfer)
{
     568:	b530      	push	{r4, r5, lr}
     56a:	b087      	sub	sp, #28
     56c:	0004      	movs	r4, r0
     56e:	000d      	movs	r5, r1
	struct spi_msg msg;

	ASSERT(spi && p_xfer);
     570:	2800      	cmp	r0, #0
     572:	d015      	beq.n	5a0 <spi_m_sync_transfer+0x38>
     574:	2900      	cmp	r1, #0
     576:	d011      	beq.n	59c <spi_m_sync_transfer+0x34>
     578:	2001      	movs	r0, #1
     57a:	22b3      	movs	r2, #179	; 0xb3
     57c:	4909      	ldr	r1, [pc, #36]	; (5a4 <spi_m_sync_transfer+0x3c>)
     57e:	4b0a      	ldr	r3, [pc, #40]	; (5a8 <spi_m_sync_transfer+0x40>)
     580:	4798      	blx	r3

	msg.txbuf = p_xfer->txbuf;
     582:	682b      	ldr	r3, [r5, #0]
     584:	9303      	str	r3, [sp, #12]
	msg.rxbuf = p_xfer->rxbuf;
     586:	686b      	ldr	r3, [r5, #4]
     588:	9304      	str	r3, [sp, #16]
	msg.size  = p_xfer->size;
     58a:	68ab      	ldr	r3, [r5, #8]
     58c:	9301      	str	r3, [sp, #4]
     58e:	9305      	str	r3, [sp, #20]
	return _spi_m_sync_trans(&spi->dev, &msg);
     590:	1d20      	adds	r0, r4, #4
     592:	a903      	add	r1, sp, #12
     594:	4b05      	ldr	r3, [pc, #20]	; (5ac <spi_m_sync_transfer+0x44>)
     596:	4798      	blx	r3
}
     598:	b007      	add	sp, #28
     59a:	bd30      	pop	{r4, r5, pc}
	ASSERT(spi && p_xfer);
     59c:	2000      	movs	r0, #0
     59e:	e7ec      	b.n	57a <spi_m_sync_transfer+0x12>
     5a0:	2000      	movs	r0, #0
     5a2:	e7ea      	b.n	57a <spi_m_sync_transfer+0x12>
     5a4:	000017a8 	.word	0x000017a8
     5a8:	00000729 	.word	0x00000729
     5ac:	00000ae9 	.word	0x00000ae9

000005b0 <_spi_m_sync_io_write>:
{
     5b0:	b570      	push	{r4, r5, r6, lr}
     5b2:	b084      	sub	sp, #16
     5b4:	0004      	movs	r4, r0
     5b6:	000e      	movs	r6, r1
     5b8:	0015      	movs	r5, r2
	ASSERT(io);
     5ba:	1e43      	subs	r3, r0, #1
     5bc:	4198      	sbcs	r0, r3
     5be:	b2c0      	uxtb	r0, r0
     5c0:	22a3      	movs	r2, #163	; 0xa3
     5c2:	4907      	ldr	r1, [pc, #28]	; (5e0 <_spi_m_sync_io_write+0x30>)
     5c4:	4b07      	ldr	r3, [pc, #28]	; (5e4 <_spi_m_sync_io_write+0x34>)
     5c6:	4798      	blx	r3
	struct spi_m_sync_descriptor *spi = CONTAINER_OF(io, struct spi_m_sync_descriptor, io);
     5c8:	0020      	movs	r0, r4
     5ca:	380c      	subs	r0, #12
	xfer.rxbuf = 0;
     5cc:	2300      	movs	r3, #0
     5ce:	9302      	str	r3, [sp, #8]
	xfer.txbuf = (uint8_t *)buf;
     5d0:	9601      	str	r6, [sp, #4]
	xfer.size  = length;
     5d2:	9503      	str	r5, [sp, #12]
	return spi_m_sync_transfer(spi, &xfer);
     5d4:	a901      	add	r1, sp, #4
     5d6:	4b04      	ldr	r3, [pc, #16]	; (5e8 <_spi_m_sync_io_write+0x38>)
     5d8:	4798      	blx	r3
}
     5da:	b004      	add	sp, #16
     5dc:	bd70      	pop	{r4, r5, r6, pc}
     5de:	46c0      	nop			; (mov r8, r8)
     5e0:	000017a8 	.word	0x000017a8
     5e4:	00000729 	.word	0x00000729
     5e8:	00000569 	.word	0x00000569

000005ec <_spi_m_sync_io_read>:
{
     5ec:	b570      	push	{r4, r5, r6, lr}
     5ee:	b084      	sub	sp, #16
     5f0:	0004      	movs	r4, r0
     5f2:	000e      	movs	r6, r1
     5f4:	0015      	movs	r5, r2
	ASSERT(io);
     5f6:	1e43      	subs	r3, r0, #1
     5f8:	4198      	sbcs	r0, r3
     5fa:	b2c0      	uxtb	r0, r0
     5fc:	2287      	movs	r2, #135	; 0x87
     5fe:	4907      	ldr	r1, [pc, #28]	; (61c <_spi_m_sync_io_read+0x30>)
     600:	4b07      	ldr	r3, [pc, #28]	; (620 <_spi_m_sync_io_read+0x34>)
     602:	4798      	blx	r3
	struct spi_m_sync_descriptor *spi = CONTAINER_OF(io, struct spi_m_sync_descriptor, io);
     604:	0020      	movs	r0, r4
     606:	380c      	subs	r0, #12
	xfer.rxbuf = buf;
     608:	9602      	str	r6, [sp, #8]
	xfer.txbuf = 0;
     60a:	2300      	movs	r3, #0
     60c:	9301      	str	r3, [sp, #4]
	xfer.size  = length;
     60e:	9503      	str	r5, [sp, #12]
	return spi_m_sync_transfer(spi, &xfer);
     610:	a901      	add	r1, sp, #4
     612:	4b04      	ldr	r3, [pc, #16]	; (624 <_spi_m_sync_io_read+0x38>)
     614:	4798      	blx	r3
}
     616:	b004      	add	sp, #16
     618:	bd70      	pop	{r4, r5, r6, pc}
     61a:	46c0      	nop			; (mov r8, r8)
     61c:	000017a8 	.word	0x000017a8
     620:	00000729 	.word	0x00000729
     624:	00000569 	.word	0x00000569

00000628 <timer_add_timer_task>:
 * \param[in] head The pointer to the head of timer task list
 * \param[in] task The pointer to task to add
 * \param[in] time Current timer time
 */
static void timer_add_timer_task(struct list_descriptor *list, struct timer_task *const new_task, const uint32_t time)
{
     628:	b5f8      	push	{r3, r4, r5, r6, r7, lr}
 * \return A pointer to the head of the given list or NULL if the list is
 * empty
 */
static inline void *list_get_head(const struct list_descriptor *const list)
{
	return (void *)list->head;
     62a:	6806      	ldr	r6, [r0, #0]
	struct timer_task *it, *prev = NULL, *head = (struct timer_task *)list_get_head(list);

	if (!head) {
     62c:	2e00      	cmp	r6, #0
     62e:	d002      	beq.n	636 <timer_add_timer_task+0xe>
     630:	0033      	movs	r3, r6
     632:	2500      	movs	r5, #0
     634:	e00c      	b.n	650 <timer_add_timer_task+0x28>
		list_insert_as_head(list, new_task);
     636:	4b10      	ldr	r3, [pc, #64]	; (678 <timer_add_timer_task+0x50>)
     638:	4798      	blx	r3
		return;
     63a:	e018      	b.n	66e <timer_add_timer_task+0x46>
		uint32_t time_left;

		if (it->time_label <= time) {
			time_left = it->interval - (time - it->time_label);
		} else {
			time_left = it->interval - (0xFFFFFFFF - it->time_label) - time;
     63c:	689f      	ldr	r7, [r3, #8]
     63e:	46bc      	mov	ip, r7
     640:	4464      	add	r4, ip
     642:	1aa4      	subs	r4, r4, r2
     644:	3401      	adds	r4, #1
		}
		if (time_left >= new_task->interval)
     646:	688f      	ldr	r7, [r1, #8]
     648:	42bc      	cmp	r4, r7
     64a:	d20b      	bcs.n	664 <timer_add_timer_task+0x3c>
			break;
		prev = it;
     64c:	001d      	movs	r5, r3
	for (it = head; it; it = (struct timer_task *)list_get_next_element(it)) {
     64e:	681b      	ldr	r3, [r3, #0]
     650:	2b00      	cmp	r3, #0
     652:	d007      	beq.n	664 <timer_add_timer_task+0x3c>
		if (it->time_label <= time) {
     654:	685c      	ldr	r4, [r3, #4]
     656:	4294      	cmp	r4, r2
     658:	d8f0      	bhi.n	63c <timer_add_timer_task+0x14>
			time_left = it->interval - (time - it->time_label);
     65a:	1aa4      	subs	r4, r4, r2
     65c:	689f      	ldr	r7, [r3, #8]
     65e:	46bc      	mov	ip, r7
     660:	4464      	add	r4, ip
     662:	e7f0      	b.n	646 <timer_add_timer_task+0x1e>
	}

	if (it == head) {
     664:	42b3      	cmp	r3, r6
     666:	d003      	beq.n	670 <timer_add_timer_task+0x48>
		list_insert_as_head(list, new_task);
	} else {
		list_insert_after(prev, new_task);
     668:	0028      	movs	r0, r5
     66a:	4b04      	ldr	r3, [pc, #16]	; (67c <timer_add_timer_task+0x54>)
     66c:	4798      	blx	r3
	}
}
     66e:	bdf8      	pop	{r3, r4, r5, r6, r7, pc}
		list_insert_as_head(list, new_task);
     670:	4b01      	ldr	r3, [pc, #4]	; (678 <timer_add_timer_task+0x50>)
     672:	4798      	blx	r3
     674:	e7fb      	b.n	66e <timer_add_timer_task+0x46>
     676:	46c0      	nop			; (mov r8, r8)
     678:	00000749 	.word	0x00000749
     67c:	00000775 	.word	0x00000775

00000680 <timer_process_counted>:

/**
 * \internal Process interrupts
 */
static void timer_process_counted(struct _timer_device *device)
{
     680:	b5f8      	push	{r3, r4, r5, r6, r7, lr}
     682:	0005      	movs	r5, r0
     684:	6944      	ldr	r4, [r0, #20]
	struct timer_descriptor *timer = CONTAINER_OF(device, struct timer_descriptor, device);
	struct timer_task *      it    = (struct timer_task *)list_get_head(&timer->tasks);
	uint32_t                 time  = ++timer->time;
     686:	6903      	ldr	r3, [r0, #16]
     688:	1c5e      	adds	r6, r3, #1
     68a:	6106      	str	r6, [r0, #16]

	if ((timer->flags & TIMER_FLAG_QUEUE_IS_TAKEN) || (timer->flags & TIMER_FLAG_INTERRUPT_TRIGERRED)) {
     68c:	7e03      	ldrb	r3, [r0, #24]
     68e:	07db      	lsls	r3, r3, #31
     690:	d402      	bmi.n	698 <timer_process_counted+0x18>
     692:	7e03      	ldrb	r3, [r0, #24]
     694:	079b      	lsls	r3, r3, #30
     696:	d50a      	bpl.n	6ae <timer_process_counted+0x2e>
		timer->flags |= TIMER_FLAG_INTERRUPT_TRIGERRED;
     698:	7e2b      	ldrb	r3, [r5, #24]
     69a:	2202      	movs	r2, #2
     69c:	4313      	orrs	r3, r2
     69e:	b2db      	uxtb	r3, r3
     6a0:	762b      	strb	r3, [r5, #24]
		}
		it = (struct timer_task *)list_get_head(&timer->tasks);

		tmp->cb(tmp);
	}
}
     6a2:	bdf8      	pop	{r3, r4, r5, r6, r7, pc}
     6a4:	696f      	ldr	r7, [r5, #20]
		tmp->cb(tmp);
     6a6:	68e3      	ldr	r3, [r4, #12]
     6a8:	0020      	movs	r0, r4
     6aa:	4798      	blx	r3
		it = (struct timer_task *)list_get_head(&timer->tasks);
     6ac:	003c      	movs	r4, r7
	while (it && ((time - it->time_label) >= it->interval)) {
     6ae:	2c00      	cmp	r4, #0
     6b0:	d0f7      	beq.n	6a2 <timer_process_counted+0x22>
     6b2:	6863      	ldr	r3, [r4, #4]
     6b4:	1af3      	subs	r3, r6, r3
     6b6:	68a2      	ldr	r2, [r4, #8]
     6b8:	4293      	cmp	r3, r2
     6ba:	d3f2      	bcc.n	6a2 <timer_process_counted+0x22>
		list_remove_head(&timer->tasks);
     6bc:	002f      	movs	r7, r5
     6be:	3714      	adds	r7, #20
     6c0:	0038      	movs	r0, r7
     6c2:	4b06      	ldr	r3, [pc, #24]	; (6dc <timer_process_counted+0x5c>)
     6c4:	4798      	blx	r3
		if (TIMER_TASK_REPEAT == tmp->mode) {
     6c6:	7c23      	ldrb	r3, [r4, #16]
     6c8:	2b01      	cmp	r3, #1
     6ca:	d1eb      	bne.n	6a4 <timer_process_counted+0x24>
			tmp->time_label = time;
     6cc:	6066      	str	r6, [r4, #4]
			timer_add_timer_task(&timer->tasks, tmp, time);
     6ce:	0032      	movs	r2, r6
     6d0:	0021      	movs	r1, r4
     6d2:	0038      	movs	r0, r7
     6d4:	4b02      	ldr	r3, [pc, #8]	; (6e0 <timer_process_counted+0x60>)
     6d6:	4798      	blx	r3
     6d8:	e7e4      	b.n	6a4 <timer_process_counted+0x24>
     6da:	46c0      	nop			; (mov r8, r8)
     6dc:	0000077d 	.word	0x0000077d
     6e0:	00000629 	.word	0x00000629

000006e4 <timer_init>:
{
     6e4:	b570      	push	{r4, r5, r6, lr}
     6e6:	0004      	movs	r4, r0
     6e8:	000d      	movs	r5, r1
	ASSERT(descr && hw);
     6ea:	2800      	cmp	r0, #0
     6ec:	d012      	beq.n	714 <timer_init+0x30>
     6ee:	2900      	cmp	r1, #0
     6f0:	d00e      	beq.n	710 <timer_init+0x2c>
     6f2:	2001      	movs	r0, #1
     6f4:	223b      	movs	r2, #59	; 0x3b
     6f6:	4908      	ldr	r1, [pc, #32]	; (718 <timer_init+0x34>)
     6f8:	4b08      	ldr	r3, [pc, #32]	; (71c <timer_init+0x38>)
     6fa:	4798      	blx	r3
	_timer_init(&descr->device, hw);
     6fc:	0029      	movs	r1, r5
     6fe:	0020      	movs	r0, r4
     700:	4b07      	ldr	r3, [pc, #28]	; (720 <timer_init+0x3c>)
     702:	4798      	blx	r3
	descr->time                           = 0;
     704:	2300      	movs	r3, #0
     706:	6123      	str	r3, [r4, #16]
	descr->device.timer_cb.period_expired = timer_process_counted;
     708:	4b06      	ldr	r3, [pc, #24]	; (724 <timer_init+0x40>)
     70a:	6023      	str	r3, [r4, #0]
}
     70c:	2000      	movs	r0, #0
     70e:	bd70      	pop	{r4, r5, r6, pc}
	ASSERT(descr && hw);
     710:	2000      	movs	r0, #0
     712:	e7ef      	b.n	6f4 <timer_init+0x10>
     714:	2000      	movs	r0, #0
     716:	e7ed      	b.n	6f4 <timer_init+0x10>
     718:	000017c4 	.word	0x000017c4
     71c:	00000729 	.word	0x00000729
     720:	00000869 	.word	0x00000869
     724:	00000681 	.word	0x00000681

00000728 <assert>:
/**
 * \brief Assert function
 */
void assert(const bool condition, const char *const file, const int line)
{
	if (!(condition)) {
     728:	2800      	cmp	r0, #0
     72a:	d100      	bne.n	72e <assert+0x6>
		__asm("BKPT #0");
     72c:	be00      	bkpt	0x0000
	}
	(void)file;
	(void)line;
}
     72e:	4770      	bx	lr

00000730 <is_list_element>:
 * \brief Check whether element belongs to list
 */
bool is_list_element(const struct list_descriptor *const list, const void *const element)
{
	struct list_element *it;
	for (it = list->head; it; it = it->next) {
     730:	6803      	ldr	r3, [r0, #0]
     732:	2b00      	cmp	r3, #0
     734:	d003      	beq.n	73e <is_list_element+0xe>
		if (it == element) {
     736:	428b      	cmp	r3, r1
     738:	d003      	beq.n	742 <is_list_element+0x12>
	for (it = list->head; it; it = it->next) {
     73a:	681b      	ldr	r3, [r3, #0]
     73c:	e7f9      	b.n	732 <is_list_element+0x2>
			return true;
		}
	}

	return false;
     73e:	2000      	movs	r0, #0
}
     740:	4770      	bx	lr
			return true;
     742:	2001      	movs	r0, #1
     744:	e7fc      	b.n	740 <is_list_element+0x10>
	...

00000748 <list_insert_as_head>:

/**
 * \brief Insert an element as list head
 */
void list_insert_as_head(struct list_descriptor *const list, void *const element)
{
     748:	b570      	push	{r4, r5, r6, lr}
     74a:	0004      	movs	r4, r0
     74c:	000d      	movs	r5, r1
	ASSERT(!is_list_element(list, element));
     74e:	4b06      	ldr	r3, [pc, #24]	; (768 <list_insert_as_head+0x20>)
     750:	4798      	blx	r3
     752:	2301      	movs	r3, #1
     754:	4058      	eors	r0, r3
     756:	b2c0      	uxtb	r0, r0
     758:	2239      	movs	r2, #57	; 0x39
     75a:	4904      	ldr	r1, [pc, #16]	; (76c <list_insert_as_head+0x24>)
     75c:	4b04      	ldr	r3, [pc, #16]	; (770 <list_insert_as_head+0x28>)
     75e:	4798      	blx	r3

	((struct list_element *)element)->next = list->head;
     760:	6823      	ldr	r3, [r4, #0]
     762:	602b      	str	r3, [r5, #0]
	list->head                             = (struct list_element *)element;
     764:	6025      	str	r5, [r4, #0]
}
     766:	bd70      	pop	{r4, r5, r6, pc}
     768:	00000731 	.word	0x00000731
     76c:	000017dc 	.word	0x000017dc
     770:	00000729 	.word	0x00000729

00000774 <list_insert_after>:
/**
 * \brief Insert an element after the given list element
 */
void list_insert_after(void *const after, void *const element)
{
	((struct list_element *)element)->next = ((struct list_element *)after)->next;
     774:	6803      	ldr	r3, [r0, #0]
     776:	600b      	str	r3, [r1, #0]
	((struct list_element *)after)->next   = (struct list_element *)element;
     778:	6001      	str	r1, [r0, #0]
}
     77a:	4770      	bx	lr

0000077c <list_remove_head>:
/**
 * \brief Removes list head
 */
void *list_remove_head(struct list_descriptor *const list)
{
	if (list->head) {
     77c:	6803      	ldr	r3, [r0, #0]
     77e:	2b00      	cmp	r3, #0
     780:	d003      	beq.n	78a <list_remove_head+0xe>
		struct list_element *tmp = list->head;

		list->head = list->head->next;
     782:	681a      	ldr	r2, [r3, #0]
     784:	6002      	str	r2, [r0, #0]
		return (void *)tmp;
     786:	0018      	movs	r0, r3
	}

	return NULL;
}
     788:	4770      	bx	lr
	return NULL;
     78a:	2000      	movs	r0, #0
     78c:	e7fc      	b.n	788 <list_remove_head+0xc>
	...

00000790 <_sbrk>:

/**
 * \brief Replacement of C library of _sbrk
 */
extern caddr_t _sbrk(int incr)
{
     790:	0003      	movs	r3, r0
	static unsigned char *heap = NULL;
	unsigned char *       prev_heap;

	if (heap == NULL) {
     792:	4a06      	ldr	r2, [pc, #24]	; (7ac <_sbrk+0x1c>)
     794:	6812      	ldr	r2, [r2, #0]
     796:	2a00      	cmp	r2, #0
     798:	d004      	beq.n	7a4 <_sbrk+0x14>
		heap = (unsigned char *)&_end;
	}
	prev_heap = heap;
     79a:	4a04      	ldr	r2, [pc, #16]	; (7ac <_sbrk+0x1c>)
     79c:	6810      	ldr	r0, [r2, #0]

	heap += incr;
     79e:	18c3      	adds	r3, r0, r3
     7a0:	6013      	str	r3, [r2, #0]

	return (caddr_t)prev_heap;
}
     7a2:	4770      	bx	lr
		heap = (unsigned char *)&_end;
     7a4:	4902      	ldr	r1, [pc, #8]	; (7b0 <_sbrk+0x20>)
     7a6:	4a01      	ldr	r2, [pc, #4]	; (7ac <_sbrk+0x1c>)
     7a8:	6011      	str	r1, [r2, #0]
     7aa:	e7f6      	b.n	79a <_sbrk+0xa>
     7ac:	20000874 	.word	0x20000874
     7b0:	20000d20 	.word	0x20000d20

000007b4 <_get_cycles_for_ms>:

/**
 * \brief Retrieve the amount of cycles to delay for the given amount of ms
 */
uint32_t _get_cycles_for_ms(const uint16_t ms)
{
     7b4:	b510      	push	{r4, lr}
     7b6:	0003      	movs	r3, r0
		return (ms * (freq / 10000) + 2) / 3 * 10;
     7b8:	20c8      	movs	r0, #200	; 0xc8
     7ba:	0080      	lsls	r0, r0, #2
     7bc:	4358      	muls	r0, r3
     7be:	3002      	adds	r0, #2
     7c0:	2103      	movs	r1, #3
     7c2:	4b03      	ldr	r3, [pc, #12]	; (7d0 <_get_cycles_for_ms+0x1c>)
     7c4:	4798      	blx	r3
     7c6:	0083      	lsls	r3, r0, #2
     7c8:	181b      	adds	r3, r3, r0
     7ca:	0058      	lsls	r0, r3, #1
	return _get_cycles_for_ms_internal(ms, CONF_CPU_FREQUENCY, CPU_FREQ_POWER);
}
     7cc:	bd10      	pop	{r4, pc}
     7ce:	46c0      	nop			; (mov r8, r8)
     7d0:	00000cd5 	.word	0x00000cd5

000007d4 <_delay_cycles>:
{
#ifndef _UNIT_TEST_
	(void)hw;
	(void)cycles;
#if defined __GNUC__
	__asm(".syntax unified\n"
     7d4:	3901      	subs	r1, #1
     7d6:	d8fd      	bhi.n	7d4 <_delay_cycles>
	__asm("__delay:\n"
	      "subs r1, r1, #1\n"
	      "bhi __delay\n");
#endif
#endif
}
     7d8:	4770      	bx	lr
	...

000007dc <_init_chip>:

/**
 * \brief Initialize the hardware abstraction layer
 */
void _init_chip(void)
{
     7dc:	b510      	push	{r4, lr}
}

static inline void hri_nvmctrl_set_CTRLB_RWS_bf(const void *const hw, hri_nvmctrl_ctrlb_reg_t mask)
{
	NVMCTRL_CRITICAL_SECTION_ENTER();
	((Nvmctrl *)hw)->CTRLB.reg |= NVMCTRL_CTRLB_RWS(mask);
     7de:	4b06      	ldr	r3, [pc, #24]	; (7f8 <_init_chip+0x1c>)
     7e0:	685a      	ldr	r2, [r3, #4]
     7e2:	605a      	str	r2, [r3, #4]
	hri_nvmctrl_set_CTRLB_RWS_bf(NVMCTRL, CONF_NVM_WAIT_STATE);

	_pm_init();
     7e4:	4b05      	ldr	r3, [pc, #20]	; (7fc <_init_chip+0x20>)
     7e6:	4798      	blx	r3
	_sysctrl_init_sources();
     7e8:	4b05      	ldr	r3, [pc, #20]	; (800 <_init_chip+0x24>)
     7ea:	4798      	blx	r3
#if _GCLK_INIT_1ST
	_gclk_init_generators_by_fref(_GCLK_INIT_1ST);
#endif
	_sysctrl_init_referenced_generators();
     7ec:	4b05      	ldr	r3, [pc, #20]	; (804 <_init_chip+0x28>)
     7ee:	4798      	blx	r3
	_gclk_init_generators_by_fref(_GCLK_INIT_LAST);
     7f0:	20ff      	movs	r0, #255	; 0xff
     7f2:	4b05      	ldr	r3, [pc, #20]	; (808 <_init_chip+0x2c>)
     7f4:	4798      	blx	r3
#if CONF_DMAC_ENABLE
	_pm_enable_bus_clock(PM_BUS_AHB, DMAC);
	_pm_enable_bus_clock(PM_BUS_APBB, DMAC);
	_dma_init();
#endif
}
     7f6:	bd10      	pop	{r4, pc}
     7f8:	41004000 	.word	0x41004000
     7fc:	0000082d 	.word	0x0000082d
     800:	00000bfd 	.word	0x00000bfd
     804:	00000c41 	.word	0x00000c41
     808:	0000080d 	.word	0x0000080d

0000080c <_gclk_init_generators_by_fref>:

void _gclk_init_generators_by_fref(uint32_t bm)
{

#if CONF_GCLK_GENERATOR_0_CONFIG == 1
	if (bm & (1ul << 0)) {
     80c:	07c3      	lsls	r3, r0, #31
     80e:	d50a      	bpl.n	826 <_gclk_init_generators_by_fref+0x1a>
}

static inline void hri_gclk_write_GENDIV_reg(const void *const hw, hri_gclk_gendiv_reg_t data)
{
	GCLK_CRITICAL_SECTION_ENTER();
	((Gclk *)hw)->GENDIV.reg = data;
     810:	4b05      	ldr	r3, [pc, #20]	; (828 <_gclk_init_generators_by_fref+0x1c>)
     812:	2280      	movs	r2, #128	; 0x80
     814:	0052      	lsls	r2, r2, #1
     816:	609a      	str	r2, [r3, #8]
	((Gclk *)hw)->GENCTRL.reg = data;
     818:	2283      	movs	r2, #131	; 0x83
     81a:	0252      	lsls	r2, r2, #9
     81c:	605a      	str	r2, [r3, #4]
	while (((const Gclk *)hw)->STATUS.bit.SYNCBUSY)
     81e:	4b02      	ldr	r3, [pc, #8]	; (828 <_gclk_init_generators_by_fref+0x1c>)
     820:	785b      	ldrb	r3, [r3, #1]
     822:	09db      	lsrs	r3, r3, #7
     824:	d1fb      	bne.n	81e <_gclk_init_generators_by_fref+0x12>
		        | (CONF_GCLK_GEN_8_DIVSEL << GCLK_GENCTRL_DIVSEL_Pos) | (CONF_GCLK_GEN_8_OE << GCLK_GENCTRL_OE_Pos)
		        | (CONF_GCLK_GEN_8_OOV << GCLK_GENCTRL_OOV_Pos) | (CONF_GCLK_GEN_8_IDC << GCLK_GENCTRL_IDC_Pos)
		        | (CONF_GCLK_GENERATOR_8_CONFIG << GCLK_GENCTRL_GENEN_Pos) | CONF_GCLK_GEN_8_SRC | GCLK_GENCTRL_ID(8));
	}
#endif
}
     826:	4770      	bx	lr
     828:	40000c00 	.word	0x40000c00

0000082c <_pm_init>:
}

static inline void hri_pm_set_CPUSEL_CPUDIV_bf(const void *const hw, hri_pm_cpusel_reg_t mask)
{
	PM_CRITICAL_SECTION_ENTER();
	((Pm *)hw)->CPUSEL.reg |= PM_CPUSEL_CPUDIV(mask);
     82c:	4b06      	ldr	r3, [pc, #24]	; (848 <_pm_init+0x1c>)
     82e:	7a1a      	ldrb	r2, [r3, #8]
     830:	b2d2      	uxtb	r2, r2
     832:	721a      	strb	r2, [r3, #8]
}

static inline void hri_pm_set_APBASEL_APBADIV_bf(const void *const hw, hri_pm_apbasel_reg_t mask)
{
	PM_CRITICAL_SECTION_ENTER();
	((Pm *)hw)->APBASEL.reg |= PM_APBASEL_APBADIV(mask);
     834:	7a5a      	ldrb	r2, [r3, #9]
     836:	b2d2      	uxtb	r2, r2
     838:	725a      	strb	r2, [r3, #9]
}

static inline void hri_pm_set_APBBSEL_APBBDIV_bf(const void *const hw, hri_pm_apbbsel_reg_t mask)
{
	PM_CRITICAL_SECTION_ENTER();
	((Pm *)hw)->APBBSEL.reg |= PM_APBBSEL_APBBDIV(mask);
     83a:	7a9a      	ldrb	r2, [r3, #10]
     83c:	b2d2      	uxtb	r2, r2
     83e:	729a      	strb	r2, [r3, #10]
}

static inline void hri_pm_set_APBCSEL_APBCDIV_bf(const void *const hw, hri_pm_apbcsel_reg_t mask)
{
	PM_CRITICAL_SECTION_ENTER();
	((Pm *)hw)->APBCSEL.reg |= PM_APBCSEL_APBCDIV(mask);
     840:	7ada      	ldrb	r2, [r3, #11]
     842:	b2d2      	uxtb	r2, r2
     844:	72da      	strb	r2, [r3, #11]
{
	hri_pm_set_CPUSEL_CPUDIV_bf(PM, CONF_CPU_DIV);
	hri_pm_set_APBASEL_APBADIV_bf(PM, CONF_APBA_DIV);
	hri_pm_set_APBBSEL_APBBDIV_bf(PM, CONF_APBB_DIV);
	hri_pm_set_APBCSEL_APBCDIV_bf(PM, CONF_APBC_DIV);
}
     846:	4770      	bx	lr
     848:	40000400 	.word	0x40000400

0000084c <_rtc_timer_interrupt_handler>:
 * \brief RTC Timer interrupt handler
 *
 * \param[in] p The pointer to calendar device struct
 */
static void _rtc_timer_interrupt_handler(struct _timer_device *dev)
{
     84c:	b510      	push	{r4, lr}
     84e:	0004      	movs	r4, r0
	return tmp;
}

static inline hri_rtcmode0_intflag_reg_t hri_rtcmode0_read_INTFLAG_reg(const void *const hw)
{
	return ((Rtc *)hw)->MODE0.INTFLAG.reg;
     850:	68c3      	ldr	r3, [r0, #12]
     852:	7a1b      	ldrb	r3, [r3, #8]
	/* Read and mask interrupt flag register */
	uint16_t flag = hri_rtcmode0_read_INTFLAG_reg(dev->hw);

	if (flag & RTC_MODE0_INTFLAG_CMP0) {
     854:	07db      	lsls	r3, r3, #31
     856:	d506      	bpl.n	866 <_rtc_timer_interrupt_handler+0x1a>
		if (dev->timer_cb.period_expired) {
     858:	6803      	ldr	r3, [r0, #0]
     85a:	2b00      	cmp	r3, #0
     85c:	d000      	beq.n	860 <_rtc_timer_interrupt_handler+0x14>
			dev->timer_cb.period_expired(dev);
     85e:	4798      	blx	r3
		}

		/* Clear interrupt flag */
		hri_rtcmode0_clear_interrupt_CMP0_bit(dev->hw);
     860:	68e3      	ldr	r3, [r4, #12]
	((Rtc *)hw)->MODE0.INTFLAG.reg = RTC_MODE0_INTFLAG_CMP0;
     862:	2201      	movs	r2, #1
     864:	721a      	strb	r2, [r3, #8]
	}
}
     866:	bd10      	pop	{r4, pc}

00000868 <_timer_init>:
{
     868:	b570      	push	{r4, r5, r6, lr}
     86a:	0004      	movs	r4, r0
     86c:	000d      	movs	r5, r1
	ASSERT(dev);
     86e:	1e43      	subs	r3, r0, #1
     870:	4198      	sbcs	r0, r3
     872:	b2c0      	uxtb	r0, r0
     874:	2233      	movs	r2, #51	; 0x33
     876:	4910      	ldr	r1, [pc, #64]	; (8b8 <_timer_init+0x50>)
     878:	4b10      	ldr	r3, [pc, #64]	; (8bc <_timer_init+0x54>)
     87a:	4798      	blx	r3
	dev->hw = hw;
     87c:	60e5      	str	r5, [r4, #12]
}

static inline void hri_rtcmode0_write_CTRL_reg(const void *const hw, hri_rtcmode0_ctrl_reg_t data)
{
	RTC_CRITICAL_SECTION_ENTER();
	((Rtc *)hw)->MODE0.CTRL.reg = data;
     87e:	2301      	movs	r3, #1
     880:	802b      	strh	r3, [r5, #0]
	while (((const Rtc *)hw)->MODE0.STATUS.bit.SYNCBUSY)
     882:	7aab      	ldrb	r3, [r5, #10]
     884:	09db      	lsrs	r3, r3, #7
     886:	d1fc      	bne.n	882 <_timer_init+0x1a>
	hri_rtcmode0_wait_for_sync(dev->hw);
     888:	68e2      	ldr	r2, [r4, #12]
     88a:	7a93      	ldrb	r3, [r2, #10]
     88c:	09db      	lsrs	r3, r3, #7
     88e:	d1fc      	bne.n	88a <_timer_init+0x22>
	((Rtc *)hw)->MODE0.CTRL.reg = data;
     890:	3380      	adds	r3, #128	; 0x80
     892:	8013      	strh	r3, [r2, #0]
	while (((const Rtc *)hw)->MODE0.STATUS.bit.SYNCBUSY)
     894:	7a93      	ldrb	r3, [r2, #10]
     896:	09db      	lsrs	r3, r3, #7
     898:	d1fc      	bne.n	894 <_timer_init+0x2c>
	hri_rtcmode0_write_COMP_COMP_bf(dev->hw, 0, CONF_RTC_COMP_VAL);
     89a:	68e2      	ldr	r2, [r4, #12]

static inline void hri_rtcmode0_write_COMP_COMP_bf(const void *const hw, uint8_t index, hri_rtcmode0_comp_reg_t data)
{
	uint32_t tmp;
	RTC_CRITICAL_SECTION_ENTER();
	tmp = ((Rtc *)hw)->MODE0.COMP[index].reg;
     89c:	6993      	ldr	r3, [r2, #24]
	tmp &= ~RTC_MODE0_COMP_COMP_Msk;
	tmp |= RTC_MODE0_COMP_COMP(data);
	((Rtc *)hw)->MODE0.COMP[index].reg = tmp;
     89e:	2380      	movs	r3, #128	; 0x80
     8a0:	00db      	lsls	r3, r3, #3
     8a2:	6193      	str	r3, [r2, #24]
	while (((const Rtc *)hw)->MODE0.STATUS.bit.SYNCBUSY)
     8a4:	7a93      	ldrb	r3, [r2, #10]
     8a6:	09db      	lsrs	r3, r3, #7
     8a8:	d1fc      	bne.n	8a4 <_timer_init+0x3c>
	((Rtc *)hw)->MODE0.INTENSET.reg = RTC_MODE0_INTENSET_CMP0;
     8aa:	3301      	adds	r3, #1
     8ac:	68e2      	ldr	r2, [r4, #12]
     8ae:	71d3      	strb	r3, [r2, #7]
	_rtc_dev = dev;
     8b0:	4b03      	ldr	r3, [pc, #12]	; (8c0 <_timer_init+0x58>)
     8b2:	601c      	str	r4, [r3, #0]
}
     8b4:	2000      	movs	r0, #0
     8b6:	bd70      	pop	{r4, r5, r6, pc}
     8b8:	000017fc 	.word	0x000017fc
     8bc:	00000729 	.word	0x00000729
     8c0:	20000878 	.word	0x20000878

000008c4 <_rtc_get_timer>:
 * \brief Retrieve timer helper functions
 */
struct _timer_hpl_interface *_rtc_get_timer(void)
{
	return NULL;
}
     8c4:	2000      	movs	r0, #0
     8c6:	4770      	bx	lr

000008c8 <RTC_Handler>:

/**
 * \brief Rtc interrupt handler
 */
void RTC_Handler(void)
{
     8c8:	b510      	push	{r4, lr}
	_rtc_timer_interrupt_handler(_rtc_dev);
     8ca:	4b02      	ldr	r3, [pc, #8]	; (8d4 <RTC_Handler+0xc>)
     8cc:	6818      	ldr	r0, [r3, #0]
     8ce:	4b02      	ldr	r3, [pc, #8]	; (8d8 <RTC_Handler+0x10>)
     8d0:	4798      	blx	r3
}
     8d2:	bd10      	pop	{r4, pc}
     8d4:	20000878 	.word	0x20000878
     8d8:	0000084d 	.word	0x0000084d

000008dc <_sercom_get_hardware_index>:
{
#ifdef _UNIT_TEST_
	return ((uint32_t)hw - (uint32_t)SERCOM0) / sizeof(Sercom);
#endif

	return ((uint32_t)hw - (uint32_t)SERCOM0) >> 10;
     8dc:	4b02      	ldr	r3, [pc, #8]	; (8e8 <_sercom_get_hardware_index+0xc>)
     8de:	469c      	mov	ip, r3
     8e0:	4460      	add	r0, ip
     8e2:	0a80      	lsrs	r0, r0, #10
     8e4:	b2c0      	uxtb	r0, r0
}
     8e6:	4770      	bx	lr
     8e8:	bdfff800 	.word	0xbdfff800

000008ec <_spi_m_sync_init>:

	return NULL;
}

int32_t _spi_m_sync_init(struct _spi_m_sync_dev *dev, void *const hw)
{
     8ec:	b570      	push	{r4, r5, r6, lr}
     8ee:	0006      	movs	r6, r0
     8f0:	000c      	movs	r4, r1
	uint8_t n = _sercom_get_hardware_index((const void *)hw_addr);
     8f2:	0008      	movs	r0, r1
     8f4:	4b71      	ldr	r3, [pc, #452]	; (abc <_spi_m_sync_init+0x1d0>)
     8f6:	4798      	blx	r3
	for (i = 0; i < sizeof(sercomspi_regs) / sizeof(struct sercomspi_regs_cfg); i++) {
     8f8:	2300      	movs	r3, #0
     8fa:	2b00      	cmp	r3, #0
     8fc:	d100      	bne.n	900 <_spi_m_sync_init+0x14>
     8fe:	e084      	b.n	a0a <_spi_m_sync_init+0x11e>
	return NULL;
     900:	2500      	movs	r5, #0
	const struct sercomspi_regs_cfg *regs = _spi_get_regs((uint32_t)hw);

	ASSERT(dev && hw);
     902:	2e00      	cmp	r6, #0
     904:	d100      	bne.n	908 <_spi_m_sync_init+0x1c>
     906:	e08d      	b.n	a24 <_spi_m_sync_init+0x138>
     908:	2c00      	cmp	r4, #0
     90a:	d100      	bne.n	90e <_spi_m_sync_init+0x22>
     90c:	e088      	b.n	a20 <_spi_m_sync_init+0x134>
     90e:	2001      	movs	r0, #1
     910:	4a6b      	ldr	r2, [pc, #428]	; (ac0 <_spi_m_sync_init+0x1d4>)
     912:	496c      	ldr	r1, [pc, #432]	; (ac4 <_spi_m_sync_init+0x1d8>)
     914:	4b6c      	ldr	r3, [pc, #432]	; (ac8 <_spi_m_sync_init+0x1dc>)
     916:	4798      	blx	r3

	if (regs == NULL) {
     918:	2d00      	cmp	r5, #0
     91a:	d100      	bne.n	91e <_spi_m_sync_init+0x32>
     91c:	e0cb      	b.n	ab6 <_spi_m_sync_init+0x1ca>
	};
}

static inline bool hri_sercomspi_is_syncing(const void *const hw, hri_sercomspi_syncbusy_reg_t reg)
{
	return ((Sercom *)hw)->SPI.SYNCBUSY.reg & reg;
     91e:	69e3      	ldr	r3, [r4, #28]
		return ERR_INVALID_ARG;
	}

	if (!hri_sercomspi_is_syncing(hw, SERCOM_SPI_SYNCBUSY_SWRST)) {
     920:	07db      	lsls	r3, r3, #31
     922:	d421      	bmi.n	968 <_spi_m_sync_init+0x7c>
		uint32_t mode = regs->ctrla & SERCOM_SPI_CTRLA_MODE_Msk;
     924:	782a      	ldrb	r2, [r5, #0]
     926:	786b      	ldrb	r3, [r5, #1]
     928:	021b      	lsls	r3, r3, #8
     92a:	4313      	orrs	r3, r2
     92c:	78aa      	ldrb	r2, [r5, #2]
     92e:	0412      	lsls	r2, r2, #16
     930:	4313      	orrs	r3, r2
     932:	78ea      	ldrb	r2, [r5, #3]
     934:	0612      	lsls	r2, r2, #24
     936:	431a      	orrs	r2, r3
     938:	231c      	movs	r3, #28
     93a:	401a      	ands	r2, r3
	while (((Sercom *)hw)->SPI.SYNCBUSY.reg & reg) {
     93c:	69e3      	ldr	r3, [r4, #28]
     93e:	079b      	lsls	r3, r3, #30
     940:	d1fc      	bne.n	93c <_spi_m_sync_init+0x50>
static inline hri_sercomspi_ctrla_reg_t hri_sercomspi_get_CTRLA_reg(const void *const         hw,
                                                                    hri_sercomspi_ctrla_reg_t mask)
{
	uint32_t tmp;
	hri_sercomspi_wait_for_sync(hw, SERCOM_SPI_SYNCBUSY_SWRST | SERCOM_SPI_SYNCBUSY_ENABLE);
	tmp = ((Sercom *)hw)->SPI.CTRLA.reg;
     942:	6823      	ldr	r3, [r4, #0]
		if (hri_sercomspi_get_CTRLA_reg(hw, SERCOM_SPI_CTRLA_ENABLE)) {
     944:	079b      	lsls	r3, r3, #30
     946:	d509      	bpl.n	95c <_spi_m_sync_init+0x70>
	((Sercom *)hw)->SPI.CTRLA.reg &= ~SERCOM_SPI_CTRLA_ENABLE;
     948:	6823      	ldr	r3, [r4, #0]
     94a:	2102      	movs	r1, #2
     94c:	438b      	bics	r3, r1
     94e:	6023      	str	r3, [r4, #0]
	while (((Sercom *)hw)->SPI.SYNCBUSY.reg & reg) {
     950:	69e3      	ldr	r3, [r4, #28]
     952:	079b      	lsls	r3, r3, #30
     954:	d1fc      	bne.n	950 <_spi_m_sync_init+0x64>
     956:	69e3      	ldr	r3, [r4, #28]
     958:	079b      	lsls	r3, r3, #30
     95a:	d4fc      	bmi.n	956 <_spi_m_sync_init+0x6a>
			hri_sercomspi_clear_CTRLA_ENABLE_bit(hw);
			hri_sercomspi_wait_for_sync(hw, SERCOM_SPI_SYNCBUSY_ENABLE);
		}
		hri_sercomspi_write_CTRLA_reg(hw, SERCOM_SPI_CTRLA_SWRST | mode);
     95c:	2301      	movs	r3, #1
     95e:	4313      	orrs	r3, r2
}

static inline void hri_sercomspi_write_CTRLA_reg(const void *const hw, hri_sercomspi_ctrla_reg_t data)
{
	SERCOM_CRITICAL_SECTION_ENTER();
	((Sercom *)hw)->SPI.CTRLA.reg = data;
     960:	6023      	str	r3, [r4, #0]
	while (((Sercom *)hw)->SPI.SYNCBUSY.reg & reg) {
     962:	69e3      	ldr	r3, [r4, #28]
     964:	079b      	lsls	r3, r3, #30
     966:	d1fc      	bne.n	962 <_spi_m_sync_init+0x76>
     968:	69e3      	ldr	r3, [r4, #28]
     96a:	07db      	lsls	r3, r3, #31
     96c:	d4fc      	bmi.n	968 <_spi_m_sync_init+0x7c>
	}
	hri_sercomspi_wait_for_sync(hw, SERCOM_SPI_SYNCBUSY_SWRST);

	dev->prvt = hw;
     96e:	6034      	str	r4, [r6, #0]

	if ((regs->ctrla & SERCOM_SPI_CTRLA_MODE_Msk) == SERCOM_USART_CTRLA_MODE_SPI_SLAVE) {
     970:	782b      	ldrb	r3, [r5, #0]
     972:	786a      	ldrb	r2, [r5, #1]
     974:	0212      	lsls	r2, r2, #8
     976:	431a      	orrs	r2, r3
     978:	78ab      	ldrb	r3, [r5, #2]
     97a:	041b      	lsls	r3, r3, #16
     97c:	431a      	orrs	r2, r3
     97e:	78eb      	ldrb	r3, [r5, #3]
     980:	061b      	lsls	r3, r3, #24
     982:	4313      	orrs	r3, r2
     984:	221c      	movs	r2, #28
     986:	4013      	ands	r3, r2
     988:	2b08      	cmp	r3, #8
     98a:	d04d      	beq.n	a28 <_spi_m_sync_init+0x13c>
	ASSERT(hw && regs);
     98c:	2c00      	cmp	r4, #0
     98e:	d100      	bne.n	992 <_spi_m_sync_init+0xa6>
     990:	e08d      	b.n	aae <_spi_m_sync_init+0x1c2>
     992:	2d00      	cmp	r5, #0
     994:	d100      	bne.n	998 <_spi_m_sync_init+0xac>
     996:	e088      	b.n	aaa <_spi_m_sync_init+0x1be>
     998:	2001      	movs	r0, #1
     99a:	4a4c      	ldr	r2, [pc, #304]	; (acc <_spi_m_sync_init+0x1e0>)
     99c:	4949      	ldr	r1, [pc, #292]	; (ac4 <_spi_m_sync_init+0x1d8>)
     99e:	4b4a      	ldr	r3, [pc, #296]	; (ac8 <_spi_m_sync_init+0x1dc>)
     9a0:	4798      	blx	r3
	    hw, regs->ctrla & ~(SERCOM_SPI_CTRLA_IBON | SERCOM_SPI_CTRLA_ENABLE | SERCOM_SPI_CTRLA_SWRST));
     9a2:	782b      	ldrb	r3, [r5, #0]
     9a4:	786a      	ldrb	r2, [r5, #1]
     9a6:	0212      	lsls	r2, r2, #8
     9a8:	431a      	orrs	r2, r3
     9aa:	78ab      	ldrb	r3, [r5, #2]
     9ac:	041b      	lsls	r3, r3, #16
     9ae:	431a      	orrs	r2, r3
     9b0:	78eb      	ldrb	r3, [r5, #3]
     9b2:	061b      	lsls	r3, r3, #24
     9b4:	4313      	orrs	r3, r2
	hri_sercomspi_write_CTRLA_reg(
     9b6:	4a46      	ldr	r2, [pc, #280]	; (ad0 <_spi_m_sync_init+0x1e4>)
     9b8:	4013      	ands	r3, r2
	((Sercom *)hw)->SPI.CTRLA.reg = data;
     9ba:	6023      	str	r3, [r4, #0]
	while (((Sercom *)hw)->SPI.SYNCBUSY.reg & reg) {
     9bc:	69e3      	ldr	r3, [r4, #28]
     9be:	079b      	lsls	r3, r3, #30
     9c0:	d1fc      	bne.n	9bc <_spi_m_sync_init+0xd0>
	    (regs->ctrlb
     9c2:	792b      	ldrb	r3, [r5, #4]
     9c4:	796a      	ldrb	r2, [r5, #5]
     9c6:	0212      	lsls	r2, r2, #8
     9c8:	431a      	orrs	r2, r3
     9ca:	79ab      	ldrb	r3, [r5, #6]
     9cc:	041b      	lsls	r3, r3, #16
     9ce:	431a      	orrs	r2, r3
     9d0:	79eb      	ldrb	r3, [r5, #7]
     9d2:	061b      	lsls	r3, r3, #24
     9d4:	4313      	orrs	r3, r2
	        | (SERCOM_SPI_CTRLB_RXEN));
     9d6:	4a3f      	ldr	r2, [pc, #252]	; (ad4 <_spi_m_sync_init+0x1e8>)
     9d8:	4013      	ands	r3, r2
	hri_sercomspi_write_CTRLB_reg(
     9da:	2280      	movs	r2, #128	; 0x80
     9dc:	0292      	lsls	r2, r2, #10
     9de:	4313      	orrs	r3, r2
}

static inline void hri_sercomspi_write_CTRLB_reg(const void *const hw, hri_sercomspi_ctrlb_reg_t data)
{
	SERCOM_CRITICAL_SECTION_ENTER();
	((Sercom *)hw)->SPI.CTRLB.reg = data;
     9e0:	6063      	str	r3, [r4, #4]
	while (((Sercom *)hw)->SPI.SYNCBUSY.reg & reg) {
     9e2:	69e3      	ldr	r3, [r4, #28]
     9e4:	075b      	lsls	r3, r3, #29
     9e6:	d1fc      	bne.n	9e2 <_spi_m_sync_init+0xf6>
	hri_sercomspi_write_BAUD_reg(hw, regs->baud);
     9e8:	7b2b      	ldrb	r3, [r5, #12]
}

static inline void hri_sercomspi_write_BAUD_reg(const void *const hw, hri_sercomspi_baud_reg_t data)
{
	SERCOM_CRITICAL_SECTION_ENTER();
	((Sercom *)hw)->SPI.BAUD.reg = data;
     9ea:	7323      	strb	r3, [r4, #12]
	hri_sercomspi_write_DBGCTRL_reg(hw, regs->dbgctrl);
     9ec:	7b6a      	ldrb	r2, [r5, #13]
}

static inline void hri_sercomspi_write_DBGCTRL_reg(const void *const hw, hri_sercomspi_dbgctrl_reg_t data)
{
	SERCOM_CRITICAL_SECTION_ENTER();
	((Sercom *)hw)->SPI.DBGCTRL.reg = data;
     9ee:	2330      	movs	r3, #48	; 0x30
     9f0:	54e2      	strb	r2, [r4, r3]
	} else {
		_spi_load_regs_master(hw, regs);
	}

	/* Load character size from default hardware configuration */
	dev->char_size = ((regs->ctrlb & SERCOM_SPI_CTRLB_CHSIZE_Msk) == 0) ? 1 : 2;
     9f2:	792b      	ldrb	r3, [r5, #4]
     9f4:	075b      	lsls	r3, r3, #29
     9f6:	d15c      	bne.n	ab2 <_spi_m_sync_init+0x1c6>
     9f8:	2301      	movs	r3, #1
     9fa:	7133      	strb	r3, [r6, #4]

	dev->dummy_byte = regs->dummy_byte;
     9fc:	7baa      	ldrb	r2, [r5, #14]
     9fe:	7beb      	ldrb	r3, [r5, #15]
     a00:	021b      	lsls	r3, r3, #8
     a02:	4313      	orrs	r3, r2
     a04:	80f3      	strh	r3, [r6, #6]

	return ERR_NONE;
     a06:	2000      	movs	r0, #0
}
     a08:	bd70      	pop	{r4, r5, r6, pc}
		if (sercomspi_regs[i].n == n) {
     a0a:	2800      	cmp	r0, #0
     a0c:	d002      	beq.n	a14 <_spi_m_sync_init+0x128>
	for (i = 0; i < sizeof(sercomspi_regs) / sizeof(struct sercomspi_regs_cfg); i++) {
     a0e:	3301      	adds	r3, #1
     a10:	b2db      	uxtb	r3, r3
     a12:	e772      	b.n	8fa <_spi_m_sync_init+0xe>
			return &sercomspi_regs[i];
     a14:	011d      	lsls	r5, r3, #4
     a16:	18ea      	adds	r2, r5, r3
     a18:	4d2f      	ldr	r5, [pc, #188]	; (ad8 <_spi_m_sync_init+0x1ec>)
     a1a:	353c      	adds	r5, #60	; 0x3c
     a1c:	18ad      	adds	r5, r5, r2
     a1e:	e770      	b.n	902 <_spi_m_sync_init+0x16>
	ASSERT(dev && hw);
     a20:	2000      	movs	r0, #0
     a22:	e775      	b.n	910 <_spi_m_sync_init+0x24>
     a24:	2000      	movs	r0, #0
     a26:	e773      	b.n	910 <_spi_m_sync_init+0x24>
	ASSERT(hw && regs);
     a28:	2c00      	cmp	r4, #0
     a2a:	d03c      	beq.n	aa6 <_spi_m_sync_init+0x1ba>
     a2c:	2d00      	cmp	r5, #0
     a2e:	d038      	beq.n	aa2 <_spi_m_sync_init+0x1b6>
     a30:	2001      	movs	r0, #1
     a32:	4a2a      	ldr	r2, [pc, #168]	; (adc <_spi_m_sync_init+0x1f0>)
     a34:	4923      	ldr	r1, [pc, #140]	; (ac4 <_spi_m_sync_init+0x1d8>)
     a36:	4b24      	ldr	r3, [pc, #144]	; (ac8 <_spi_m_sync_init+0x1dc>)
     a38:	4798      	blx	r3
	    hw, regs->ctrla & ~(SERCOM_SPI_CTRLA_IBON | SERCOM_SPI_CTRLA_ENABLE | SERCOM_SPI_CTRLA_SWRST));
     a3a:	782b      	ldrb	r3, [r5, #0]
     a3c:	786a      	ldrb	r2, [r5, #1]
     a3e:	0212      	lsls	r2, r2, #8
     a40:	431a      	orrs	r2, r3
     a42:	78ab      	ldrb	r3, [r5, #2]
     a44:	041b      	lsls	r3, r3, #16
     a46:	431a      	orrs	r2, r3
     a48:	78eb      	ldrb	r3, [r5, #3]
     a4a:	061b      	lsls	r3, r3, #24
     a4c:	4313      	orrs	r3, r2
	hri_sercomspi_write_CTRLA_reg(
     a4e:	4a20      	ldr	r2, [pc, #128]	; (ad0 <_spi_m_sync_init+0x1e4>)
     a50:	4013      	ands	r3, r2
	((Sercom *)hw)->SPI.CTRLA.reg = data;
     a52:	6023      	str	r3, [r4, #0]
	while (((Sercom *)hw)->SPI.SYNCBUSY.reg & reg) {
     a54:	69e3      	ldr	r3, [r4, #28]
     a56:	079b      	lsls	r3, r3, #30
     a58:	d1fc      	bne.n	a54 <_spi_m_sync_init+0x168>
	                              (regs->ctrlb & ~(SERCOM_SPI_CTRLB_MSSEN))
     a5a:	792b      	ldrb	r3, [r5, #4]
     a5c:	796a      	ldrb	r2, [r5, #5]
     a5e:	0212      	lsls	r2, r2, #8
     a60:	431a      	orrs	r2, r3
     a62:	79ab      	ldrb	r3, [r5, #6]
     a64:	041b      	lsls	r3, r3, #16
     a66:	431a      	orrs	r2, r3
     a68:	79eb      	ldrb	r3, [r5, #7]
     a6a:	061b      	lsls	r3, r3, #24
     a6c:	4313      	orrs	r3, r2
	                                  | (SERCOM_SPI_CTRLB_RXEN | SERCOM_SPI_CTRLB_SSDE | SERCOM_SPI_CTRLB_PLOADEN));
     a6e:	4a1c      	ldr	r2, [pc, #112]	; (ae0 <_spi_m_sync_init+0x1f4>)
     a70:	4013      	ands	r3, r2
	hri_sercomspi_write_CTRLB_reg(hw,
     a72:	4a1c      	ldr	r2, [pc, #112]	; (ae4 <_spi_m_sync_init+0x1f8>)
     a74:	4313      	orrs	r3, r2
	((Sercom *)hw)->SPI.CTRLB.reg = data;
     a76:	6063      	str	r3, [r4, #4]
	while (((Sercom *)hw)->SPI.SYNCBUSY.reg & reg) {
     a78:	69e3      	ldr	r3, [r4, #28]
     a7a:	075b      	lsls	r3, r3, #29
     a7c:	d1fc      	bne.n	a78 <_spi_m_sync_init+0x18c>
	hri_sercomspi_write_ADDR_reg(hw, regs->addr);
     a7e:	7a2b      	ldrb	r3, [r5, #8]
     a80:	7a6a      	ldrb	r2, [r5, #9]
     a82:	0212      	lsls	r2, r2, #8
     a84:	431a      	orrs	r2, r3
     a86:	7aab      	ldrb	r3, [r5, #10]
     a88:	041b      	lsls	r3, r3, #16
     a8a:	431a      	orrs	r2, r3
     a8c:	7aeb      	ldrb	r3, [r5, #11]
     a8e:	061b      	lsls	r3, r3, #24
     a90:	4313      	orrs	r3, r2
	((Sercom *)hw)->SPI.ADDR.reg = data;
     a92:	6263      	str	r3, [r4, #36]	; 0x24
	hri_sercomspi_write_DBGCTRL_reg(hw, regs->dbgctrl);
     a94:	7b6a      	ldrb	r2, [r5, #13]
	((Sercom *)hw)->SPI.DBGCTRL.reg = data;
     a96:	2330      	movs	r3, #48	; 0x30
     a98:	54e2      	strb	r2, [r4, r3]
	return ((Sercom *)hw)->SPI.SYNCBUSY.reg & reg;
     a9a:	69e3      	ldr	r3, [r4, #28]
	while (hri_sercomspi_is_syncing(hw, 0xFFFFFFFF))
     a9c:	2b00      	cmp	r3, #0
     a9e:	d1fc      	bne.n	a9a <_spi_m_sync_init+0x1ae>
     aa0:	e7a7      	b.n	9f2 <_spi_m_sync_init+0x106>
	ASSERT(hw && regs);
     aa2:	2000      	movs	r0, #0
     aa4:	e7c5      	b.n	a32 <_spi_m_sync_init+0x146>
     aa6:	2000      	movs	r0, #0
     aa8:	e7c3      	b.n	a32 <_spi_m_sync_init+0x146>
	ASSERT(hw && regs);
     aaa:	2000      	movs	r0, #0
     aac:	e775      	b.n	99a <_spi_m_sync_init+0xae>
     aae:	2000      	movs	r0, #0
     ab0:	e773      	b.n	99a <_spi_m_sync_init+0xae>
	dev->char_size = ((regs->ctrlb & SERCOM_SPI_CTRLB_CHSIZE_Msk) == 0) ? 1 : 2;
     ab2:	2302      	movs	r3, #2
     ab4:	e7a1      	b.n	9fa <_spi_m_sync_init+0x10e>
		return ERR_INVALID_ARG;
     ab6:	200d      	movs	r0, #13
     ab8:	4240      	negs	r0, r0
     aba:	e7a5      	b.n	a08 <_spi_m_sync_init+0x11c>
     abc:	000008dd 	.word	0x000008dd
     ac0:	00000925 	.word	0x00000925
     ac4:	00001864 	.word	0x00001864
     ac8:	00000729 	.word	0x00000729
     acc:	000008ef 	.word	0x000008ef
     ad0:	fffffefc 	.word	0xfffffefc
     ad4:	fffd1dbf 	.word	0xfffd1dbf
     ad8:	00001814 	.word	0x00001814
     adc:	00000903 	.word	0x00000903
     ae0:	fffdddbf 	.word	0xfffdddbf
     ae4:	00020240 	.word	0x00020240

00000ae8 <_spi_m_sync_trans>:

	return ERR_NONE;
}

int32_t _spi_m_sync_trans(struct _spi_m_sync_dev *dev, const struct spi_msg *msg)
{
     ae8:	b5f0      	push	{r4, r5, r6, r7, lr}
     aea:	46ce      	mov	lr, r9
     aec:	4647      	mov	r7, r8
     aee:	b580      	push	{r7, lr}
     af0:	b089      	sub	sp, #36	; 0x24
     af2:	4681      	mov	r9, r0
     af4:	000d      	movs	r5, r1
	void *                 hw   = dev->prvt;
     af6:	6804      	ldr	r4, [r0, #0]
	int32_t                rc   = 0;
	struct _spi_trans_ctrl ctrl = {msg->txbuf, msg->rxbuf, 0, 0, dev->char_size};
     af8:	680b      	ldr	r3, [r1, #0]
     afa:	9303      	str	r3, [sp, #12]
     afc:	684b      	ldr	r3, [r1, #4]
     afe:	9304      	str	r3, [sp, #16]
     b00:	2300      	movs	r3, #0
     b02:	9305      	str	r3, [sp, #20]
     b04:	9306      	str	r3, [sp, #24]
     b06:	7906      	ldrb	r6, [r0, #4]

	ASSERT(dev && hw);
     b08:	2800      	cmp	r0, #0
     b0a:	d014      	beq.n	b36 <_spi_m_sync_trans+0x4e>
     b0c:	2c00      	cmp	r4, #0
     b0e:	d010      	beq.n	b32 <_spi_m_sync_trans+0x4a>
     b10:	2001      	movs	r0, #1
     b12:	4a37      	ldr	r2, [pc, #220]	; (bf0 <_spi_m_sync_trans+0x108>)
     b14:	4937      	ldr	r1, [pc, #220]	; (bf4 <_spi_m_sync_trans+0x10c>)
     b16:	4b38      	ldr	r3, [pc, #224]	; (bf8 <_spi_m_sync_trans+0x110>)
     b18:	4798      	blx	r3
     b1a:	69e3      	ldr	r3, [r4, #28]

	/* If settings are not applied (pending), we can not go on */
	if (hri_sercomspi_is_syncing(
     b1c:	075b      	lsls	r3, r3, #29
     b1e:	d164      	bne.n	bea <_spi_m_sync_trans+0x102>
	while (((Sercom *)hw)->SPI.SYNCBUSY.reg & reg) {
     b20:	69e3      	ldr	r3, [r4, #28]
     b22:	079b      	lsls	r3, r3, #30
     b24:	d1fc      	bne.n	b20 <_spi_m_sync_trans+0x38>
	tmp = ((Sercom *)hw)->SPI.CTRLA.reg;
     b26:	6823      	ldr	r3, [r4, #0]
	        hw, (SERCOM_SPI_SYNCBUSY_SWRST | SERCOM_SPI_SYNCBUSY_ENABLE | SERCOM_SPI_SYNCBUSY_CTRLB))) {
		return ERR_BUSY;
	}

	/* SPI must be enabled to start synchronous transfer */
	if (!hri_sercomspi_get_CTRLA_ENABLE_bit(hw)) {
     b28:	079b      	lsls	r3, r3, #30
     b2a:	d420      	bmi.n	b6e <_spi_m_sync_trans+0x86>
		return ERR_NOT_INITIALIZED;
     b2c:	2014      	movs	r0, #20
     b2e:	4240      	negs	r0, r0
     b30:	e056      	b.n	be0 <_spi_m_sync_trans+0xf8>
	ASSERT(dev && hw);
     b32:	2000      	movs	r0, #0
     b34:	e7ed      	b.n	b12 <_spi_m_sync_trans+0x2a>
     b36:	2000      	movs	r0, #0
     b38:	e7eb      	b.n	b12 <_spi_m_sync_trans+0x2a>
		return false;
     b3a:	2200      	movs	r2, #0
     b3c:	e02d      	b.n	b9a <_spi_m_sync_trans+0xb2>
			data |= (*ctrl->txbuf) << 8;
     b3e:	7848      	ldrb	r0, [r1, #1]
     b40:	0200      	lsls	r0, r0, #8
     b42:	4647      	mov	r7, r8
     b44:	4307      	orrs	r7, r0
     b46:	46b8      	mov	r8, r7
			ctrl->txbuf++;
     b48:	3102      	adds	r1, #2
     b4a:	9103      	str	r1, [sp, #12]
	ctrl->txcnt++;
     b4c:	3201      	adds	r2, #1
     b4e:	9205      	str	r2, [sp, #20]
	((Sercom *)hw)->SPI.DATA.reg = data;
     b50:	4642      	mov	r2, r8
     b52:	62a2      	str	r2, [r4, #40]	; 0x28
	if (SERCOM_SPI_INTFLAG_ERROR & iflag) {
     b54:	b25b      	sxtb	r3, r3
     b56:	2b00      	cmp	r3, #0
     b58:	db35      	blt.n	bc6 <_spi_m_sync_trans+0xde>
	return ERR_NONE;
     b5a:	2000      	movs	r0, #0
			}
		}

		rc = _spi_err_check(iflag, hw);

		if (rc < 0) {
     b5c:	2800      	cmp	r0, #0
     b5e:	db3a      	blt.n	bd6 <_spi_m_sync_trans+0xee>
			break;
		}
		if (ctrl.txcnt >= msg->size && ctrl.rxcnt >= msg->size) {
     b60:	9805      	ldr	r0, [sp, #20]
     b62:	68ab      	ldr	r3, [r5, #8]
     b64:	4298      	cmp	r0, r3
     b66:	d302      	bcc.n	b6e <_spi_m_sync_trans+0x86>
     b68:	9a06      	ldr	r2, [sp, #24]
     b6a:	4293      	cmp	r3, r2
     b6c:	d933      	bls.n	bd6 <_spi_m_sync_trans+0xee>
	return ((Sercom *)hw)->SPI.INTFLAG.reg;
     b6e:	7e23      	ldrb	r3, [r4, #24]
     b70:	b2db      	uxtb	r3, r3
	if (!(iflag & SERCOM_SPI_INTFLAG_RXC)) {
     b72:	075a      	lsls	r2, r3, #29
     b74:	d5e1      	bpl.n	b3a <_spi_m_sync_trans+0x52>
	return ((Sercom *)hw)->SPI.DATA.reg;
     b76:	6aa1      	ldr	r1, [r4, #40]	; 0x28
	if (ctrl->rxbuf) {
     b78:	9a04      	ldr	r2, [sp, #16]
     b7a:	2a00      	cmp	r2, #0
     b7c:	d008      	beq.n	b90 <_spi_m_sync_trans+0xa8>
		*ctrl->rxbuf++ = (uint8_t)data;
     b7e:	1c50      	adds	r0, r2, #1
     b80:	9004      	str	r0, [sp, #16]
     b82:	7011      	strb	r1, [r2, #0]
		if (ctrl->char_size > 1) {
     b84:	2e01      	cmp	r6, #1
     b86:	d903      	bls.n	b90 <_spi_m_sync_trans+0xa8>
			*ctrl->rxbuf++ = (uint8_t)(data >> 8);
     b88:	1c90      	adds	r0, r2, #2
     b8a:	9004      	str	r0, [sp, #16]
     b8c:	0a09      	lsrs	r1, r1, #8
     b8e:	7051      	strb	r1, [r2, #1]
	ctrl->rxcnt++;
     b90:	9a06      	ldr	r2, [sp, #24]
     b92:	9201      	str	r2, [sp, #4]
     b94:	3201      	adds	r2, #1
     b96:	9206      	str	r2, [sp, #24]
	return true;
     b98:	2201      	movs	r2, #1
		if (!_spi_rx_check_and_receive(hw, iflag, &ctrl)) {
     b9a:	2a00      	cmp	r2, #0
     b9c:	d1da      	bne.n	b54 <_spi_m_sync_trans+0x6c>
			if (ctrl.rxcnt >= ctrl.txcnt) {
     b9e:	9906      	ldr	r1, [sp, #24]
     ba0:	9a05      	ldr	r2, [sp, #20]
     ba2:	4291      	cmp	r1, r2
     ba4:	d3d6      	bcc.n	b54 <_spi_m_sync_trans+0x6c>
				_spi_tx_check_and_send(hw, iflag, &ctrl, dev->dummy_byte);
     ba6:	4649      	mov	r1, r9
     ba8:	88c8      	ldrh	r0, [r1, #6]
	if (!(SERCOM_SPI_INTFLAG_DRE & iflag)) {
     baa:	07d9      	lsls	r1, r3, #31
     bac:	d5d2      	bpl.n	b54 <_spi_m_sync_trans+0x6c>
	if (ctrl->txbuf) {
     bae:	9903      	ldr	r1, [sp, #12]
     bb0:	2900      	cmp	r1, #0
     bb2:	d006      	beq.n	bc2 <_spi_m_sync_trans+0xda>
		data = *ctrl->txbuf++;
     bb4:	1c48      	adds	r0, r1, #1
     bb6:	9003      	str	r0, [sp, #12]
     bb8:	7808      	ldrb	r0, [r1, #0]
     bba:	4680      	mov	r8, r0
		if (ctrl->char_size > 1) {
     bbc:	2e01      	cmp	r6, #1
     bbe:	d8be      	bhi.n	b3e <_spi_m_sync_trans+0x56>
     bc0:	e7c4      	b.n	b4c <_spi_m_sync_trans+0x64>
		data = dummy;
     bc2:	4680      	mov	r8, r0
     bc4:	e7c2      	b.n	b4c <_spi_m_sync_trans+0x64>
}

static inline void hri_sercomspi_clear_STATUS_reg(const void *const hw, hri_sercomspi_status_reg_t mask)
{
	SERCOM_CRITICAL_SECTION_ENTER();
	((Sercom *)hw)->SPI.STATUS.reg = mask;
     bc6:	2301      	movs	r3, #1
     bc8:	425b      	negs	r3, r3
     bca:	8363      	strh	r3, [r4, #26]
	((Sercom *)hw)->SPI.INTFLAG.reg = mask;
     bcc:	3381      	adds	r3, #129	; 0x81
     bce:	7623      	strb	r3, [r4, #24]
		return ERR_OVERFLOW;
     bd0:	2013      	movs	r0, #19
     bd2:	4240      	negs	r0, r0
     bd4:	e7c2      	b.n	b5c <_spi_m_sync_trans+0x74>
	tmp = ((Sercom *)hw)->SPI.INTFLAG.reg;
     bd6:	7e23      	ldrb	r3, [r4, #24]
	while (!(hri_sercomspi_get_INTFLAG_reg(hw, SERCOM_SPI_INTFLAG_TXC | SERCOM_SPI_INTFLAG_DRE))) {
     bd8:	079b      	lsls	r3, r3, #30
     bda:	d0fc      	beq.n	bd6 <_spi_m_sync_trans+0xee>
	((Sercom *)hw)->SPI.INTFLAG.reg = mask;
     bdc:	2303      	movs	r3, #3
     bde:	7623      	strb	r3, [r4, #24]
	}
	/* Wait until SPI bus idle */
	_spi_wait_bus_idle(hw);

	return rc;
}
     be0:	b009      	add	sp, #36	; 0x24
     be2:	bc0c      	pop	{r2, r3}
     be4:	4690      	mov	r8, r2
     be6:	4699      	mov	r9, r3
     be8:	bdf0      	pop	{r4, r5, r6, r7, pc}
		return ERR_BUSY;
     bea:	2004      	movs	r0, #4
     bec:	4240      	negs	r0, r0
     bee:	e7f7      	b.n	be0 <_spi_m_sync_trans+0xf8>
     bf0:	00000a85 	.word	0x00000a85
     bf4:	00001864 	.word	0x00001864
     bf8:	00000729 	.word	0x00000729

00000bfc <_sysctrl_init_sources>:
}

static inline hri_sysctrl_osc8m_reg_t hri_sysctrl_read_OSC8M_CALIB_bf(const void *const hw)
{
	uint32_t tmp;
	tmp = ((Sysctrl *)hw)->OSC8M.reg;
     bfc:	4a0e      	ldr	r2, [pc, #56]	; (c38 <_sysctrl_init_sources+0x3c>)
     bfe:	6a11      	ldr	r1, [r2, #32]
	tmp = (tmp & SYSCTRL_OSC8M_CALIB_Msk) >> SYSCTRL_OSC8M_CALIB_Pos;
     c00:	0c09      	lsrs	r1, r1, #16
}

static inline hri_sysctrl_osc8m_reg_t hri_sysctrl_read_OSC8M_FRANGE_bf(const void *const hw)
{
	uint32_t tmp;
	tmp = ((Sysctrl *)hw)->OSC8M.reg;
     c02:	6a13      	ldr	r3, [r2, #32]

#if CONF_OSC8M_CONFIG == 1
	calib = hri_sysctrl_read_OSC8M_CALIB_bf(hw);

	hri_sysctrl_write_OSC8M_reg(hw,
	                            SYSCTRL_OSC8M_FRANGE(hri_sysctrl_read_OSC8M_FRANGE_bf(hw)) |
     c04:	0f9b      	lsrs	r3, r3, #30
     c06:	079b      	lsls	r3, r3, #30
#if CONF_OSC8M_OVERWRITE_CALIBRATION == 1
	                                SYSCTRL_OSC8M_CALIB(CONF_OSC8M_CALIB) |
#else
	                                SYSCTRL_OSC8M_CALIB(calib) |
     c08:	0409      	lsls	r1, r1, #16
     c0a:	480c      	ldr	r0, [pc, #48]	; (c3c <_sysctrl_init_sources+0x40>)
     c0c:	4001      	ands	r1, r0
#endif
	                                SYSCTRL_OSC8M_PRESC(CONF_OSC8M_PRESC)
	                                | (CONF_OSC8M_RUNSTDBY << SYSCTRL_OSC8M_RUNSTDBY_Pos)
     c0e:	430b      	orrs	r3, r1
	hri_sysctrl_write_OSC8M_reg(hw,
     c10:	2102      	movs	r1, #2
     c12:	430b      	orrs	r3, r1
}

static inline void hri_sysctrl_write_OSC8M_reg(const void *const hw, hri_sysctrl_osc8m_reg_t data)
{
	SYSCTRL_CRITICAL_SECTION_ENTER();
	((Sysctrl *)hw)->OSC8M.reg = data;
     c14:	6213      	str	r3, [r2, #32]
	((Sysctrl *)hw)->OSC32K.reg |= SYSCTRL_OSC32K_ENABLE;
     c16:	6993      	ldr	r3, [r2, #24]
     c18:	430b      	orrs	r3, r1
     c1a:	6193      	str	r3, [r2, #24]
	tmp = ((Sysctrl *)hw)->OSCULP32K.reg;
     c1c:	7f13      	ldrb	r3, [r2, #28]
	tmp = (tmp & SYSCTRL_OSCULP32K_CALIB_Msk) >> SYSCTRL_OSCULP32K_CALIB_Pos;
     c1e:	311d      	adds	r1, #29
     c20:	400b      	ands	r3, r1
	((Sysctrl *)hw)->OSCULP32K.reg = data;
     c22:	7713      	strb	r3, [r2, #28]
	return (((Sysctrl *)hw)->PCLKSR.reg & SYSCTRL_PCLKSR_OSC8MRDY) >> SYSCTRL_PCLKSR_OSC8MRDY_Pos;
     c24:	4b04      	ldr	r3, [pc, #16]	; (c38 <_sysctrl_init_sources+0x3c>)
     c26:	68db      	ldr	r3, [r3, #12]
#endif
#endif

#if CONF_OSC8M_CONFIG == 1
#if CONF_OSC8M_ENABLE == 1
	while (!hri_sysctrl_get_PCLKSR_OSC8MRDY_bit(hw))
     c28:	071b      	lsls	r3, r3, #28
     c2a:	d5fb      	bpl.n	c24 <_sysctrl_init_sources+0x28>
	((Sysctrl *)hw)->OSC8M.reg |= SYSCTRL_OSC8M_ONDEMAND;
     c2c:	4a02      	ldr	r2, [pc, #8]	; (c38 <_sysctrl_init_sources+0x3c>)
     c2e:	6a13      	ldr	r3, [r2, #32]
     c30:	2180      	movs	r1, #128	; 0x80
     c32:	430b      	orrs	r3, r1
     c34:	6213      	str	r3, [r2, #32]
	hri_sysctrl_set_OSC8M_ONDEMAND_bit(hw);
#endif
#endif

	(void)calib, (void)hw;
}
     c36:	4770      	bx	lr
     c38:	40000800 	.word	0x40000800
     c3c:	0fff0000 	.word	0x0fff0000

00000c40 <_sysctrl_init_referenced_generators>:
	((Sysctrl *)hw)->OSC32K.reg &= ~SYSCTRL_OSC32K_ENABLE;
     c40:	4a02      	ldr	r2, [pc, #8]	; (c4c <_sysctrl_init_referenced_generators+0xc>)
     c42:	6993      	ldr	r3, [r2, #24]
     c44:	2102      	movs	r1, #2
     c46:	438b      	bics	r3, r1
     c48:	6193      	str	r3, [r2, #24]
	/* Disable after all possible configurations needs sync written. */
	hri_sysctrl_clear_OSC32K_ENABLE_bit(hw);
#endif

	(void)hw;
}
     c4a:	4770      	bx	lr
     c4c:	40000800 	.word	0x40000800

00000c50 <_Z13helloSequencev>:
	spi_m_sync_enable(&SPI_0);	// enable spi sync
	spi_m_sync_get_io_descriptor(&SPI_0, &io); // create io descriptor for read/write
	spi_m_sync_set_mode(&SPI_0, SPI_MODE_0);
}

void helloSequence(){
     c50:	b5f8      	push	{r3, r4, r5, r6, r7, lr}
	color.set_color(0b00100000);
     c52:	4d0c      	ldr	r5, [pc, #48]	; (c84 <_Z13helloSequencev+0x34>)
     c54:	2120      	movs	r1, #32
     c56:	0028      	movs	r0, r5
     c58:	4c0b      	ldr	r4, [pc, #44]	; (c88 <_Z13helloSequencev+0x38>)
     c5a:	47a0      	blx	r4
	delay_ms(500);
     c5c:	27fa      	movs	r7, #250	; 0xfa
     c5e:	007f      	lsls	r7, r7, #1
     c60:	0038      	movs	r0, r7
     c62:	4e0a      	ldr	r6, [pc, #40]	; (c8c <_Z13helloSequencev+0x3c>)
     c64:	47b0      	blx	r6
	color.set_color(0b00100100);
     c66:	2124      	movs	r1, #36	; 0x24
     c68:	0028      	movs	r0, r5
     c6a:	47a0      	blx	r4
	delay_ms(500);
     c6c:	0038      	movs	r0, r7
     c6e:	47b0      	blx	r6
	color.set_color(0b00000001);
     c70:	2101      	movs	r1, #1
     c72:	0028      	movs	r0, r5
     c74:	47a0      	blx	r4
	delay_ms(500);
     c76:	0038      	movs	r0, r7
     c78:	47b0      	blx	r6
	color.set_color(0b00000000);
     c7a:	2100      	movs	r1, #0
     c7c:	0028      	movs	r0, r5
     c7e:	47a0      	blx	r4
}
     c80:	bdf8      	pop	{r3, r4, r5, r6, r7, pc}
     c82:	46c0      	nop			; (mov r8, r8)
     c84:	20000000 	.word	0x20000000
     c88:	00000121 	.word	0x00000121
     c8c:	000004f1 	.word	0x000004f1

00000c90 <main>:

int main(void)
{		
     c90:	b510      	push	{r4, lr}
	// SPI_0: Mode 0
	// MSb first
	// SO latched on falling edge
	
	// TIMER_0, gpio
	atmel_start_init();
     c92:	4b03      	ldr	r3, [pc, #12]	; (ca0 <main+0x10>)
     c94:	4798      	blx	r3
	helloSequence();
     c96:	4b03      	ldr	r3, [pc, #12]	; (ca4 <main+0x14>)
     c98:	4798      	blx	r3
		//}else{
		//color.set_color(0b00100100);
	//}

	while (1) {
		helloSequence();
     c9a:	4b02      	ldr	r3, [pc, #8]	; (ca4 <main+0x14>)
     c9c:	4798      	blx	r3
     c9e:	e7fc      	b.n	c9a <main+0xa>
     ca0:	00000115 	.word	0x00000115
     ca4:	00000c51 	.word	0x00000c51

00000ca8 <_GLOBAL__sub_I__ZN9__gnu_cxx9__freeresEv>:
     ca8:	b570      	push	{r4, r5, r6, lr}
     caa:	259e      	movs	r5, #158	; 0x9e
     cac:	4c08      	ldr	r4, [pc, #32]	; (cd0 <_GLOBAL__sub_I__ZN9__gnu_cxx9__freeresEv+0x28>)
     cae:	012d      	lsls	r5, r5, #4
     cb0:	0028      	movs	r0, r5
     cb2:	60e5      	str	r5, [r4, #12]
     cb4:	f000 f8c2 	bl	e3c <malloc>
     cb8:	60a0      	str	r0, [r4, #8]
     cba:	2800      	cmp	r0, #0
     cbc:	d004      	beq.n	cc8 <_GLOBAL__sub_I__ZN9__gnu_cxx9__freeresEv+0x20>
     cbe:	2300      	movs	r3, #0
     cc0:	6060      	str	r0, [r4, #4]
     cc2:	6005      	str	r5, [r0, #0]
     cc4:	6043      	str	r3, [r0, #4]
     cc6:	bd70      	pop	{r4, r5, r6, pc}
     cc8:	60e0      	str	r0, [r4, #12]
     cca:	6060      	str	r0, [r4, #4]
     ccc:	e7fb      	b.n	cc6 <_GLOBAL__sub_I__ZN9__gnu_cxx9__freeresEv+0x1e>
     cce:	46c0      	nop			; (mov r8, r8)
     cd0:	2000087c 	.word	0x2000087c

00000cd4 <__udivsi3>:
     cd4:	2200      	movs	r2, #0
     cd6:	0843      	lsrs	r3, r0, #1
     cd8:	428b      	cmp	r3, r1
     cda:	d374      	bcc.n	dc6 <__udivsi3+0xf2>
     cdc:	0903      	lsrs	r3, r0, #4
     cde:	428b      	cmp	r3, r1
     ce0:	d35f      	bcc.n	da2 <__udivsi3+0xce>
     ce2:	0a03      	lsrs	r3, r0, #8
     ce4:	428b      	cmp	r3, r1
     ce6:	d344      	bcc.n	d72 <__udivsi3+0x9e>
     ce8:	0b03      	lsrs	r3, r0, #12
     cea:	428b      	cmp	r3, r1
     cec:	d328      	bcc.n	d40 <__udivsi3+0x6c>
     cee:	0c03      	lsrs	r3, r0, #16
     cf0:	428b      	cmp	r3, r1
     cf2:	d30d      	bcc.n	d10 <__udivsi3+0x3c>
     cf4:	22ff      	movs	r2, #255	; 0xff
     cf6:	0209      	lsls	r1, r1, #8
     cf8:	ba12      	rev	r2, r2
     cfa:	0c03      	lsrs	r3, r0, #16
     cfc:	428b      	cmp	r3, r1
     cfe:	d302      	bcc.n	d06 <__udivsi3+0x32>
     d00:	1212      	asrs	r2, r2, #8
     d02:	0209      	lsls	r1, r1, #8
     d04:	d065      	beq.n	dd2 <__udivsi3+0xfe>
     d06:	0b03      	lsrs	r3, r0, #12
     d08:	428b      	cmp	r3, r1
     d0a:	d319      	bcc.n	d40 <__udivsi3+0x6c>
     d0c:	e000      	b.n	d10 <__udivsi3+0x3c>
     d0e:	0a09      	lsrs	r1, r1, #8
     d10:	0bc3      	lsrs	r3, r0, #15
     d12:	428b      	cmp	r3, r1
     d14:	d301      	bcc.n	d1a <__udivsi3+0x46>
     d16:	03cb      	lsls	r3, r1, #15
     d18:	1ac0      	subs	r0, r0, r3
     d1a:	4152      	adcs	r2, r2
     d1c:	0b83      	lsrs	r3, r0, #14
     d1e:	428b      	cmp	r3, r1
     d20:	d301      	bcc.n	d26 <__udivsi3+0x52>
     d22:	038b      	lsls	r3, r1, #14
     d24:	1ac0      	subs	r0, r0, r3
     d26:	4152      	adcs	r2, r2
     d28:	0b43      	lsrs	r3, r0, #13
     d2a:	428b      	cmp	r3, r1
     d2c:	d301      	bcc.n	d32 <__udivsi3+0x5e>
     d2e:	034b      	lsls	r3, r1, #13
     d30:	1ac0      	subs	r0, r0, r3
     d32:	4152      	adcs	r2, r2
     d34:	0b03      	lsrs	r3, r0, #12
     d36:	428b      	cmp	r3, r1
     d38:	d301      	bcc.n	d3e <__udivsi3+0x6a>
     d3a:	030b      	lsls	r3, r1, #12
     d3c:	1ac0      	subs	r0, r0, r3
     d3e:	4152      	adcs	r2, r2
     d40:	0ac3      	lsrs	r3, r0, #11
     d42:	428b      	cmp	r3, r1
     d44:	d301      	bcc.n	d4a <__udivsi3+0x76>
     d46:	02cb      	lsls	r3, r1, #11
     d48:	1ac0      	subs	r0, r0, r3
     d4a:	4152      	adcs	r2, r2
     d4c:	0a83      	lsrs	r3, r0, #10
     d4e:	428b      	cmp	r3, r1
     d50:	d301      	bcc.n	d56 <__udivsi3+0x82>
     d52:	028b      	lsls	r3, r1, #10
     d54:	1ac0      	subs	r0, r0, r3
     d56:	4152      	adcs	r2, r2
     d58:	0a43      	lsrs	r3, r0, #9
     d5a:	428b      	cmp	r3, r1
     d5c:	d301      	bcc.n	d62 <__udivsi3+0x8e>
     d5e:	024b      	lsls	r3, r1, #9
     d60:	1ac0      	subs	r0, r0, r3
     d62:	4152      	adcs	r2, r2
     d64:	0a03      	lsrs	r3, r0, #8
     d66:	428b      	cmp	r3, r1
     d68:	d301      	bcc.n	d6e <__udivsi3+0x9a>
     d6a:	020b      	lsls	r3, r1, #8
     d6c:	1ac0      	subs	r0, r0, r3
     d6e:	4152      	adcs	r2, r2
     d70:	d2cd      	bcs.n	d0e <__udivsi3+0x3a>
     d72:	09c3      	lsrs	r3, r0, #7
     d74:	428b      	cmp	r3, r1
     d76:	d301      	bcc.n	d7c <__udivsi3+0xa8>
     d78:	01cb      	lsls	r3, r1, #7
     d7a:	1ac0      	subs	r0, r0, r3
     d7c:	4152      	adcs	r2, r2
     d7e:	0983      	lsrs	r3, r0, #6
     d80:	428b      	cmp	r3, r1
     d82:	d301      	bcc.n	d88 <__udivsi3+0xb4>
     d84:	018b      	lsls	r3, r1, #6
     d86:	1ac0      	subs	r0, r0, r3
     d88:	4152      	adcs	r2, r2
     d8a:	0943      	lsrs	r3, r0, #5
     d8c:	428b      	cmp	r3, r1
     d8e:	d301      	bcc.n	d94 <__udivsi3+0xc0>
     d90:	014b      	lsls	r3, r1, #5
     d92:	1ac0      	subs	r0, r0, r3
     d94:	4152      	adcs	r2, r2
     d96:	0903      	lsrs	r3, r0, #4
     d98:	428b      	cmp	r3, r1
     d9a:	d301      	bcc.n	da0 <__udivsi3+0xcc>
     d9c:	010b      	lsls	r3, r1, #4
     d9e:	1ac0      	subs	r0, r0, r3
     da0:	4152      	adcs	r2, r2
     da2:	08c3      	lsrs	r3, r0, #3
     da4:	428b      	cmp	r3, r1
     da6:	d301      	bcc.n	dac <__udivsi3+0xd8>
     da8:	00cb      	lsls	r3, r1, #3
     daa:	1ac0      	subs	r0, r0, r3
     dac:	4152      	adcs	r2, r2
     dae:	0883      	lsrs	r3, r0, #2
     db0:	428b      	cmp	r3, r1
     db2:	d301      	bcc.n	db8 <__udivsi3+0xe4>
     db4:	008b      	lsls	r3, r1, #2
     db6:	1ac0      	subs	r0, r0, r3
     db8:	4152      	adcs	r2, r2
     dba:	0843      	lsrs	r3, r0, #1
     dbc:	428b      	cmp	r3, r1
     dbe:	d301      	bcc.n	dc4 <__udivsi3+0xf0>
     dc0:	004b      	lsls	r3, r1, #1
     dc2:	1ac0      	subs	r0, r0, r3
     dc4:	4152      	adcs	r2, r2
     dc6:	1a41      	subs	r1, r0, r1
     dc8:	d200      	bcs.n	dcc <__udivsi3+0xf8>
     dca:	4601      	mov	r1, r0
     dcc:	4152      	adcs	r2, r2
     dce:	4610      	mov	r0, r2
     dd0:	4770      	bx	lr
     dd2:	e7ff      	b.n	dd4 <__udivsi3+0x100>
     dd4:	b501      	push	{r0, lr}
     dd6:	2000      	movs	r0, #0
     dd8:	f000 f806 	bl	de8 <__aeabi_idiv0>
     ddc:	bd02      	pop	{r1, pc}
     dde:	46c0      	nop			; (mov r8, r8)

00000de0 <__aeabi_uidivmod>:
     de0:	2900      	cmp	r1, #0
     de2:	d0f7      	beq.n	dd4 <__udivsi3+0x100>
     de4:	e776      	b.n	cd4 <__udivsi3>
     de6:	4770      	bx	lr

00000de8 <__aeabi_idiv0>:
     de8:	4770      	bx	lr
     dea:	46c0      	nop			; (mov r8, r8)

00000dec <__libc_init_array>:
     dec:	b570      	push	{r4, r5, r6, lr}
     dee:	4e0d      	ldr	r6, [pc, #52]	; (e24 <__libc_init_array+0x38>)
     df0:	4d0d      	ldr	r5, [pc, #52]	; (e28 <__libc_init_array+0x3c>)
     df2:	2400      	movs	r4, #0
     df4:	1bad      	subs	r5, r5, r6
     df6:	10ad      	asrs	r5, r5, #2
     df8:	d005      	beq.n	e06 <__libc_init_array+0x1a>
     dfa:	00a3      	lsls	r3, r4, #2
     dfc:	58f3      	ldr	r3, [r6, r3]
     dfe:	3401      	adds	r4, #1
     e00:	4798      	blx	r3
     e02:	42a5      	cmp	r5, r4
     e04:	d1f9      	bne.n	dfa <__libc_init_array+0xe>
     e06:	f000 fd3d 	bl	1884 <_init>
     e0a:	4e08      	ldr	r6, [pc, #32]	; (e2c <__libc_init_array+0x40>)
     e0c:	4d08      	ldr	r5, [pc, #32]	; (e30 <__libc_init_array+0x44>)
     e0e:	2400      	movs	r4, #0
     e10:	1bad      	subs	r5, r5, r6
     e12:	10ad      	asrs	r5, r5, #2
     e14:	d005      	beq.n	e22 <__libc_init_array+0x36>
     e16:	00a3      	lsls	r3, r4, #2
     e18:	58f3      	ldr	r3, [r6, r3]
     e1a:	3401      	adds	r4, #1
     e1c:	4798      	blx	r3
     e1e:	42a5      	cmp	r5, r4
     e20:	d1f9      	bne.n	e16 <__libc_init_array+0x2a>
     e22:	bd70      	pop	{r4, r5, r6, pc}
     e24:	00001890 	.word	0x00001890
     e28:	00001890 	.word	0x00001890
     e2c:	00001890 	.word	0x00001890
     e30:	0000189c 	.word	0x0000189c

00000e34 <__retarget_lock_acquire_recursive>:
     e34:	4770      	bx	lr
     e36:	46c0      	nop			; (mov r8, r8)

00000e38 <__retarget_lock_release_recursive>:
     e38:	4770      	bx	lr
     e3a:	46c0      	nop			; (mov r8, r8)

00000e3c <malloc>:
     e3c:	b510      	push	{r4, lr}
     e3e:	4b03      	ldr	r3, [pc, #12]	; (e4c <malloc+0x10>)
     e40:	0001      	movs	r1, r0
     e42:	6818      	ldr	r0, [r3, #0]
     e44:	f000 f804 	bl	e50 <_malloc_r>
     e48:	bd10      	pop	{r4, pc}
     e4a:	46c0      	nop			; (mov r8, r8)
     e4c:	20000010 	.word	0x20000010

00000e50 <_malloc_r>:
     e50:	b5f0      	push	{r4, r5, r6, r7, lr}
     e52:	4657      	mov	r7, sl
     e54:	4645      	mov	r5, r8
     e56:	46de      	mov	lr, fp
     e58:	464e      	mov	r6, r9
     e5a:	b5e0      	push	{r5, r6, r7, lr}
     e5c:	000d      	movs	r5, r1
     e5e:	350b      	adds	r5, #11
     e60:	b083      	sub	sp, #12
     e62:	0007      	movs	r7, r0
     e64:	2d16      	cmp	r5, #22
     e66:	d800      	bhi.n	e6a <_malloc_r+0x1a>
     e68:	e09f      	b.n	faa <_malloc_r+0x15a>
     e6a:	2307      	movs	r3, #7
     e6c:	439d      	bics	r5, r3
     e6e:	d500      	bpl.n	e72 <_malloc_r+0x22>
     e70:	e0c4      	b.n	ffc <_malloc_r+0x1ac>
     e72:	42a9      	cmp	r1, r5
     e74:	d900      	bls.n	e78 <_malloc_r+0x28>
     e76:	e0c1      	b.n	ffc <_malloc_r+0x1ac>
     e78:	f000 fa9e 	bl	13b8 <__malloc_lock>
     e7c:	23f8      	movs	r3, #248	; 0xf8
     e7e:	33ff      	adds	r3, #255	; 0xff
     e80:	429d      	cmp	r5, r3
     e82:	d800      	bhi.n	e86 <_malloc_r+0x36>
     e84:	e28f      	b.n	13a6 <_malloc_r+0x556>
     e86:	0a68      	lsrs	r0, r5, #9
     e88:	d100      	bne.n	e8c <_malloc_r+0x3c>
     e8a:	e0bb      	b.n	1004 <_malloc_r+0x1b4>
     e8c:	2804      	cmp	r0, #4
     e8e:	d900      	bls.n	e92 <_malloc_r+0x42>
     e90:	e162      	b.n	1158 <_malloc_r+0x308>
     e92:	2338      	movs	r3, #56	; 0x38
     e94:	4698      	mov	r8, r3
     e96:	09a8      	lsrs	r0, r5, #6
     e98:	4480      	add	r8, r0
     e9a:	3039      	adds	r0, #57	; 0x39
     e9c:	00c1      	lsls	r1, r0, #3
     e9e:	4ed2      	ldr	r6, [pc, #840]	; (11e8 <_malloc_r+0x398>)
     ea0:	1871      	adds	r1, r6, r1
     ea2:	3908      	subs	r1, #8
     ea4:	68cc      	ldr	r4, [r1, #12]
     ea6:	42a1      	cmp	r1, r4
     ea8:	d019      	beq.n	ede <_malloc_r+0x8e>
     eaa:	2303      	movs	r3, #3
     eac:	6862      	ldr	r2, [r4, #4]
     eae:	439a      	bics	r2, r3
     eb0:	0013      	movs	r3, r2
     eb2:	1b52      	subs	r2, r2, r5
     eb4:	2a0f      	cmp	r2, #15
     eb6:	dd00      	ble.n	eba <_malloc_r+0x6a>
     eb8:	e0aa      	b.n	1010 <_malloc_r+0x1c0>
     eba:	2a00      	cmp	r2, #0
     ebc:	db00      	blt.n	ec0 <_malloc_r+0x70>
     ebe:	e088      	b.n	fd2 <_malloc_r+0x182>
     ec0:	2303      	movs	r3, #3
     ec2:	469c      	mov	ip, r3
     ec4:	e008      	b.n	ed8 <_malloc_r+0x88>
     ec6:	4662      	mov	r2, ip
     ec8:	6863      	ldr	r3, [r4, #4]
     eca:	4393      	bics	r3, r2
     ecc:	1b5a      	subs	r2, r3, r5
     ece:	2a0f      	cmp	r2, #15
     ed0:	dd00      	ble.n	ed4 <_malloc_r+0x84>
     ed2:	e09d      	b.n	1010 <_malloc_r+0x1c0>
     ed4:	2a00      	cmp	r2, #0
     ed6:	da7c      	bge.n	fd2 <_malloc_r+0x182>
     ed8:	68e4      	ldr	r4, [r4, #12]
     eda:	42a1      	cmp	r1, r4
     edc:	d1f3      	bne.n	ec6 <_malloc_r+0x76>
     ede:	0032      	movs	r2, r6
     ee0:	6934      	ldr	r4, [r6, #16]
     ee2:	3208      	adds	r2, #8
     ee4:	4294      	cmp	r4, r2
     ee6:	d100      	bne.n	eea <_malloc_r+0x9a>
     ee8:	e190      	b.n	120c <_malloc_r+0x3bc>
     eea:	2303      	movs	r3, #3
     eec:	6861      	ldr	r1, [r4, #4]
     eee:	4399      	bics	r1, r3
     ef0:	4689      	mov	r9, r1
     ef2:	1b49      	subs	r1, r1, r5
     ef4:	290f      	cmp	r1, #15
     ef6:	dd00      	ble.n	efa <_malloc_r+0xaa>
     ef8:	e162      	b.n	11c0 <_malloc_r+0x370>
     efa:	6172      	str	r2, [r6, #20]
     efc:	6132      	str	r2, [r6, #16]
     efe:	2900      	cmp	r1, #0
     f00:	db00      	blt.n	f04 <_malloc_r+0xb4>
     f02:	e087      	b.n	1014 <_malloc_r+0x1c4>
     f04:	4ab9      	ldr	r2, [pc, #740]	; (11ec <_malloc_r+0x39c>)
     f06:	464b      	mov	r3, r9
     f08:	4591      	cmp	r9, r2
     f0a:	d900      	bls.n	f0e <_malloc_r+0xbe>
     f0c:	e130      	b.n	1170 <_malloc_r+0x320>
     f0e:	08db      	lsrs	r3, r3, #3
     f10:	3aff      	subs	r2, #255	; 0xff
     f12:	1099      	asrs	r1, r3, #2
     f14:	3aff      	subs	r2, #255	; 0xff
     f16:	408a      	lsls	r2, r1
     f18:	00db      	lsls	r3, r3, #3
     f1a:	6871      	ldr	r1, [r6, #4]
     f1c:	199b      	adds	r3, r3, r6
     f1e:	430a      	orrs	r2, r1
     f20:	6899      	ldr	r1, [r3, #8]
     f22:	6072      	str	r2, [r6, #4]
     f24:	60e3      	str	r3, [r4, #12]
     f26:	60a1      	str	r1, [r4, #8]
     f28:	609c      	str	r4, [r3, #8]
     f2a:	0013      	movs	r3, r2
     f2c:	60cc      	str	r4, [r1, #12]
     f2e:	2101      	movs	r1, #1
     f30:	1082      	asrs	r2, r0, #2
     f32:	4091      	lsls	r1, r2
     f34:	4299      	cmp	r1, r3
     f36:	d86f      	bhi.n	1018 <_malloc_r+0x1c8>
     f38:	420b      	tst	r3, r1
     f3a:	d105      	bne.n	f48 <_malloc_r+0xf8>
     f3c:	2203      	movs	r2, #3
     f3e:	4390      	bics	r0, r2
     f40:	0049      	lsls	r1, r1, #1
     f42:	3004      	adds	r0, #4
     f44:	420b      	tst	r3, r1
     f46:	d0fb      	beq.n	f40 <_malloc_r+0xf0>
     f48:	2303      	movs	r3, #3
     f4a:	4698      	mov	r8, r3
     f4c:	00c3      	lsls	r3, r0, #3
     f4e:	4699      	mov	r9, r3
     f50:	44b1      	add	r9, r6
     f52:	46cc      	mov	ip, r9
     f54:	4682      	mov	sl, r0
     f56:	4663      	mov	r3, ip
     f58:	68dc      	ldr	r4, [r3, #12]
     f5a:	45a4      	cmp	ip, r4
     f5c:	d107      	bne.n	f6e <_malloc_r+0x11e>
     f5e:	e157      	b.n	1210 <_malloc_r+0x3c0>
     f60:	2a00      	cmp	r2, #0
     f62:	db00      	blt.n	f66 <_malloc_r+0x116>
     f64:	e166      	b.n	1234 <_malloc_r+0x3e4>
     f66:	68e4      	ldr	r4, [r4, #12]
     f68:	45a4      	cmp	ip, r4
     f6a:	d100      	bne.n	f6e <_malloc_r+0x11e>
     f6c:	e150      	b.n	1210 <_malloc_r+0x3c0>
     f6e:	4642      	mov	r2, r8
     f70:	6863      	ldr	r3, [r4, #4]
     f72:	4393      	bics	r3, r2
     f74:	1b5a      	subs	r2, r3, r5
     f76:	2a0f      	cmp	r2, #15
     f78:	ddf2      	ble.n	f60 <_malloc_r+0x110>
     f7a:	2001      	movs	r0, #1
     f7c:	4680      	mov	r8, r0
     f7e:	1961      	adds	r1, r4, r5
     f80:	4305      	orrs	r5, r0
     f82:	6065      	str	r5, [r4, #4]
     f84:	68a0      	ldr	r0, [r4, #8]
     f86:	68e5      	ldr	r5, [r4, #12]
     f88:	3608      	adds	r6, #8
     f8a:	60c5      	str	r5, [r0, #12]
     f8c:	60a8      	str	r0, [r5, #8]
     f8e:	4640      	mov	r0, r8
     f90:	60f1      	str	r1, [r6, #12]
     f92:	60b1      	str	r1, [r6, #8]
     f94:	4310      	orrs	r0, r2
     f96:	6048      	str	r0, [r1, #4]
     f98:	60ce      	str	r6, [r1, #12]
     f9a:	608e      	str	r6, [r1, #8]
     f9c:	0038      	movs	r0, r7
     f9e:	50e2      	str	r2, [r4, r3]
     fa0:	f000 fa12 	bl	13c8 <__malloc_unlock>
     fa4:	0020      	movs	r0, r4
     fa6:	3008      	adds	r0, #8
     fa8:	e021      	b.n	fee <_malloc_r+0x19e>
     faa:	2910      	cmp	r1, #16
     fac:	d826      	bhi.n	ffc <_malloc_r+0x1ac>
     fae:	0038      	movs	r0, r7
     fb0:	f000 fa02 	bl	13b8 <__malloc_lock>
     fb4:	2510      	movs	r5, #16
     fb6:	2318      	movs	r3, #24
     fb8:	2002      	movs	r0, #2
     fba:	4e8b      	ldr	r6, [pc, #556]	; (11e8 <_malloc_r+0x398>)
     fbc:	18f3      	adds	r3, r6, r3
     fbe:	001a      	movs	r2, r3
     fc0:	685c      	ldr	r4, [r3, #4]
     fc2:	3a08      	subs	r2, #8
     fc4:	4294      	cmp	r4, r2
     fc6:	d100      	bne.n	fca <_malloc_r+0x17a>
     fc8:	e12e      	b.n	1228 <_malloc_r+0x3d8>
     fca:	2303      	movs	r3, #3
     fcc:	6862      	ldr	r2, [r4, #4]
     fce:	439a      	bics	r2, r3
     fd0:	0013      	movs	r3, r2
     fd2:	68e2      	ldr	r2, [r4, #12]
     fd4:	68a1      	ldr	r1, [r4, #8]
     fd6:	60ca      	str	r2, [r1, #12]
     fd8:	6091      	str	r1, [r2, #8]
     fda:	2201      	movs	r2, #1
     fdc:	18e3      	adds	r3, r4, r3
     fde:	6859      	ldr	r1, [r3, #4]
     fe0:	0038      	movs	r0, r7
     fe2:	430a      	orrs	r2, r1
     fe4:	605a      	str	r2, [r3, #4]
     fe6:	f000 f9ef 	bl	13c8 <__malloc_unlock>
     fea:	0020      	movs	r0, r4
     fec:	3008      	adds	r0, #8
     fee:	b003      	add	sp, #12
     ff0:	bc3c      	pop	{r2, r3, r4, r5}
     ff2:	4690      	mov	r8, r2
     ff4:	4699      	mov	r9, r3
     ff6:	46a2      	mov	sl, r4
     ff8:	46ab      	mov	fp, r5
     ffa:	bdf0      	pop	{r4, r5, r6, r7, pc}
     ffc:	230c      	movs	r3, #12
     ffe:	2000      	movs	r0, #0
    1000:	603b      	str	r3, [r7, #0]
    1002:	e7f4      	b.n	fee <_malloc_r+0x19e>
    1004:	2180      	movs	r1, #128	; 0x80
    1006:	233f      	movs	r3, #63	; 0x3f
    1008:	2040      	movs	r0, #64	; 0x40
    100a:	0089      	lsls	r1, r1, #2
    100c:	4698      	mov	r8, r3
    100e:	e746      	b.n	e9e <_malloc_r+0x4e>
    1010:	4640      	mov	r0, r8
    1012:	e764      	b.n	ede <_malloc_r+0x8e>
    1014:	464b      	mov	r3, r9
    1016:	e7e0      	b.n	fda <_malloc_r+0x18a>
    1018:	2303      	movs	r3, #3
    101a:	68b4      	ldr	r4, [r6, #8]
    101c:	6862      	ldr	r2, [r4, #4]
    101e:	439a      	bics	r2, r3
    1020:	4690      	mov	r8, r2
    1022:	42aa      	cmp	r2, r5
    1024:	d303      	bcc.n	102e <_malloc_r+0x1de>
    1026:	1b53      	subs	r3, r2, r5
    1028:	2b0f      	cmp	r3, #15
    102a:	dd00      	ble.n	102e <_malloc_r+0x1de>
    102c:	e086      	b.n	113c <_malloc_r+0x2ec>
    102e:	0023      	movs	r3, r4
    1030:	4443      	add	r3, r8
    1032:	4a6f      	ldr	r2, [pc, #444]	; (11f0 <_malloc_r+0x3a0>)
    1034:	9301      	str	r3, [sp, #4]
    1036:	4b6f      	ldr	r3, [pc, #444]	; (11f4 <_malloc_r+0x3a4>)
    1038:	4693      	mov	fp, r2
    103a:	681b      	ldr	r3, [r3, #0]
    103c:	6812      	ldr	r2, [r2, #0]
    103e:	18eb      	adds	r3, r5, r3
    1040:	3201      	adds	r2, #1
    1042:	d100      	bne.n	1046 <_malloc_r+0x1f6>
    1044:	e168      	b.n	1318 <_malloc_r+0x4c8>
    1046:	4a6c      	ldr	r2, [pc, #432]	; (11f8 <_malloc_r+0x3a8>)
    1048:	4694      	mov	ip, r2
    104a:	4463      	add	r3, ip
    104c:	0b1b      	lsrs	r3, r3, #12
    104e:	031b      	lsls	r3, r3, #12
    1050:	9300      	str	r3, [sp, #0]
    1052:	9900      	ldr	r1, [sp, #0]
    1054:	0038      	movs	r0, r7
    1056:	f000 f9bf 	bl	13d8 <_sbrk_r>
    105a:	0003      	movs	r3, r0
    105c:	4681      	mov	r9, r0
    105e:	3301      	adds	r3, #1
    1060:	d061      	beq.n	1126 <_malloc_r+0x2d6>
    1062:	9b01      	ldr	r3, [sp, #4]
    1064:	4283      	cmp	r3, r0
    1066:	d900      	bls.n	106a <_malloc_r+0x21a>
    1068:	e0ff      	b.n	126a <_malloc_r+0x41a>
    106a:	4b64      	ldr	r3, [pc, #400]	; (11fc <_malloc_r+0x3ac>)
    106c:	9a00      	ldr	r2, [sp, #0]
    106e:	469a      	mov	sl, r3
    1070:	681b      	ldr	r3, [r3, #0]
    1072:	469c      	mov	ip, r3
    1074:	4653      	mov	r3, sl
    1076:	4462      	add	r2, ip
    1078:	601a      	str	r2, [r3, #0]
    107a:	9b01      	ldr	r3, [sp, #4]
    107c:	0011      	movs	r1, r2
    107e:	4283      	cmp	r3, r0
    1080:	d100      	bne.n	1084 <_malloc_r+0x234>
    1082:	e155      	b.n	1330 <_malloc_r+0x4e0>
    1084:	465b      	mov	r3, fp
    1086:	681b      	ldr	r3, [r3, #0]
    1088:	3301      	adds	r3, #1
    108a:	d100      	bne.n	108e <_malloc_r+0x23e>
    108c:	e16c      	b.n	1368 <_malloc_r+0x518>
    108e:	464b      	mov	r3, r9
    1090:	9a01      	ldr	r2, [sp, #4]
    1092:	1a9b      	subs	r3, r3, r2
    1094:	1859      	adds	r1, r3, r1
    1096:	4653      	mov	r3, sl
    1098:	6019      	str	r1, [r3, #0]
    109a:	2307      	movs	r3, #7
    109c:	464a      	mov	r2, r9
    109e:	4013      	ands	r3, r2
    10a0:	d100      	bne.n	10a4 <_malloc_r+0x254>
    10a2:	e124      	b.n	12ee <_malloc_r+0x49e>
    10a4:	2108      	movs	r1, #8
    10a6:	4689      	mov	r9, r1
    10a8:	4955      	ldr	r1, [pc, #340]	; (1200 <_malloc_r+0x3b0>)
    10aa:	1ad2      	subs	r2, r2, r3
    10ac:	4491      	add	r9, r2
    10ae:	1acb      	subs	r3, r1, r3
    10b0:	9a00      	ldr	r2, [sp, #0]
    10b2:	0038      	movs	r0, r7
    10b4:	444a      	add	r2, r9
    10b6:	0511      	lsls	r1, r2, #20
    10b8:	0d09      	lsrs	r1, r1, #20
    10ba:	1a5b      	subs	r3, r3, r1
    10bc:	0019      	movs	r1, r3
    10be:	469b      	mov	fp, r3
    10c0:	f000 f98a 	bl	13d8 <_sbrk_r>
    10c4:	1c43      	adds	r3, r0, #1
    10c6:	d100      	bne.n	10ca <_malloc_r+0x27a>
    10c8:	e142      	b.n	1350 <_malloc_r+0x500>
    10ca:	464b      	mov	r3, r9
    10cc:	1ac0      	subs	r0, r0, r3
    10ce:	2301      	movs	r3, #1
    10d0:	4458      	add	r0, fp
    10d2:	4318      	orrs	r0, r3
    10d4:	4653      	mov	r3, sl
    10d6:	681b      	ldr	r3, [r3, #0]
    10d8:	445b      	add	r3, fp
    10da:	0019      	movs	r1, r3
    10dc:	4653      	mov	r3, sl
    10de:	6019      	str	r1, [r3, #0]
    10e0:	464b      	mov	r3, r9
    10e2:	60b3      	str	r3, [r6, #8]
    10e4:	6058      	str	r0, [r3, #4]
    10e6:	42b4      	cmp	r4, r6
    10e8:	d013      	beq.n	1112 <_malloc_r+0x2c2>
    10ea:	4643      	mov	r3, r8
    10ec:	2b0f      	cmp	r3, #15
    10ee:	d800      	bhi.n	10f2 <_malloc_r+0x2a2>
    10f0:	e0e8      	b.n	12c4 <_malloc_r+0x474>
    10f2:	4643      	mov	r3, r8
    10f4:	2207      	movs	r2, #7
    10f6:	6860      	ldr	r0, [r4, #4]
    10f8:	3b0c      	subs	r3, #12
    10fa:	4393      	bics	r3, r2
    10fc:	3a06      	subs	r2, #6
    10fe:	4002      	ands	r2, r0
    1100:	2005      	movs	r0, #5
    1102:	431a      	orrs	r2, r3
    1104:	6062      	str	r2, [r4, #4]
    1106:	18e2      	adds	r2, r4, r3
    1108:	6050      	str	r0, [r2, #4]
    110a:	6090      	str	r0, [r2, #8]
    110c:	2b0f      	cmp	r3, #15
    110e:	d900      	bls.n	1112 <_malloc_r+0x2c2>
    1110:	e122      	b.n	1358 <_malloc_r+0x508>
    1112:	4b3c      	ldr	r3, [pc, #240]	; (1204 <_malloc_r+0x3b4>)
    1114:	681a      	ldr	r2, [r3, #0]
    1116:	4291      	cmp	r1, r2
    1118:	d900      	bls.n	111c <_malloc_r+0x2cc>
    111a:	6019      	str	r1, [r3, #0]
    111c:	4b3a      	ldr	r3, [pc, #232]	; (1208 <_malloc_r+0x3b8>)
    111e:	681a      	ldr	r2, [r3, #0]
    1120:	4291      	cmp	r1, r2
    1122:	d900      	bls.n	1126 <_malloc_r+0x2d6>
    1124:	6019      	str	r1, [r3, #0]
    1126:	2303      	movs	r3, #3
    1128:	68b4      	ldr	r4, [r6, #8]
    112a:	6862      	ldr	r2, [r4, #4]
    112c:	439a      	bics	r2, r3
    112e:	1b53      	subs	r3, r2, r5
    1130:	4295      	cmp	r5, r2
    1132:	d900      	bls.n	1136 <_malloc_r+0x2e6>
    1134:	e0c9      	b.n	12ca <_malloc_r+0x47a>
    1136:	2b0f      	cmp	r3, #15
    1138:	dc00      	bgt.n	113c <_malloc_r+0x2ec>
    113a:	e0c6      	b.n	12ca <_malloc_r+0x47a>
    113c:	2201      	movs	r2, #1
    113e:	0029      	movs	r1, r5
    1140:	4313      	orrs	r3, r2
    1142:	4311      	orrs	r1, r2
    1144:	1965      	adds	r5, r4, r5
    1146:	6061      	str	r1, [r4, #4]
    1148:	0038      	movs	r0, r7
    114a:	60b5      	str	r5, [r6, #8]
    114c:	606b      	str	r3, [r5, #4]
    114e:	f000 f93b 	bl	13c8 <__malloc_unlock>
    1152:	0020      	movs	r0, r4
    1154:	3008      	adds	r0, #8
    1156:	e74a      	b.n	fee <_malloc_r+0x19e>
    1158:	2814      	cmp	r0, #20
    115a:	d97a      	bls.n	1252 <_malloc_r+0x402>
    115c:	2854      	cmp	r0, #84	; 0x54
    115e:	d900      	bls.n	1162 <_malloc_r+0x312>
    1160:	e0ba      	b.n	12d8 <_malloc_r+0x488>
    1162:	236e      	movs	r3, #110	; 0x6e
    1164:	4698      	mov	r8, r3
    1166:	0b28      	lsrs	r0, r5, #12
    1168:	4480      	add	r8, r0
    116a:	306f      	adds	r0, #111	; 0x6f
    116c:	00c1      	lsls	r1, r0, #3
    116e:	e696      	b.n	e9e <_malloc_r+0x4e>
    1170:	0a5a      	lsrs	r2, r3, #9
    1172:	2a04      	cmp	r2, #4
    1174:	d973      	bls.n	125e <_malloc_r+0x40e>
    1176:	2a14      	cmp	r2, #20
    1178:	d900      	bls.n	117c <_malloc_r+0x32c>
    117a:	e0d0      	b.n	131e <_malloc_r+0x4ce>
    117c:	0011      	movs	r1, r2
    117e:	325c      	adds	r2, #92	; 0x5c
    1180:	315b      	adds	r1, #91	; 0x5b
    1182:	00d2      	lsls	r2, r2, #3
    1184:	2308      	movs	r3, #8
    1186:	425b      	negs	r3, r3
    1188:	469c      	mov	ip, r3
    118a:	18b2      	adds	r2, r6, r2
    118c:	4494      	add	ip, r2
    118e:	4663      	mov	r3, ip
    1190:	689a      	ldr	r2, [r3, #8]
    1192:	2303      	movs	r3, #3
    1194:	4698      	mov	r8, r3
    1196:	4594      	cmp	ip, r2
    1198:	d100      	bne.n	119c <_malloc_r+0x34c>
    119a:	e0ab      	b.n	12f4 <_malloc_r+0x4a4>
    119c:	4643      	mov	r3, r8
    119e:	6851      	ldr	r1, [r2, #4]
    11a0:	4399      	bics	r1, r3
    11a2:	4589      	cmp	r9, r1
    11a4:	d300      	bcc.n	11a8 <_malloc_r+0x358>
    11a6:	e095      	b.n	12d4 <_malloc_r+0x484>
    11a8:	6892      	ldr	r2, [r2, #8]
    11aa:	4594      	cmp	ip, r2
    11ac:	d1f6      	bne.n	119c <_malloc_r+0x34c>
    11ae:	4663      	mov	r3, ip
    11b0:	68da      	ldr	r2, [r3, #12]
    11b2:	6873      	ldr	r3, [r6, #4]
    11b4:	4661      	mov	r1, ip
    11b6:	60e2      	str	r2, [r4, #12]
    11b8:	60a1      	str	r1, [r4, #8]
    11ba:	6094      	str	r4, [r2, #8]
    11bc:	60cc      	str	r4, [r1, #12]
    11be:	e6b6      	b.n	f2e <_malloc_r+0xde>
    11c0:	2301      	movs	r3, #1
    11c2:	1960      	adds	r0, r4, r5
    11c4:	431d      	orrs	r5, r3
    11c6:	6065      	str	r5, [r4, #4]
    11c8:	6170      	str	r0, [r6, #20]
    11ca:	6130      	str	r0, [r6, #16]
    11cc:	60c2      	str	r2, [r0, #12]
    11ce:	6082      	str	r2, [r0, #8]
    11d0:	001a      	movs	r2, r3
    11d2:	464b      	mov	r3, r9
    11d4:	430a      	orrs	r2, r1
    11d6:	6042      	str	r2, [r0, #4]
    11d8:	0038      	movs	r0, r7
    11da:	50e1      	str	r1, [r4, r3]
    11dc:	f000 f8f4 	bl	13c8 <__malloc_unlock>
    11e0:	0020      	movs	r0, r4
    11e2:	3008      	adds	r0, #8
    11e4:	e703      	b.n	fee <_malloc_r+0x19e>
    11e6:	46c0      	nop			; (mov r8, r8)
    11e8:	20000440 	.word	0x20000440
    11ec:	000001ff 	.word	0x000001ff
    11f0:	20000848 	.word	0x20000848
    11f4:	200008bc 	.word	0x200008bc
    11f8:	0000100f 	.word	0x0000100f
    11fc:	2000088c 	.word	0x2000088c
    1200:	00001008 	.word	0x00001008
    1204:	200008b4 	.word	0x200008b4
    1208:	200008b8 	.word	0x200008b8
    120c:	6873      	ldr	r3, [r6, #4]
    120e:	e68e      	b.n	f2e <_malloc_r+0xde>
    1210:	2308      	movs	r3, #8
    1212:	469b      	mov	fp, r3
    1214:	3b07      	subs	r3, #7
    1216:	44dc      	add	ip, fp
    1218:	469b      	mov	fp, r3
    121a:	44da      	add	sl, fp
    121c:	4643      	mov	r3, r8
    121e:	4652      	mov	r2, sl
    1220:	4213      	tst	r3, r2
    1222:	d000      	beq.n	1226 <_malloc_r+0x3d6>
    1224:	e697      	b.n	f56 <_malloc_r+0x106>
    1226:	e037      	b.n	1298 <_malloc_r+0x448>
    1228:	68dc      	ldr	r4, [r3, #12]
    122a:	3002      	adds	r0, #2
    122c:	42a3      	cmp	r3, r4
    122e:	d100      	bne.n	1232 <_malloc_r+0x3e2>
    1230:	e655      	b.n	ede <_malloc_r+0x8e>
    1232:	e6ca      	b.n	fca <_malloc_r+0x17a>
    1234:	2201      	movs	r2, #1
    1236:	18e3      	adds	r3, r4, r3
    1238:	6859      	ldr	r1, [r3, #4]
    123a:	0038      	movs	r0, r7
    123c:	430a      	orrs	r2, r1
    123e:	605a      	str	r2, [r3, #4]
    1240:	68e3      	ldr	r3, [r4, #12]
    1242:	68a2      	ldr	r2, [r4, #8]
    1244:	60d3      	str	r3, [r2, #12]
    1246:	609a      	str	r2, [r3, #8]
    1248:	f000 f8be 	bl	13c8 <__malloc_unlock>
    124c:	0020      	movs	r0, r4
    124e:	3008      	adds	r0, #8
    1250:	e6cd      	b.n	fee <_malloc_r+0x19e>
    1252:	235b      	movs	r3, #91	; 0x5b
    1254:	4698      	mov	r8, r3
    1256:	4480      	add	r8, r0
    1258:	305c      	adds	r0, #92	; 0x5c
    125a:	00c1      	lsls	r1, r0, #3
    125c:	e61f      	b.n	e9e <_malloc_r+0x4e>
    125e:	099a      	lsrs	r2, r3, #6
    1260:	0011      	movs	r1, r2
    1262:	3239      	adds	r2, #57	; 0x39
    1264:	3138      	adds	r1, #56	; 0x38
    1266:	00d2      	lsls	r2, r2, #3
    1268:	e78c      	b.n	1184 <_malloc_r+0x334>
    126a:	42b4      	cmp	r4, r6
    126c:	d000      	beq.n	1270 <_malloc_r+0x420>
    126e:	e75a      	b.n	1126 <_malloc_r+0x2d6>
    1270:	4b4f      	ldr	r3, [pc, #316]	; (13b0 <_malloc_r+0x560>)
    1272:	9a00      	ldr	r2, [sp, #0]
    1274:	469a      	mov	sl, r3
    1276:	681b      	ldr	r3, [r3, #0]
    1278:	469c      	mov	ip, r3
    127a:	4653      	mov	r3, sl
    127c:	4462      	add	r2, ip
    127e:	0011      	movs	r1, r2
    1280:	601a      	str	r2, [r3, #0]
    1282:	e6ff      	b.n	1084 <_malloc_r+0x234>
    1284:	2308      	movs	r3, #8
    1286:	425b      	negs	r3, r3
    1288:	469c      	mov	ip, r3
    128a:	44e1      	add	r9, ip
    128c:	464b      	mov	r3, r9
    128e:	689b      	ldr	r3, [r3, #8]
    1290:	3801      	subs	r0, #1
    1292:	4599      	cmp	r9, r3
    1294:	d000      	beq.n	1298 <_malloc_r+0x448>
    1296:	e084      	b.n	13a2 <_malloc_r+0x552>
    1298:	4643      	mov	r3, r8
    129a:	4203      	tst	r3, r0
    129c:	d1f2      	bne.n	1284 <_malloc_r+0x434>
    129e:	6873      	ldr	r3, [r6, #4]
    12a0:	438b      	bics	r3, r1
    12a2:	6073      	str	r3, [r6, #4]
    12a4:	0049      	lsls	r1, r1, #1
    12a6:	4299      	cmp	r1, r3
    12a8:	d900      	bls.n	12ac <_malloc_r+0x45c>
    12aa:	e6b5      	b.n	1018 <_malloc_r+0x1c8>
    12ac:	2900      	cmp	r1, #0
    12ae:	d100      	bne.n	12b2 <_malloc_r+0x462>
    12b0:	e6b2      	b.n	1018 <_malloc_r+0x1c8>
    12b2:	4650      	mov	r0, sl
    12b4:	420b      	tst	r3, r1
    12b6:	d000      	beq.n	12ba <_malloc_r+0x46a>
    12b8:	e648      	b.n	f4c <_malloc_r+0xfc>
    12ba:	0049      	lsls	r1, r1, #1
    12bc:	3004      	adds	r0, #4
    12be:	420b      	tst	r3, r1
    12c0:	d0fb      	beq.n	12ba <_malloc_r+0x46a>
    12c2:	e643      	b.n	f4c <_malloc_r+0xfc>
    12c4:	2301      	movs	r3, #1
    12c6:	464a      	mov	r2, r9
    12c8:	6053      	str	r3, [r2, #4]
    12ca:	0038      	movs	r0, r7
    12cc:	f000 f87c 	bl	13c8 <__malloc_unlock>
    12d0:	2000      	movs	r0, #0
    12d2:	e68c      	b.n	fee <_malloc_r+0x19e>
    12d4:	4694      	mov	ip, r2
    12d6:	e76a      	b.n	11ae <_malloc_r+0x35e>
    12d8:	23aa      	movs	r3, #170	; 0xaa
    12da:	005b      	lsls	r3, r3, #1
    12dc:	4298      	cmp	r0, r3
    12de:	d811      	bhi.n	1304 <_malloc_r+0x4b4>
    12e0:	3bdd      	subs	r3, #221	; 0xdd
    12e2:	4698      	mov	r8, r3
    12e4:	0be8      	lsrs	r0, r5, #15
    12e6:	4480      	add	r8, r0
    12e8:	3078      	adds	r0, #120	; 0x78
    12ea:	00c1      	lsls	r1, r0, #3
    12ec:	e5d7      	b.n	e9e <_malloc_r+0x4e>
    12ee:	2380      	movs	r3, #128	; 0x80
    12f0:	015b      	lsls	r3, r3, #5
    12f2:	e6dd      	b.n	10b0 <_malloc_r+0x260>
    12f4:	1089      	asrs	r1, r1, #2
    12f6:	3b02      	subs	r3, #2
    12f8:	408b      	lsls	r3, r1
    12fa:	6872      	ldr	r2, [r6, #4]
    12fc:	4313      	orrs	r3, r2
    12fe:	6073      	str	r3, [r6, #4]
    1300:	4662      	mov	r2, ip
    1302:	e757      	b.n	11b4 <_malloc_r+0x364>
    1304:	4b2b      	ldr	r3, [pc, #172]	; (13b4 <_malloc_r+0x564>)
    1306:	4298      	cmp	r0, r3
    1308:	d81c      	bhi.n	1344 <_malloc_r+0x4f4>
    130a:	237c      	movs	r3, #124	; 0x7c
    130c:	4698      	mov	r8, r3
    130e:	0ca8      	lsrs	r0, r5, #18
    1310:	4480      	add	r8, r0
    1312:	307d      	adds	r0, #125	; 0x7d
    1314:	00c1      	lsls	r1, r0, #3
    1316:	e5c2      	b.n	e9e <_malloc_r+0x4e>
    1318:	3310      	adds	r3, #16
    131a:	9300      	str	r3, [sp, #0]
    131c:	e699      	b.n	1052 <_malloc_r+0x202>
    131e:	2a54      	cmp	r2, #84	; 0x54
    1320:	d826      	bhi.n	1370 <_malloc_r+0x520>
    1322:	464b      	mov	r3, r9
    1324:	0b1a      	lsrs	r2, r3, #12
    1326:	0011      	movs	r1, r2
    1328:	326f      	adds	r2, #111	; 0x6f
    132a:	316e      	adds	r1, #110	; 0x6e
    132c:	00d2      	lsls	r2, r2, #3
    132e:	e729      	b.n	1184 <_malloc_r+0x334>
    1330:	051b      	lsls	r3, r3, #20
    1332:	d000      	beq.n	1336 <_malloc_r+0x4e6>
    1334:	e6a6      	b.n	1084 <_malloc_r+0x234>
    1336:	2001      	movs	r0, #1
    1338:	9b00      	ldr	r3, [sp, #0]
    133a:	68b2      	ldr	r2, [r6, #8]
    133c:	4443      	add	r3, r8
    133e:	4303      	orrs	r3, r0
    1340:	6053      	str	r3, [r2, #4]
    1342:	e6e6      	b.n	1112 <_malloc_r+0x2c2>
    1344:	21fe      	movs	r1, #254	; 0xfe
    1346:	237e      	movs	r3, #126	; 0x7e
    1348:	207f      	movs	r0, #127	; 0x7f
    134a:	0089      	lsls	r1, r1, #2
    134c:	4698      	mov	r8, r3
    134e:	e5a6      	b.n	e9e <_malloc_r+0x4e>
    1350:	2300      	movs	r3, #0
    1352:	2001      	movs	r0, #1
    1354:	469b      	mov	fp, r3
    1356:	e6bd      	b.n	10d4 <_malloc_r+0x284>
    1358:	0021      	movs	r1, r4
    135a:	0038      	movs	r0, r7
    135c:	3108      	adds	r1, #8
    135e:	f000 f8cb 	bl	14f8 <_free_r>
    1362:	4653      	mov	r3, sl
    1364:	6819      	ldr	r1, [r3, #0]
    1366:	e6d4      	b.n	1112 <_malloc_r+0x2c2>
    1368:	465b      	mov	r3, fp
    136a:	464a      	mov	r2, r9
    136c:	601a      	str	r2, [r3, #0]
    136e:	e694      	b.n	109a <_malloc_r+0x24a>
    1370:	21aa      	movs	r1, #170	; 0xaa
    1372:	0049      	lsls	r1, r1, #1
    1374:	428a      	cmp	r2, r1
    1376:	d806      	bhi.n	1386 <_malloc_r+0x536>
    1378:	464b      	mov	r3, r9
    137a:	0bda      	lsrs	r2, r3, #15
    137c:	0011      	movs	r1, r2
    137e:	3278      	adds	r2, #120	; 0x78
    1380:	3177      	adds	r1, #119	; 0x77
    1382:	00d2      	lsls	r2, r2, #3
    1384:	e6fe      	b.n	1184 <_malloc_r+0x334>
    1386:	490b      	ldr	r1, [pc, #44]	; (13b4 <_malloc_r+0x564>)
    1388:	428a      	cmp	r2, r1
    138a:	d806      	bhi.n	139a <_malloc_r+0x54a>
    138c:	464b      	mov	r3, r9
    138e:	0c9a      	lsrs	r2, r3, #18
    1390:	0011      	movs	r1, r2
    1392:	327d      	adds	r2, #125	; 0x7d
    1394:	317c      	adds	r1, #124	; 0x7c
    1396:	00d2      	lsls	r2, r2, #3
    1398:	e6f4      	b.n	1184 <_malloc_r+0x334>
    139a:	22fe      	movs	r2, #254	; 0xfe
    139c:	217e      	movs	r1, #126	; 0x7e
    139e:	0092      	lsls	r2, r2, #2
    13a0:	e6f0      	b.n	1184 <_malloc_r+0x334>
    13a2:	6873      	ldr	r3, [r6, #4]
    13a4:	e77e      	b.n	12a4 <_malloc_r+0x454>
    13a6:	002b      	movs	r3, r5
    13a8:	08e8      	lsrs	r0, r5, #3
    13aa:	3308      	adds	r3, #8
    13ac:	e605      	b.n	fba <_malloc_r+0x16a>
    13ae:	46c0      	nop			; (mov r8, r8)
    13b0:	2000088c 	.word	0x2000088c
    13b4:	00000554 	.word	0x00000554

000013b8 <__malloc_lock>:
    13b8:	b510      	push	{r4, lr}
    13ba:	4802      	ldr	r0, [pc, #8]	; (13c4 <__malloc_lock+0xc>)
    13bc:	f7ff fd3a 	bl	e34 <__retarget_lock_acquire_recursive>
    13c0:	bd10      	pop	{r4, pc}
    13c2:	46c0      	nop			; (mov r8, r8)
    13c4:	20000904 	.word	0x20000904

000013c8 <__malloc_unlock>:
    13c8:	b510      	push	{r4, lr}
    13ca:	4802      	ldr	r0, [pc, #8]	; (13d4 <__malloc_unlock+0xc>)
    13cc:	f7ff fd34 	bl	e38 <__retarget_lock_release_recursive>
    13d0:	bd10      	pop	{r4, pc}
    13d2:	46c0      	nop			; (mov r8, r8)
    13d4:	20000904 	.word	0x20000904

000013d8 <_sbrk_r>:
    13d8:	2300      	movs	r3, #0
    13da:	b570      	push	{r4, r5, r6, lr}
    13dc:	4c06      	ldr	r4, [pc, #24]	; (13f8 <_sbrk_r+0x20>)
    13de:	0005      	movs	r5, r0
    13e0:	0008      	movs	r0, r1
    13e2:	6023      	str	r3, [r4, #0]
    13e4:	f7ff f9d4 	bl	790 <_sbrk>
    13e8:	1c43      	adds	r3, r0, #1
    13ea:	d000      	beq.n	13ee <_sbrk_r+0x16>
    13ec:	bd70      	pop	{r4, r5, r6, pc}
    13ee:	6823      	ldr	r3, [r4, #0]
    13f0:	2b00      	cmp	r3, #0
    13f2:	d0fb      	beq.n	13ec <_sbrk_r+0x14>
    13f4:	602b      	str	r3, [r5, #0]
    13f6:	e7f9      	b.n	13ec <_sbrk_r+0x14>
    13f8:	20000918 	.word	0x20000918

000013fc <register_fini>:
    13fc:	4b03      	ldr	r3, [pc, #12]	; (140c <register_fini+0x10>)
    13fe:	b510      	push	{r4, lr}
    1400:	2b00      	cmp	r3, #0
    1402:	d002      	beq.n	140a <register_fini+0xe>
    1404:	4802      	ldr	r0, [pc, #8]	; (1410 <register_fini+0x14>)
    1406:	f000 f805 	bl	1414 <atexit>
    140a:	bd10      	pop	{r4, pc}
    140c:	00000000 	.word	0x00000000
    1410:	00001425 	.word	0x00001425

00001414 <atexit>:
    1414:	b510      	push	{r4, lr}
    1416:	0001      	movs	r1, r0
    1418:	2300      	movs	r3, #0
    141a:	2200      	movs	r2, #0
    141c:	2000      	movs	r0, #0
    141e:	f000 f949 	bl	16b4 <__register_exitproc>
    1422:	bd10      	pop	{r4, pc}

00001424 <__libc_fini_array>:
    1424:	b570      	push	{r4, r5, r6, lr}
    1426:	4b09      	ldr	r3, [pc, #36]	; (144c <__libc_fini_array+0x28>)
    1428:	4c09      	ldr	r4, [pc, #36]	; (1450 <__libc_fini_array+0x2c>)
    142a:	1ae4      	subs	r4, r4, r3
    142c:	10a4      	asrs	r4, r4, #2
    142e:	d009      	beq.n	1444 <__libc_fini_array+0x20>
    1430:	4a08      	ldr	r2, [pc, #32]	; (1454 <__libc_fini_array+0x30>)
    1432:	18a5      	adds	r5, r4, r2
    1434:	00ad      	lsls	r5, r5, #2
    1436:	18ed      	adds	r5, r5, r3
    1438:	682b      	ldr	r3, [r5, #0]
    143a:	3c01      	subs	r4, #1
    143c:	4798      	blx	r3
    143e:	3d04      	subs	r5, #4
    1440:	2c00      	cmp	r4, #0
    1442:	d1f9      	bne.n	1438 <__libc_fini_array+0x14>
    1444:	f000 fa2a 	bl	189c <_fini>
    1448:	bd70      	pop	{r4, r5, r6, pc}
    144a:	46c0      	nop			; (mov r8, r8)
    144c:	000018a8 	.word	0x000018a8
    1450:	000018ac 	.word	0x000018ac
    1454:	3fffffff 	.word	0x3fffffff

00001458 <_malloc_trim_r>:
    1458:	b5f8      	push	{r3, r4, r5, r6, r7, lr}
    145a:	000c      	movs	r4, r1
    145c:	0006      	movs	r6, r0
    145e:	f7ff ffab 	bl	13b8 <__malloc_lock>
    1462:	4f20      	ldr	r7, [pc, #128]	; (14e4 <_malloc_trim_r+0x8c>)
    1464:	68bb      	ldr	r3, [r7, #8]
    1466:	685d      	ldr	r5, [r3, #4]
    1468:	2303      	movs	r3, #3
    146a:	439d      	bics	r5, r3
    146c:	4b1e      	ldr	r3, [pc, #120]	; (14e8 <_malloc_trim_r+0x90>)
    146e:	1b2c      	subs	r4, r5, r4
    1470:	469c      	mov	ip, r3
    1472:	4464      	add	r4, ip
    1474:	0b24      	lsrs	r4, r4, #12
    1476:	4b1d      	ldr	r3, [pc, #116]	; (14ec <_malloc_trim_r+0x94>)
    1478:	3c01      	subs	r4, #1
    147a:	0324      	lsls	r4, r4, #12
    147c:	429c      	cmp	r4, r3
    147e:	dd07      	ble.n	1490 <_malloc_trim_r+0x38>
    1480:	2100      	movs	r1, #0
    1482:	0030      	movs	r0, r6
    1484:	f7ff ffa8 	bl	13d8 <_sbrk_r>
    1488:	68bb      	ldr	r3, [r7, #8]
    148a:	195b      	adds	r3, r3, r5
    148c:	4298      	cmp	r0, r3
    148e:	d004      	beq.n	149a <_malloc_trim_r+0x42>
    1490:	0030      	movs	r0, r6
    1492:	f7ff ff99 	bl	13c8 <__malloc_unlock>
    1496:	2000      	movs	r0, #0
    1498:	bdf8      	pop	{r3, r4, r5, r6, r7, pc}
    149a:	4261      	negs	r1, r4
    149c:	0030      	movs	r0, r6
    149e:	f7ff ff9b 	bl	13d8 <_sbrk_r>
    14a2:	1c43      	adds	r3, r0, #1
    14a4:	d00d      	beq.n	14c2 <_malloc_trim_r+0x6a>
    14a6:	2201      	movs	r2, #1
    14a8:	68bb      	ldr	r3, [r7, #8]
    14aa:	1b2d      	subs	r5, r5, r4
    14ac:	4315      	orrs	r5, r2
    14ae:	605d      	str	r5, [r3, #4]
    14b0:	4b0f      	ldr	r3, [pc, #60]	; (14f0 <_malloc_trim_r+0x98>)
    14b2:	0030      	movs	r0, r6
    14b4:	681a      	ldr	r2, [r3, #0]
    14b6:	1b14      	subs	r4, r2, r4
    14b8:	601c      	str	r4, [r3, #0]
    14ba:	f7ff ff85 	bl	13c8 <__malloc_unlock>
    14be:	2001      	movs	r0, #1
    14c0:	e7ea      	b.n	1498 <_malloc_trim_r+0x40>
    14c2:	2100      	movs	r1, #0
    14c4:	0030      	movs	r0, r6
    14c6:	f7ff ff87 	bl	13d8 <_sbrk_r>
    14ca:	68ba      	ldr	r2, [r7, #8]
    14cc:	1a83      	subs	r3, r0, r2
    14ce:	2b0f      	cmp	r3, #15
    14d0:	ddde      	ble.n	1490 <_malloc_trim_r+0x38>
    14d2:	4908      	ldr	r1, [pc, #32]	; (14f4 <_malloc_trim_r+0x9c>)
    14d4:	6809      	ldr	r1, [r1, #0]
    14d6:	1a40      	subs	r0, r0, r1
    14d8:	4905      	ldr	r1, [pc, #20]	; (14f0 <_malloc_trim_r+0x98>)
    14da:	6008      	str	r0, [r1, #0]
    14dc:	2101      	movs	r1, #1
    14de:	430b      	orrs	r3, r1
    14e0:	6053      	str	r3, [r2, #4]
    14e2:	e7d5      	b.n	1490 <_malloc_trim_r+0x38>
    14e4:	20000440 	.word	0x20000440
    14e8:	00000fef 	.word	0x00000fef
    14ec:	00000fff 	.word	0x00000fff
    14f0:	2000088c 	.word	0x2000088c
    14f4:	20000848 	.word	0x20000848

000014f8 <_free_r>:
    14f8:	b5f8      	push	{r3, r4, r5, r6, r7, lr}
    14fa:	0004      	movs	r4, r0
    14fc:	1e0d      	subs	r5, r1, #0
    14fe:	d03c      	beq.n	157a <_free_r+0x82>
    1500:	f7ff ff5a 	bl	13b8 <__malloc_lock>
    1504:	0029      	movs	r1, r5
    1506:	3908      	subs	r1, #8
    1508:	6848      	ldr	r0, [r1, #4]
    150a:	2301      	movs	r3, #1
    150c:	0005      	movs	r5, r0
    150e:	2603      	movs	r6, #3
    1510:	439d      	bics	r5, r3
    1512:	194a      	adds	r2, r1, r5
    1514:	469c      	mov	ip, r3
    1516:	4f61      	ldr	r7, [pc, #388]	; (169c <_free_r+0x1a4>)
    1518:	6853      	ldr	r3, [r2, #4]
    151a:	43b3      	bics	r3, r6
    151c:	68be      	ldr	r6, [r7, #8]
    151e:	42b2      	cmp	r2, r6
    1520:	d056      	beq.n	15d0 <_free_r+0xd8>
    1522:	4666      	mov	r6, ip
    1524:	6053      	str	r3, [r2, #4]
    1526:	4206      	tst	r6, r0
    1528:	d10a      	bne.n	1540 <_free_r+0x48>
    152a:	003e      	movs	r6, r7
    152c:	6808      	ldr	r0, [r1, #0]
    152e:	3608      	adds	r6, #8
    1530:	1a09      	subs	r1, r1, r0
    1532:	182d      	adds	r5, r5, r0
    1534:	6888      	ldr	r0, [r1, #8]
    1536:	42b0      	cmp	r0, r6
    1538:	d065      	beq.n	1606 <_free_r+0x10e>
    153a:	68ce      	ldr	r6, [r1, #12]
    153c:	60c6      	str	r6, [r0, #12]
    153e:	60b0      	str	r0, [r6, #8]
    1540:	2001      	movs	r0, #1
    1542:	18d6      	adds	r6, r2, r3
    1544:	6876      	ldr	r6, [r6, #4]
    1546:	4206      	tst	r6, r0
    1548:	d033      	beq.n	15b2 <_free_r+0xba>
    154a:	4b55      	ldr	r3, [pc, #340]	; (16a0 <_free_r+0x1a8>)
    154c:	4328      	orrs	r0, r5
    154e:	6048      	str	r0, [r1, #4]
    1550:	514d      	str	r5, [r1, r5]
    1552:	429d      	cmp	r5, r3
    1554:	d812      	bhi.n	157c <_free_r+0x84>
    1556:	08ed      	lsrs	r5, r5, #3
    1558:	3bff      	subs	r3, #255	; 0xff
    155a:	10aa      	asrs	r2, r5, #2
    155c:	3bff      	subs	r3, #255	; 0xff
    155e:	4093      	lsls	r3, r2
    1560:	687a      	ldr	r2, [r7, #4]
    1562:	00ed      	lsls	r5, r5, #3
    1564:	4313      	orrs	r3, r2
    1566:	607b      	str	r3, [r7, #4]
    1568:	19ef      	adds	r7, r5, r7
    156a:	68bb      	ldr	r3, [r7, #8]
    156c:	60cf      	str	r7, [r1, #12]
    156e:	608b      	str	r3, [r1, #8]
    1570:	60b9      	str	r1, [r7, #8]
    1572:	60d9      	str	r1, [r3, #12]
    1574:	0020      	movs	r0, r4
    1576:	f7ff ff27 	bl	13c8 <__malloc_unlock>
    157a:	bdf8      	pop	{r3, r4, r5, r6, r7, pc}
    157c:	0a68      	lsrs	r0, r5, #9
    157e:	2804      	cmp	r0, #4
    1580:	d850      	bhi.n	1624 <_free_r+0x12c>
    1582:	09a8      	lsrs	r0, r5, #6
    1584:	0002      	movs	r2, r0
    1586:	3039      	adds	r0, #57	; 0x39
    1588:	3238      	adds	r2, #56	; 0x38
    158a:	00c0      	lsls	r0, r0, #3
    158c:	1838      	adds	r0, r7, r0
    158e:	3808      	subs	r0, #8
    1590:	6883      	ldr	r3, [r0, #8]
    1592:	2603      	movs	r6, #3
    1594:	4298      	cmp	r0, r3
    1596:	d04c      	beq.n	1632 <_free_r+0x13a>
    1598:	685a      	ldr	r2, [r3, #4]
    159a:	43b2      	bics	r2, r6
    159c:	4295      	cmp	r5, r2
    159e:	d230      	bcs.n	1602 <_free_r+0x10a>
    15a0:	689b      	ldr	r3, [r3, #8]
    15a2:	4298      	cmp	r0, r3
    15a4:	d1f8      	bne.n	1598 <_free_r+0xa0>
    15a6:	68c3      	ldr	r3, [r0, #12]
    15a8:	60cb      	str	r3, [r1, #12]
    15aa:	6088      	str	r0, [r1, #8]
    15ac:	6099      	str	r1, [r3, #8]
    15ae:	60c1      	str	r1, [r0, #12]
    15b0:	e7e0      	b.n	1574 <_free_r+0x7c>
    15b2:	18ed      	adds	r5, r5, r3
    15b4:	4e3b      	ldr	r6, [pc, #236]	; (16a4 <_free_r+0x1ac>)
    15b6:	6893      	ldr	r3, [r2, #8]
    15b8:	42b3      	cmp	r3, r6
    15ba:	d042      	beq.n	1642 <_free_r+0x14a>
    15bc:	68d2      	ldr	r2, [r2, #12]
    15be:	4328      	orrs	r0, r5
    15c0:	60da      	str	r2, [r3, #12]
    15c2:	6093      	str	r3, [r2, #8]
    15c4:	4b36      	ldr	r3, [pc, #216]	; (16a0 <_free_r+0x1a8>)
    15c6:	6048      	str	r0, [r1, #4]
    15c8:	514d      	str	r5, [r1, r5]
    15ca:	429d      	cmp	r5, r3
    15cc:	d8d6      	bhi.n	157c <_free_r+0x84>
    15ce:	e7c2      	b.n	1556 <_free_r+0x5e>
    15d0:	4662      	mov	r2, ip
    15d2:	18eb      	adds	r3, r5, r3
    15d4:	4202      	tst	r2, r0
    15d6:	d106      	bne.n	15e6 <_free_r+0xee>
    15d8:	680a      	ldr	r2, [r1, #0]
    15da:	1a89      	subs	r1, r1, r2
    15dc:	6888      	ldr	r0, [r1, #8]
    15de:	189b      	adds	r3, r3, r2
    15e0:	68ca      	ldr	r2, [r1, #12]
    15e2:	60c2      	str	r2, [r0, #12]
    15e4:	6090      	str	r0, [r2, #8]
    15e6:	2201      	movs	r2, #1
    15e8:	431a      	orrs	r2, r3
    15ea:	604a      	str	r2, [r1, #4]
    15ec:	4a2e      	ldr	r2, [pc, #184]	; (16a8 <_free_r+0x1b0>)
    15ee:	60b9      	str	r1, [r7, #8]
    15f0:	6812      	ldr	r2, [r2, #0]
    15f2:	4293      	cmp	r3, r2
    15f4:	d3be      	bcc.n	1574 <_free_r+0x7c>
    15f6:	4b2d      	ldr	r3, [pc, #180]	; (16ac <_free_r+0x1b4>)
    15f8:	0020      	movs	r0, r4
    15fa:	6819      	ldr	r1, [r3, #0]
    15fc:	f7ff ff2c 	bl	1458 <_malloc_trim_r>
    1600:	e7b8      	b.n	1574 <_free_r+0x7c>
    1602:	0018      	movs	r0, r3
    1604:	e7cf      	b.n	15a6 <_free_r+0xae>
    1606:	4666      	mov	r6, ip
    1608:	18d0      	adds	r0, r2, r3
    160a:	6840      	ldr	r0, [r0, #4]
    160c:	4230      	tst	r0, r6
    160e:	d13f      	bne.n	1690 <_free_r+0x198>
    1610:	6890      	ldr	r0, [r2, #8]
    1612:	195d      	adds	r5, r3, r5
    1614:	68d3      	ldr	r3, [r2, #12]
    1616:	60c3      	str	r3, [r0, #12]
    1618:	6098      	str	r0, [r3, #8]
    161a:	4663      	mov	r3, ip
    161c:	432b      	orrs	r3, r5
    161e:	604b      	str	r3, [r1, #4]
    1620:	514d      	str	r5, [r1, r5]
    1622:	e7a7      	b.n	1574 <_free_r+0x7c>
    1624:	2814      	cmp	r0, #20
    1626:	d814      	bhi.n	1652 <_free_r+0x15a>
    1628:	0002      	movs	r2, r0
    162a:	305c      	adds	r0, #92	; 0x5c
    162c:	325b      	adds	r2, #91	; 0x5b
    162e:	00c0      	lsls	r0, r0, #3
    1630:	e7ac      	b.n	158c <_free_r+0x94>
    1632:	2301      	movs	r3, #1
    1634:	1092      	asrs	r2, r2, #2
    1636:	4093      	lsls	r3, r2
    1638:	687a      	ldr	r2, [r7, #4]
    163a:	4313      	orrs	r3, r2
    163c:	607b      	str	r3, [r7, #4]
    163e:	0003      	movs	r3, r0
    1640:	e7b2      	b.n	15a8 <_free_r+0xb0>
    1642:	4328      	orrs	r0, r5
    1644:	60d9      	str	r1, [r3, #12]
    1646:	6099      	str	r1, [r3, #8]
    1648:	60cb      	str	r3, [r1, #12]
    164a:	608b      	str	r3, [r1, #8]
    164c:	6048      	str	r0, [r1, #4]
    164e:	514d      	str	r5, [r1, r5]
    1650:	e790      	b.n	1574 <_free_r+0x7c>
    1652:	2854      	cmp	r0, #84	; 0x54
    1654:	d805      	bhi.n	1662 <_free_r+0x16a>
    1656:	0b28      	lsrs	r0, r5, #12
    1658:	0002      	movs	r2, r0
    165a:	306f      	adds	r0, #111	; 0x6f
    165c:	326e      	adds	r2, #110	; 0x6e
    165e:	00c0      	lsls	r0, r0, #3
    1660:	e794      	b.n	158c <_free_r+0x94>
    1662:	22aa      	movs	r2, #170	; 0xaa
    1664:	0052      	lsls	r2, r2, #1
    1666:	4290      	cmp	r0, r2
    1668:	d805      	bhi.n	1676 <_free_r+0x17e>
    166a:	0be8      	lsrs	r0, r5, #15
    166c:	0002      	movs	r2, r0
    166e:	3078      	adds	r0, #120	; 0x78
    1670:	3277      	adds	r2, #119	; 0x77
    1672:	00c0      	lsls	r0, r0, #3
    1674:	e78a      	b.n	158c <_free_r+0x94>
    1676:	4a0e      	ldr	r2, [pc, #56]	; (16b0 <_free_r+0x1b8>)
    1678:	4290      	cmp	r0, r2
    167a:	d805      	bhi.n	1688 <_free_r+0x190>
    167c:	0ca8      	lsrs	r0, r5, #18
    167e:	0002      	movs	r2, r0
    1680:	307d      	adds	r0, #125	; 0x7d
    1682:	327c      	adds	r2, #124	; 0x7c
    1684:	00c0      	lsls	r0, r0, #3
    1686:	e781      	b.n	158c <_free_r+0x94>
    1688:	20fe      	movs	r0, #254	; 0xfe
    168a:	227e      	movs	r2, #126	; 0x7e
    168c:	0080      	lsls	r0, r0, #2
    168e:	e77d      	b.n	158c <_free_r+0x94>
    1690:	4663      	mov	r3, ip
    1692:	432b      	orrs	r3, r5
    1694:	604b      	str	r3, [r1, #4]
    1696:	6015      	str	r5, [r2, #0]
    1698:	e76c      	b.n	1574 <_free_r+0x7c>
    169a:	46c0      	nop			; (mov r8, r8)
    169c:	20000440 	.word	0x20000440
    16a0:	000001ff 	.word	0x000001ff
    16a4:	20000448 	.word	0x20000448
    16a8:	2000084c 	.word	0x2000084c
    16ac:	200008bc 	.word	0x200008bc
    16b0:	00000554 	.word	0x00000554

000016b4 <__register_exitproc>:
    16b4:	b5f0      	push	{r4, r5, r6, r7, lr}
    16b6:	464e      	mov	r6, r9
    16b8:	4645      	mov	r5, r8
    16ba:	46de      	mov	lr, fp
    16bc:	4657      	mov	r7, sl
    16be:	b5e0      	push	{r5, r6, r7, lr}
    16c0:	4d36      	ldr	r5, [pc, #216]	; (179c <__register_exitproc+0xe8>)
    16c2:	b083      	sub	sp, #12
    16c4:	0006      	movs	r6, r0
    16c6:	6828      	ldr	r0, [r5, #0]
    16c8:	4698      	mov	r8, r3
    16ca:	000f      	movs	r7, r1
    16cc:	4691      	mov	r9, r2
    16ce:	f7ff fbb1 	bl	e34 <__retarget_lock_acquire_recursive>
    16d2:	4b33      	ldr	r3, [pc, #204]	; (17a0 <__register_exitproc+0xec>)
    16d4:	681c      	ldr	r4, [r3, #0]
    16d6:	23a4      	movs	r3, #164	; 0xa4
    16d8:	005b      	lsls	r3, r3, #1
    16da:	58e0      	ldr	r0, [r4, r3]
    16dc:	2800      	cmp	r0, #0
    16de:	d052      	beq.n	1786 <__register_exitproc+0xd2>
    16e0:	6843      	ldr	r3, [r0, #4]
    16e2:	2b1f      	cmp	r3, #31
    16e4:	dc13      	bgt.n	170e <__register_exitproc+0x5a>
    16e6:	1c5a      	adds	r2, r3, #1
    16e8:	9201      	str	r2, [sp, #4]
    16ea:	2e00      	cmp	r6, #0
    16ec:	d128      	bne.n	1740 <__register_exitproc+0x8c>
    16ee:	9a01      	ldr	r2, [sp, #4]
    16f0:	3302      	adds	r3, #2
    16f2:	009b      	lsls	r3, r3, #2
    16f4:	6042      	str	r2, [r0, #4]
    16f6:	501f      	str	r7, [r3, r0]
    16f8:	6828      	ldr	r0, [r5, #0]
    16fa:	f7ff fb9d 	bl	e38 <__retarget_lock_release_recursive>
    16fe:	2000      	movs	r0, #0
    1700:	b003      	add	sp, #12
    1702:	bc3c      	pop	{r2, r3, r4, r5}
    1704:	4690      	mov	r8, r2
    1706:	4699      	mov	r9, r3
    1708:	46a2      	mov	sl, r4
    170a:	46ab      	mov	fp, r5
    170c:	bdf0      	pop	{r4, r5, r6, r7, pc}
    170e:	4b25      	ldr	r3, [pc, #148]	; (17a4 <__register_exitproc+0xf0>)
    1710:	2b00      	cmp	r3, #0
    1712:	d03d      	beq.n	1790 <__register_exitproc+0xdc>
    1714:	20c8      	movs	r0, #200	; 0xc8
    1716:	0040      	lsls	r0, r0, #1
    1718:	f7ff fb90 	bl	e3c <malloc>
    171c:	2800      	cmp	r0, #0
    171e:	d037      	beq.n	1790 <__register_exitproc+0xdc>
    1720:	22a4      	movs	r2, #164	; 0xa4
    1722:	2300      	movs	r3, #0
    1724:	0052      	lsls	r2, r2, #1
    1726:	58a1      	ldr	r1, [r4, r2]
    1728:	6043      	str	r3, [r0, #4]
    172a:	6001      	str	r1, [r0, #0]
    172c:	50a0      	str	r0, [r4, r2]
    172e:	3240      	adds	r2, #64	; 0x40
    1730:	5083      	str	r3, [r0, r2]
    1732:	3204      	adds	r2, #4
    1734:	5083      	str	r3, [r0, r2]
    1736:	3301      	adds	r3, #1
    1738:	9301      	str	r3, [sp, #4]
    173a:	2300      	movs	r3, #0
    173c:	2e00      	cmp	r6, #0
    173e:	d0d6      	beq.n	16ee <__register_exitproc+0x3a>
    1740:	009a      	lsls	r2, r3, #2
    1742:	4692      	mov	sl, r2
    1744:	4482      	add	sl, r0
    1746:	464a      	mov	r2, r9
    1748:	2188      	movs	r1, #136	; 0x88
    174a:	4654      	mov	r4, sl
    174c:	5062      	str	r2, [r4, r1]
    174e:	22c4      	movs	r2, #196	; 0xc4
    1750:	0052      	lsls	r2, r2, #1
    1752:	4691      	mov	r9, r2
    1754:	4481      	add	r9, r0
    1756:	464a      	mov	r2, r9
    1758:	3987      	subs	r1, #135	; 0x87
    175a:	4099      	lsls	r1, r3
    175c:	6812      	ldr	r2, [r2, #0]
    175e:	468b      	mov	fp, r1
    1760:	430a      	orrs	r2, r1
    1762:	4694      	mov	ip, r2
    1764:	464a      	mov	r2, r9
    1766:	4661      	mov	r1, ip
    1768:	6011      	str	r1, [r2, #0]
    176a:	2284      	movs	r2, #132	; 0x84
    176c:	4641      	mov	r1, r8
    176e:	0052      	lsls	r2, r2, #1
    1770:	50a1      	str	r1, [r4, r2]
    1772:	2e02      	cmp	r6, #2
    1774:	d1bb      	bne.n	16ee <__register_exitproc+0x3a>
    1776:	0002      	movs	r2, r0
    1778:	465c      	mov	r4, fp
    177a:	328d      	adds	r2, #141	; 0x8d
    177c:	32ff      	adds	r2, #255	; 0xff
    177e:	6811      	ldr	r1, [r2, #0]
    1780:	430c      	orrs	r4, r1
    1782:	6014      	str	r4, [r2, #0]
    1784:	e7b3      	b.n	16ee <__register_exitproc+0x3a>
    1786:	0020      	movs	r0, r4
    1788:	304d      	adds	r0, #77	; 0x4d
    178a:	30ff      	adds	r0, #255	; 0xff
    178c:	50e0      	str	r0, [r4, r3]
    178e:	e7a7      	b.n	16e0 <__register_exitproc+0x2c>
    1790:	6828      	ldr	r0, [r5, #0]
    1792:	f7ff fb51 	bl	e38 <__retarget_lock_release_recursive>
    1796:	2001      	movs	r0, #1
    1798:	4240      	negs	r0, r0
    179a:	e7b1      	b.n	1700 <__register_exitproc+0x4c>
    179c:	20000850 	.word	0x20000850
    17a0:	00001880 	.word	0x00001880
    17a4:	00000e3d 	.word	0x00000e3d
    17a8:	682f2e2e 	.word	0x682f2e2e
    17ac:	732f6c61 	.word	0x732f6c61
    17b0:	682f6372 	.word	0x682f6372
    17b4:	735f6c61 	.word	0x735f6c61
    17b8:	6d5f6970 	.word	0x6d5f6970
    17bc:	6e79735f 	.word	0x6e79735f
    17c0:	00632e63 	.word	0x00632e63
    17c4:	682f2e2e 	.word	0x682f2e2e
    17c8:	732f6c61 	.word	0x732f6c61
    17cc:	682f6372 	.word	0x682f6372
    17d0:	745f6c61 	.word	0x745f6c61
    17d4:	72656d69 	.word	0x72656d69
    17d8:	0000632e 	.word	0x0000632e
    17dc:	682f2e2e 	.word	0x682f2e2e
    17e0:	752f6c61 	.word	0x752f6c61
    17e4:	736c6974 	.word	0x736c6974
    17e8:	6372732f 	.word	0x6372732f
    17ec:	6974752f 	.word	0x6974752f
    17f0:	6c5f736c 	.word	0x6c5f736c
    17f4:	2e747369 	.word	0x2e747369
    17f8:	00000063 	.word	0x00000063
    17fc:	682f2e2e 	.word	0x682f2e2e
    1800:	722f6c70 	.word	0x722f6c70
    1804:	682f6374 	.word	0x682f6374
    1808:	725f6c70 	.word	0x725f6c70
    180c:	632e6374 	.word	0x632e6374
    1810:	00000000 	.word	0x00000000

00001814 <_usarts>:
	...

00001828 <_i2cms>:
	...

00001840 <_i2css>:
	...

00001850 <sercomspi_regs>:
    1850:	0020000c 00020000 00000000 01ff004f     .. .........O...
    1860:	00000000 682f2e2e 732f6c70 6f637265     ....../hpl/serco
    1870:	70682f6d 65735f6c 6d6f6372 0000632e     m/hpl_sercom.c..

00001880 <_global_impure_ptr>:
    1880:	20000018                                ... 

00001884 <_init>:
    1884:	b5f8      	push	{r3, r4, r5, r6, r7, lr}
    1886:	46c0      	nop			; (mov r8, r8)
    1888:	bcf8      	pop	{r3, r4, r5, r6, r7}
    188a:	bc08      	pop	{r3}
    188c:	469e      	mov	lr, r3
    188e:	4770      	bx	lr

00001890 <__init_array_start>:
    1890:	000013fd 	.word	0x000013fd

00001894 <__frame_dummy_init_array_entry>:
    1894:	000000dd 00000ca9                       ........

0000189c <_fini>:
    189c:	b5f8      	push	{r3, r4, r5, r6, r7, lr}
    189e:	46c0      	nop			; (mov r8, r8)
    18a0:	bcf8      	pop	{r3, r4, r5, r6, r7}
    18a2:	bc08      	pop	{r3}
    18a4:	469e      	mov	lr, r3
    18a6:	4770      	bx	lr

000018a8 <__fini_array_start>:
    18a8:	000000b5 	.word	0x000000b5
